:0800000C32322E312E322E316A
:1000000AF51016F83C3117F23743472601262C041F
:1000000A442F3308100E131014121718135A4E40A7
:1000000A0B60535D421A383B1D5D4A393C22293147
:1000000A2B30342F2F3337322F3D35363B3F3A3A98
:1000000A3E423D3A3F494A454A4545494D4845538E
:1000000A53555055505054585350555F5F5B605B81
:1000000A5B5F635E5B62676A666B66666A6E696699
:1000000A896B8D5E9483866C868A6FAF8D72BBAF67
:0B00000AA16CA291947AA4A87DA2A290
:020000040800F2
:40800000C0FC02202DA60A083FA60A0879640C0843A60A0845A60A0847A60A0800000000000000000000000000000000B58300084BA60A080000000079840008ED840008DD
:4080400051A60A0851A60A0851A60A0851A60A0851A60A0851A60A0851A60A0851A60A0851A60A0851A60A0851A60A08B9D80608C3D8060851A60A08CFD80608DBD80608D6
:40808000E7D80608F3D80608FFBB0608B5C106088BC2060851A60A0851A60A0851A60A0851A60A0851A60A0851A60A0851A60A08932507089F25070851A60A08B5130708BA
:4080C000C5130708D5130708DF1307083B24070845240708E1F3060831F406083BF4060851A60A0851A60A0851A60A0851A60A0851A60A0851A60A0851A60A08FFD8060845
:4081000051A60A0851A60A08A92507084F24070845F406084FF4060851A60A08132707080BD9060815D9060821D906082DD9060839D9060851A60A0851A60A081FC20608B9
:4081400011C3060897C3060851A60A0851A60A0845D9060851D906085DD9060859F40608E9130708F913070851A60A0851A60A0851A60A0851A60A0851A60A08000000004D
:4081800051A60A0851A60A0863F406086DF406085924070851A60A0851A60A0851A60A08000000000000000051A60A0800F002F800F0BDF80AA090E8000C82448344AAF144
:4081C0000107DA4501D100F0B2F8AFF2090EBAE80F0013F0010F18BFFB1A43F001031847604E1D00A04E1D000A444FF0000C10F8013B13F0070408BF10F8014B1D1108BF1D
:4082000010F8015B641E05D010F8016B641E01F8016BF9D113F0080F1EBF10F8014BAD1C0C1B09D16D1E58BF01F801CBFAD505E014F8016B01F8016B6D1EF9D59142D6D37C
:40824000704700000023002400250026103A28BF78C1FBD8520728BF30C148BF0B6070476E293BF02F8F70293BF07388662903F0CAAD652903F0C7AD672903F0C4AD612973
:40828000AFF3008003681B0A28BF41F0800169293AF0E48F64293AF0E18F75293AF0DE8F6F293CF02C8A78293BF03F88E9293CF0C789E4293CF0C489F5293CF0C189EF291B
:4082C0003CF0298AF8293BF03E880368DB0928BF41F0800163293CF0488973293CF04D89E3293CF0638CF3293CF0688C002070471FB5C3F01AFD9DE80300BBF035FEBBF095
:408300005CFABBF00AFE040000200021C2F06EFC401C606000200021C2F07EFCE060BBF0E5FD1FBD10B50020BCF0F1FA10BDBCF016FF1146FFF7DCFF15F08AF8BDF0B6F98C
:4083400003B4FFF7EFFF03BCBCF07CFB80F309887047EFF309807047684680F3098804480078C00714BF0220032080F314887047AC4A0F08DFF818C0EFF305831B0618BF6A
:408380006047EFF31483DB0708BF604700DF70479F9D0C08DFF818C0EFF305831B0618BF6047EFF31483DB0708BF604700DF7047A59F0C08EFF30980816911F8021C01B1CA
:4083C00042E010B590E80F10E047BDE81040EFF3098C254B93E80600914232D041B91EF0100F16D12149086820F00100086010E00CB41EF0100F06BF2CED108A03230123A6
:4084000081F826302CE9F00FC1F82CC0C2F07CF90CBC1A60D2F82CC0BCE8F00F92F8263013F0020F1ABFBCEC108A6FF0120E6FF0020E8CF3098813F0010F08BF704792F8CA
:408440002500CCF80000704710B5094A1268914209D8084C54F8214090E80F10A047EFF3098C8CE80F0010BD7C16001034EF00E068640C0868640C0810B5C1F0DDFFBDE874
:408480001040194B93E80600914208BF70470CB4EFF3098C1EF0100F06BF2CED108A0223002381F826302CE9F00FC1F82CC0C2F02BF90CBC1A60D2F82CC0BCE8F00F92F88F
:4084C000263013F0020F1ABFBCEC108A6FF0120E6FF0020E8CF3098813F0010F1CBF92F82530CCF8003070477C16001010B5C2F0DBF9C4E710B5C1F051FCC2F0D5F9BEE701
:408500000B49D1F800C04A685CF8043B1068184442F8040B8C4528BFA1F1DC0C8A4228BFA1F1DC02C1F800C04A6020F000407047B8F802202DE9F04104460D46174698468C
:40854000069EA0B23246294696F077FB32462946204628F069FFA1B233462A46F748A0F0D9FABDE8F0812DE9F84305460C4616461F46DDF82080E0B23B4632460021009005
:408580002846FFF7D7FFBDE8F88338B50446002003460246042100902046FFF7E4FF38BD07B588B00020069000210A98017008980088702801F0F08674DC702883F03B8174
:4085C000DFE810F0480139193919391939193919391939194A016601AB01EE012D02BA02EF0239192A0353039803AE03130484044F05B405E106391939194507F30701085D
:4086000034086708391907097309B109E2094D0AAD0B140C7E0CD10C380D9F0D3919F20D39195D0E6B0EC60EFE0E11152C154915391939190D0F210B670B160F2D0F5B0F30
:408640007B0F810F870F8D0F930FB60FE30F02103919391939193919391924104E10A010311140113919391939193919391939193919391939193919391939193919411158
:40868000561175118311EA04BB0ACB0AFE15F10AD50A010B110BE311A2083919EB1133122512D60EC62802F066845DDCA42874D037DC932802F0F3811DDC8A2802F0BF812C
:4086C0000CDC712801F07286732867D07A2802F030807C2843F0AF8002F096B88C2802F0B8818E2802F0BE81912802F0C4819228F0D102F0CAB99438102883F09C80DFE8B4
:4087000010F0D811E211091213121D129A189A1827124E129A189A189A184F129A189A187805A6381E28E8D2DFE810F053128D12C712D812061334135F138A13B513C11322
:40874000EB13151485179517A917851885188518561485188518851885188518851885188518B214BF14C914EE2802F0DF863ADCDB2802F0C6851FDCCD2802F051850EDCC6
:40878000C72802F0AA84CA2802F00185CB2802F02185CC289ED102F02BBDFCE392E2CE2802F05285D02802F08D85D12802F09885DA288FD102F095BDDC3812289DD2DFE838
:4087C00010F0AA153A18BA153A183A1803163A183A183B163A183A183A18E6093A184F16601671168216FC2802F0B48712DCA0F1EF000D2897D2DFE810F0D6160D171E184C
:40880000CC161E181E18561766177817841790171E189D1740F20F12811A904201F044800EDCA0F20510002802F0A387012802F0AE87032802F0C7870428ABD102F0B9BF2E
:40884000012902F02D85022902F0D7870829A1D102F0DDBF02F0F0BF03F0BCFC18B101210A98017013E00898007A03280FD10898807A0490324890F8A80503900898007993
:408880000290DDE90312B2F0EDFB0A990870E1E703F0A0FCE0BB0898007A03280CD10898807A04900898808880B20390049911F0D2F90A9908702FE00898007A012811D13F
:4088C00011F029F90122099902FB010080B204900898807A01460390049811F0BCF90A99087019E00898007A022815D111F013F90122099902FB110080B204900898807A88
:4089000001460390049811F0A6F90A99087003E0FFE701210A9801709CE70898007A032810D10898807A04900898808880B203900499B2F034FB0A9908702EE0BCDD001084
:40894000602A00200898007A012811D1B1F026F80122099902FB010080B204900898807A014603900498B2F01AFB0A99087014E00898007A022810D1B1F010F80122099977
:4089800002FB110080B204900898807A014603900498B2F004FB0A9908700120069059E70898007A03280CD10898807A04900898808880B203900499B2F010FB0A990870FE
:4089C0002AE00898007A012811D1B0F006FB0122099902FB010080B204900898807A014603900498B2F0FAFA0A99087014E00898007A022810D1B0F0F0FA0122099902FBF8
:408A0000110080B204900898807A014603900498B2F0E4FA0A990870012006901AE70898406842F2067188420AD00898406846F21E31884204D008984068491C884209D1A7
:408A400020F04DF930B1012027F078FD0C20FFF79CFD6AE00898007A03280DD1089890ED010AB8EEC00A8DED040A9DED040A11F0C5F90A99087058E00898007A012828D1E4
:408A800082F016FE90B911F09DF8DDED090AF8EE600AB1EE041A01EE200A8DED040A9DED040A11F0ABF90A9908703EE011F08AF8DDED090AF8EE600A9FEDFE1A01EE200AE3
:408AC0008DED040A9DED040A11F098F90A9908702BE00898007A022827D182F0E9FD90B911F070F8DDED090AF8EE600AB1EE041A01EE600A8DED040A9DED040A11F07EF97D
:408B00000A99087011E011F05DF8DDED090AF8EE600A9FEDE81A01EE600A8DED040A9DED040A11F06BF90A9908709FEDE30A11F0ECF8012006908DE603F04CFB68BB08989A
:408B4000007A032807D108984068049011F005F90A9908701EE00898007A01280BD110F0EAFF0122099902FB0100049011F0F5F80A9908700EE00898007A02280AD110F00F
:408B8000DAFF0122099902FB1100049011F0E5F80A9908700120069002E001210A98017058E603F017FB90BB0898007A032808D10898808880B2049011F0FEF80A99087082
:408BC00022E00898007A01280DD1BC48B0F85C240121099801FB002080B2049011F0ECF80A99087010E00898007A02280CD1B348B0F85C140122099802FB101080B20490B6
:408C000011F0DAF80A9908700120069003E0FFE701210A9801701DE603F0DCFA20BB0898007A032820D1A54890F840140898406881420BD0002011F04DF90020A04908701D
:408C4000A0480978405C049011F028F908980079049011F00BF90A9908709B4856F0E6FE10B10120A7F084FBF4E503F0B3FA00BB0898007A032824D108980079039012F04B
:408C800005F9049011F026F90A99087000208C49087008980079049012F0F8F8172809D1864890F84004401EC0B20590059811F0F5F806E0834882490978405C049011F00A
:408CC000EDF8C7E503F086FA98B90898007A03280FD10898406800280BDD089800797849087078480978405C049011F0D7F80A990870AFE51BF083FEFA2810D01BF07FFE4A
:408D0000FB280CD00898007A032808D10898807A0490089800790390049911F0F3F899E50898007A032812D1644890F8A9050490624890F8A80503900898808800B2029039
:408D4000DDE9031215F01CFF0A9908704AE00898007A012821D1594890F8A81500F5AD6000EB8101554890F8A90531F810200121099801FB002000B20290504890F8A9050C
:408D800004904E4890F8A80503900146049A029815F0F6FE0A99087024E00898007A022820D1464890F8A81500F5AD6000EB8101424890F8A90531F810100122099802FBE9
:408DC000101000B202903D4890F8A90504903B4890F8A80503900146049A029815F0D0FE0A9908700120069034E50898007A032812D1324890F8A9050490304890F8A8051F
:408E000003900898808800B20290DDE9031215F0F4FC0A9908704AE00898007A012821D1264890F8A81500F5A56000EB8101234890F8A90531F810100122099802FB001094
:408E400000B202901D4890F8A90504901B4890F8A80503900146049A029815F0CEFC0A99087024E00898007A022820D1134890F8A81500F5A56000EB8101104890F8A9051D
:408E800031F810100122099802FB101000B202900A4890F8A9050490084890F8A80503900146049A029815F0A8FC0A99087001200690CFE45C8F224000000000602A00206C
:408EC000B6140010F4E00C08186202200898007A032812D1F94890F8A9050490F74890F8A80503900898808800B20290DDE9031215F0D2FC0A9908704AE00898007A0128B8
:408F000021D1EE4890F8A81500F5A66000EB8101EA4890F8A90531F810100122099802FB001000B20290E54890F8A9050490E34890F8A80503900146049A029815F0ACFC80
:408F40000A99087024E00898007A022820D1DB4890F8A81500F5A66000EB8101D74890F8A90531F810100122099802FB101000B20290D24890F8A9050490D04890F8A805D9
:408F800003900146049A029815F086FC0A990870012006905EE493E10898007A032812D1C64890F8A9050490C44890F8A80503900898808800B20290DDE9031215F029FEC9
:408FC0000A9908704AE00898007A012821D1BB4890F8A81500F5AC6000EB8101B74890F8A90531F810100122099802FB001000B20290B24890F8A9050490B04890F8A805BD
:4090000003900146049A029815F003FE0A99087024E00898007A022820D1A84890F8A81500F5AC6000EB8101A44890F8A90531F810100122099802FB101000B202909F48AA
:4090400090F8A90504909D4890F8A80503900146049A029815F0DDFD0A9908700120069015E40898007A032812D1944890F8A9050490924890F8A80503900898808800B286
:409080000290DDE9031215F045FC0A9908704AE00898007A012821D1884890F8A81500F5A76000EB8101854890F8A90531F810100122099802FB001000B202907F4890F855
:4090C000A90504907D4890F8A80503900146049A029815F01FFC0A99087024E00898007A022820D1754890F8A81500F5A76000EB8101724890F8A90531F810100122099846
:4091000002FB101000B202906C4890F8A90504906A4890F8A80503900146049A029815F0F9FB0A9908700120069038E40898007A032810D1614890F8A90504905F4890F8A8
:40914000A80503900898808800B20290DDE9031215F05CFC4AE00898007A012821D1574890F8A81500F5A86000EB8101534890F8A90531F810100122099802FB001000B241
:4091800002904E4890F8A90504904C4890F8A80503900146049A029815F038FC0A99087024E00898007A022820D1444890F8A81500F5A86000EB8101404890F8A90531F833
:4091C00010100122099802FB101000B202903B4890F8A9050490394890F8A80503900146049A029815F012FC0A9908700120069014E40898007A032812D1304890F8A90562
:4092000004902E4890F8A80503900898808800B20290DDE9031215F0BBFB0A9908704AE00898007A012821D1244890F8A81500F5AA6000EB8101214890F8A90531F810105B
:409240000122099802FB001000B202901B4890F8A9050490194890F8A80503900146049A029815F095FB0A99087024E00898007A022820D1114890F8A81500F5AA6000EB93
:4092800081010E4890F8A90531F810100122099802FB101000B20290084890F8A9050490064890F8A80503900146049A029815F06FFB0A990870012006903CE4602A002078
:4092C0000898007A032810D1F84890F8A9050490F64890F8A80503900898808800B20290DDE9031215F0D0FB4AE00898007A012821D1EE4890F8A81500F5AB6000EB81015A
:40930000EA4890F8A90531F810200121099801FB002000B20290E54890F8A9050490E34890F8A80503900146049A029815F0ACFB0A99087024E00898007A022820D1DB48BD
:4093400090F8A81500F5AB6000EB8101D74890F8A90531F810100122099802FB101000B20290D24890F8A9050490D04890F8A80503900146049A029815F086FB0A99087094
:40938000012006900CE40898007A032811D1C74890F8A9050490C54890F8A8050390089800790290DDE9031215F0ACFB0A9908704AE00898007A012821D1BC4890F8A8153C
:4093C00000F5A96000EB8101B84890F8A90531F810100122099802FB001000B20290B34890F8A9050490B14890F8A80503900146049A029815F086FB0A99087024E0089824
:40940000007A022820D1A94890F8A81500F5A96000EB8101A54890F8A90531F810100122099802FB101000B20290A04890F8A90504909E4890F8A80503900146049A029886
:4094400015F060FB0A990870012006900CE40898007A03286FD108984068F1280CD119F094FE01460490002017F08AFF1420DFF840C200DF03DF91E008984068F22809D166
:409480008C48D0F8B001014604900220DFF828C200DF83E008984068F32803D1032023F0E2F87BE008984068F7280AD18148D0F8B001014604904FF40070DFF8FCC100DF38
:4094C0006CE008984068F42809D17A48D0F8B001014604908020DFF8E0C100DF5EE008984068F5280AD17348D0F8B001014604904FF48070DFF8C0C100DF4FE00898406867
:40950000F62809D16B48D0F8B001014604900120DFF8A4C100DF41E008984068F8280BD16448D0F8B001014604904FF48060DFF888C100DF32E012E008984068F9280AD121
:409540005C48D0F8B001014604904FF40060DFF868C100DF22E006210A9801701EE00898007A012809D15348D0F8B001014604900420DFF844C100DF10E00898007A022818
:4095800009D14C48D0F8B001014604900820DFF828C100DF02E007210A9801701B20FEF7F4FF11204EF0DEF91EE40898007A012802D1002023F057F81C20FEF7E6FF2C20A0
:4095C0004EF0D0F910E40898007A032808D10898808800B204900CF03DFC0A99087022E00898007A01280DD13048B0F8AA150122099802FB001000B204900CF02BFC0A9935
:40960000087010E00898007A02280CD12748B0F8AA150122099802FB101000B204900CF019FC0A9908700120069042E40898007A032808D10898808880B204900CF07FFC98
:409640000A99087022E00898007A01280DD11748B0F8B4150122099802FB001080B204900CF06DFC0A99087010E00898007A02280CD10E48B0F8B4150122099802FB10100C
:4096800080B204900CF05BFC0A990870012006900FE40898007A032810D10898808880B204900CF07BFC0A9908702AE0602A0020A99E0C08F8FF0020099F0C080898007AAE
:4096C00001280DD1FE48B0F8B6250121099801FB002080B204900CF061FC0A99087010E00898007A02280CD1F548B0F8B6150122099802FB101080B204900CF04FFC0A992F
:4097000008700120069045E40898007A032812D1EB4890F8A9050490E94890F8A80503900898808800B20290DDE903120CF0C4FB0A9908704AE00898007A012821D1E0488F
:4097400090F8A81500F2AC5000EB8101DC4890F8A90531F810100122099802FB001000B20290D74890F8A9050490D54890F8A80503900146049A02980CF09EFB0A99087094
:4097800024E00898007A022820D1CD4890F8A81500F2AC5000EB8101C94890F8A90531F810100122099802FB101000B20290C44890F8A9050490C24890F8A8050390014617
:4097C000049A02980CF078FB0A9908700120069046E40898007A032814D10898807A0490B74890F8A9050390B54890F8A805029008980079019002A90EC9ADF03DFA0A993F
:4098000008704EE00898007A012823D1AC4890F8A81500F2944000EB4101A94890F8A905095C0122099802FB001001900898807A0490A34890F8A9050390A14890F8A80531
:4098400002900146DDE903230198ADF015FA0A99087026E00898007A022822D1984890F8A81500F2944000EB4101954890F8A905095C0122099802FB101001900898807AEA
:4098800004908F4890F8A90503908D4890F8A80502900146DDE903230198ADF0EDF90A9908700120069040E43FE40898007A03280BD10898807A04900898007903900499D8
:4098C000ADF087FA0A9908702AE00898007A012811D17B4890F841160122099802FB001003900898807A014604900398ADF071FA0A99087014E00898007A022810D17048F6
:4099000090F841160122099802FB101003900898807A014604900398ADF05BFA0A9908700120069064E40898007A032807D10898007904900CF061FB0A99087021E00898DA
:40994000007A01280CD15E4890F810160122099802FB001004900CF050FB0A99087010E00898007A02280CD1554890F810160122099802FB101080B204900CF03EFB0A9971
:4099800008700120069033E40898007A032814D10898807A04904A4890F8A9050390484890F8A805029008980079019002A90EC9ADF0B1FA0A9908704EE00898007A012857
:4099C00023D13F4890F8A81500F5936000EB41013B4890F8A905095C0122099802FB001001900898807A0490354890F8A9050390334890F8A80502900146DDE90323019890
:409A0000ADF089FA0A99087026E00898007A022822D12B4890F8A81500F5936000EB4101274890F8A905095C0122099802FB101001900898807A0490214890F8A905039005
:409A40001F4890F8A80502900146DDE903230198ADF061FA0A990870012006902DE40898007A032814D10898807A0490144890F8A9050390124890F8A8050290089800795A
:409A8000019002A90EC9ADF007FB0A99087051E00898007A012826D1094890F8A81500F29C4000EB4101064890F8A905095C0122099802FB001001900898807A049001E083
:409AC000602A0020FD4890F8A9050390FB4890F8A80502900146DDE903230198ADF0DCFA0A99087026E00898007A022822D1F34890F8A81500F29C4000EB4101EF4890F8D3
:409B0000A905095C0122099802FB101001900898807A0490E94890F8A9050390E74890F8A80502900146DDE903230198ADF0B4FA0A9908700120069024E40898007A03284C
:409B40000AD10898807A04900898007903900499AEF017F90A99087014E40898007A032804D108980079049033F0DBF90AE40898007A03280AD10898807A049008980079BF
:409B800003900499ABF0C2FC0A9908705EE40898007A032806D108980079049029F062FC0A99087052E40898007A03280AD10898807A04900898007903900499ABF0C0FC40
:409BC0000A99087042E40898007A03280AD10898807A04900898007903900499ABF0CAFC0A99087032E40898007A03280AD10898807A04900898007903900499ABF0D4FCF9
:409C00000A99087022E40898007A032811D1089890ED010AF8EEC00AB2EE041A80EE810A8DED040A9DED040AAEF059F80A9908702CE00898007A012812D1AEF034F9012203
:409C4000099902FB110000EE100AB8EEC00A8DED040A9DED040AAEF042F80A99087015E00898007A022811D1AEF01DF90122099902FB010000EE100AB8EEC00A8DED040A17
:409C80009DED040AAEF02BF80A990870012006908AE40898007A032811D1089890ED010AF8EEC00AB2EE041A80EE810A8DED040A9DED040AAEF03CF80A9908702CE008989C
:409CC000007A012812D1AEF0F7F80122099902FB010000EE100AB8EEC00A8DED040A9DED040AAEF025F80A99087015E00898007A022811D1AEF0E0F80122099902FB1100BC
:409D000000EE100AB8EEC00A8DED040A9DED040AAEF00EF80A9908700120069044E40898007A032818D1089890ED010AF8EEC00AB2EE041A80EE810A8DED040A807A03901B
:409D40005E4890F8A905029003999DED040AADF065FA0A99087046E00898007A01281FD1564890F8A91500F2A44000EB8100D0ED000A9DED090AB8EEC00A30EE800A8DEDB5
:409D8000020A0898807A04904C4890F8A905039004999DED020AADF041FA0A99087022E00898007A02281ED1444890F8A91500F2A44000EB8100D0ED000A9DED090AB8EE93
:409DC000C00A30EEC00A8DED020A0898807A04903A4890F8A905039004999DED020AADF01DFA0A990870012006901EE40898007A032818D1089890ED010AF8EEC00AB2EE51
:409E0000041A80EE810A8DED040A807A03902B4890F8A905029003999DED040AADF0E7FA0A99087046E00898007A01281FD1234890F8A91500F2B44000EB8100D0ED000ACB
:409E40009DED090AB8EEC00A30EE800A8DED020A0898807A0490194890F8A905039004999DED020AADF0C3FA0A99087022E00898007A02281ED1114890F8A91500F2B440ED
:409E800000EB8100D0ED000A9DED090AB8EEC00A30EEC00A8DED020A0898807A0490074890F8A905039004999DED020AADF09FFA0A9908700120069025E40000602A0020C0
:409EC0000898007A032810D10898807A0490FE4890F8A9050390089800790290DDE90312ADF099FD0A9908703AE00898007A012819D1F54890F8A91500F2CC40415C0122A3
:409F0000099802FB001002900898807A0490EE4890F8A90503900146049A0298ADF07BFD0A9908701CE00898007A022818D1E64890F8A91500F2CC40415C0122099802FB0C
:409F4000101002900898807A0490DF4890F8A90503900146049A0298ADF05DFD0A9908700120069034E40898007A032818D1089890ED010AF8EEC00AB2EE041A80EE810AF4
:409F80008DED040A807A0390CF4890F8A905029003999DED040AADF044FB0A99087046E00898007A01281FD1C74890F8A91500F2AC4000EB8100D0ED000A9DED090AB8EE80
:409FC000C00A30EE800A8DED020A0898807A0490BD4890F8A905039004999DED020AADF020FB0A99087022E00898007A02281ED1B54890F8A91500F2AC4000EB8100D0EDE8
:40A00000000A9DED090AB8EEC00A30EEC00A8DED020A0898807A0490AB4890F8A905039004999DED020AADF0FCFA0A9908700120069038E40898007A032818D1089890EDB2
:40A04000010AF8EEC00AB2EE041A80EE810A8DED040A807A03909C4890F8A905029003999DED040AADF0C6FB0A99087046E00898007A01281FD1944890F8A91500F2BC4097
:40A0800000EB8100D0ED000A9DED090AB8EEC00A30EE800A8DED020A0898807A04908A4890F8A905039004999DED020AADF0A2FB0A99087022E00898007A02281ED18248E2
:40A0C00090F8A91500F2BC4000EB8100D0ED000A9DED090AB8EEC00A30EEC00A8DED020A0898807A0490784890F8A905039004999DED020AADF07EFB0A99087001200690AC
:40A1000010E40898007A032810D10898807A04906D4890F8A9050390089800790290DDE90312ADF01EFD0A9908703AE00898007A012819D1644890F8A91500F2CE40415C2A
:40A140000122099802FB001002900898807A04905D4890F8A90503900146049A0298ADF000FD0A9908701CE00898007A022818D1554890F8A91500F2CE40415C012209983F
:40A1800002FB101002900898807A04904E4890F8A90503900146049A0298ADF0E2FC0A9908700120069059E40898007A032814D10898807A0490444890F8A9050390424823
:40A1C00090F8A805029008980079019002A90EC9ACF081FC0A9908704EE00898007A012823D1394890F8A81500F5946000EB4101354890F8A905095C0122099802FB00100E
:40A2000001900898807A04902F4890F8A90503902D4890F8A80502900146DDE903230198ACF059FC0A99087026E00898007A022822D1254890F8A81500F5946000EB410106
:40A24000214890F8A905095C0122099802FB101001900898807A04901B4890F8A9050390194890F8A80502900146DDE903230198ACF031FC0A990870012006905CE408989F
:40A28000007A032808D10898807A04900898007903900499A9F0BBF84EE40898007A032816D10898807A04900898808880B200EE100AB8EE400A8DED030A04989DED030A45
:40A2C000A8F074FD0A9901E0602A002008703CE00898007A01281AD1A9F0EEFAF0EE400AF94890ED851A9DED090AF8EE401AB0EE410A00EEA10A8DED040A0898807A03904B
:40A300009DED040AA8F052FD0A9908701DE00898007A022819D1A9F0CFFAF0EE400AEA4890ED851A9DED090AF8EE401AB0EE410A00EEE10A8DED040A0898807A03909DEDA2
:40A34000040AA8F033FD0A990870012006900DE40898007A03280AD10898807A04900898007903900499B0F014FD0A9908700DE40898007A03280ED1089890ED010AF8EEBE
:40A38000C00A9FEDD21A80EE810A8DED040A9DED040A0BF0C2FF05E40898007A032804D10898007904900BF019FF0BE40898007A032804D10898007904900BF0DAFE11E445
:40A3C0000898807A0490C24890F8410808B9012000E0002003900499AEF08DFA12E40898007A032803D108980079BA49087009E40898007A032807D100229FEDB70A0321DD
:40A400001020A7F023F909E00898007A30B900229FEDB10A11461046A7F018F938E40898007A03281ED1AA4890F8A91500F2A44000EB810090ED000A8DED070A9DED070A18
:40A44000B5EEC00AF1EE10FA03D19FEDA40A8DED070A4FF0FF329DED070A03210820A7F0F5F809E00898007A30B900229FED9A0A11460820A7F0EAF80AE40898007A0328A9
:40A4800010D1ADF010FD00EE100AB8EEC00A8DED040A6FF009029DED040A03210A20A7F0D5F809E00898007A30B900229FED8A0A11460820A7F0CAF830E40898007A0328FE
:40A4C00000D000BF2AE40898007A032800D000BF24E40898007A032800D000BF1EE40898007A032800D000BF18E40898007A032813D1774890F8A91500F2B44000EB8100BD
:40A5000090ED000A8DED040A6FF001029DED040A03210820A7F09AF809E00898007A30B900229FED6D0A11460820A7F08FF85CE40898007A03281DD1654890F8A91500F297
:40A54000AC4000EB810090ED000A8DED070A9DED070AB5EEC00AF1EE10FA03D19FED600A8DED070A01229DED070A03210820A7F06DF809E00898007A30B900229FED560A2B
:40A5800011460820A7F062F82FE40898007A03280FD1ADF091FC00EE100AB8EEC00A8DED040A0A229DED040A03211046A7F04EF809E00898007A30B900229FED470A11466C
:40A5C0000820A7F043F810E40898007A032812D13F4890F8A91500F2BC4000EB810090ED000A8DED040A02229DED040A03210820A7F02CF809E00898007A30B900229FEDB2
:40A60000360A11460820A7F021F855E40898007A032807D108980079049023F059FA0A9908701CE00898007A01280AD1284890F84006401CC0B2049023F04AFA0A990870FB
:40A640000DE00898007A022809D1214890F84006401EC0B2049023F03BFA0A9908702BE40898007A03284CD10898406888B9184890F8A9050490164890F8A80503900499EA
:40A680000FF04FF8124890F8A90504900FF0F6F837E008984068012806D10D4890F8A90504900FF0EBF82CE008984068022819D1074890F8A9050490054890F8A80503904D
:40A6C00004990EF075FE1CE0602E002000007A44602A00208502001000000000CDCCCCBDCDCCCC3D0898406803280AD1FB4890F8A9050490F94890F8A805039004990EF0E0
:40A7000065FF2FE40898007A032809D108980079049007F086FD0A990870042007F01DF9EE4890F8F805012802D0002008F06AFD18E40898007A032865D1089840680728ED
:40A7400052D2DFE800F0040F1A25303B4600012007F0D7FC0A990870002007F0BAFC0A9908704CE0032007F0CCFC0A990870832007F0AFFC0A99087041E0032007F0C1FC8C
:40A780000A990870852007F0A4FC0A99087036E0032007F0B6FC0A9908708A2007F099FC0A9908702BE0042007F0ABFC0A990870782007F08EFC0A99087020E0042007F0A2
:40A7C000A0FC0A9908707C2007F083FC0A99087015E0042007F095FC0A9908707E2007F078FC0A9908700AE0012007F08AFC0A990870002007F06DFC0A99087000BF00BFD9
:40A80000402007F0AAF814E40898007A032809D108980079049007F08CFD0A990870802007F09BF805E40898007A032809D108980079049007F052FD0A990870022007F067
:40A840008CF85DE45CE40898007A03280FD1A021A348B9F0DEF967F005FFA149886567F001FF9F49C86667F0FDFE9D49086747E40898007A032819D1A0219A48B9F0C9F9D4
:40A880004FF47F619848B9F0C4F94FF47F619748B9F0BFF967F0E6FE9249886567F0E2FE9049C86667F0DEFE8E49086728E40898007A032808D18E48D0F8B00101460490BE
:40A8C0000220DFF830C200DF1AE440F0D0FD0899897A884232D10FF028FDD8B14AF0ADFBC0B1854890F80501012809D18348844B01220321009041F2D50052F0B3FA43E039
:40A900007E487F4B00220321009041F2D50052F0A9FA39E0784890F80501012800D100E0002080F00100049009F08BFF26F06FF97448007808B325F013FE25E00FF0F5FC53
:40A9400078B14AF07AFB60B16C480090089840686B4B02460321049041F2D50052F082FA12E008984068012808D1002009F069FF6448007808B125F0F3FD05E0089840681A
:40A9800010B9012009F05DFF0DE40898007A012802D1022019F00AFC05E40898007A03280DD1089890ED010AB8EEC00A8DED040A9DED040A07F0FAFB0A99087026E00898AF
:40A9C000007A01280FD1504890ED020AF7EE000A30EE200A8DED040A9DED040A07F0E6FB0A99087012E00898007A02280ED1464890ED020AF7EE000A30EE600A8DED040A3E
:40AA00009DED040A07F0D2FB0A99087036E40898007A032808D10898807A04900898007903900499ABF0D4FD28E40898007A032804D108F060FC202006F08FFF1EE40898A4
:40AA4000007A032804D108980079049001F0F9F814E40898007A032803D1089800792B4908700BE40898007A032803D1089800792749087010E40898007A032804D1089800
:40AA80004068049026F0B9FD06E40898007A032804D108980079049027F0F9FC57E40898007A032804D108980079049027F01BFD4DE40898007A032804D1089800790490A8
:40AAC00027F03DFD43E40898007A032804D108980079049027F05FFD39E40000602A0020C83800206839002074B5002064C50020F8FF0020099F0C0858200020406B022032
:40AB0000585E0220E722001060320020C0140010C11400100898007A032804D108980079049027F0A1FD12E40898007A032804D108980079049027F0C3FD08E40898007A93
:40AB4000032804D108980079049027F0E5FD0EE40898007A032821D108984068052818D2DFE800F003070B0F1300002008F029FE13E0012008F025FE0FE0022008F021FE23
:40AB80000BE0032008F01DFE07E0042008F019FE03E0002008F015FE00BF00BF05E404E40898007A032813D1FA4890F8A805012807D10898807A0146049000200FF0EBFCE1
:40ABC00006E00898807A0146049001200FF0E3FC04E40898007A03280DD10898807A04900898808880B203900121049A59F0CBF90A99087026E00898007A01280FD10898A4
:40AC0000807A0490E348B0F82208401C80B203900121049A59F0B7F90A99087012E00898007A02280ED10898807A0490D948B0F82208401E80B203900121049A59F0A3F996
:40AC40000A99087018E40898007A03280DD10898807A04900898808880B203900121049A59F039FA0A99087026E00898007A01280FD10898807A0490C648B0F82408401C13
:40AC800080B203900121049A59F025FA0A99087012E00898007A02280ED10898807A0490BC48B0F82408401E80B203900121049A59F011FA0A99087004E40898007A0328F2
:40ACC0000BD10898807A04900898808880B20390049959F0ADFA0A99087005E40898007A032809D10898808880B20121049059F055FB0A9908701EE00898007A01280BD1CC
:40AD0000A448B0F82608401C80B20121049059F045FB0A9908700EE00898007A02280AD19C48B0F82608401E80B20121049059F035FB0A99087027E40898007A032809D19E
:40AD40000898808880B20121049059F064FB0A9908701EE00898007A01280BD18D48B0F82808401C80B20121049059F054FB0A9908700EE00898007A02280AD18548B0F83D
:40AD80002808401E80B20121049059F044FB0A99087014E20898007A032808D10898808880B2049059F074FB0A9908701CE00898007A01280AD17748B0F82A08401C80B2E4
:40ADC000049059F065FB0A9908700DE00898007A022809D16F48B0F82A08401E80B2049059F056FB0A990870E9E10898007A032808D10898808880B2049059F07FFB0A99CA
:40AE000008701CE00898007A01280AD16148B0F82C08401C80B2049059F070FB0A9908700DE00898007A022809D15A48B0F82C08401E80B2049059F061FB0A990870BEE1FE
:40AE40000898007A032808D10898808880B2049014F024F90A9908701CE00898007A01280AD14C48B0F82E08401C80B2049014F015F90A9908700DE00898007A022809D124
:40AE80004448B0F82E08401E80B2049014F006F90A99087093E10898007A032806D108980079049059F060FB0A99087087E10898007A032807D108980079049059F088FBEC
:40AEC0000A9908701CE00898007A01280AD1314890F83108401CC0B2049059F079FB0A9908700DE00898007A022809D1294890F83108401EC0B2049059F06AFB0A9908703F
:40AF00005DE10898007A032807D108980079049059F092FB0A9908701CE00898007A01280AD11C4890F83208401CC0B2049059F083FB0A9908700DE00898007A022809D189
:40AF4000144890F83208401EC0B2049059F074FB0A99087033E10898007A03280AD10898807A0490089800790390049958F04EFE0A99087023E10898007A03280CD108985C
:40AF8000808880B20121049059F01CFC0A99087021E00000602A00200898007A01280BD1F948B0F83408401C80B20121049059F009FC0A9908700EE00898007A02280AD17C
:40AFC000F148B0F83408401E80B20121049059F0F9FB0A990870F2E00898007A032801D118F091FEEBE00898007A032815D10FF089FA04900898807A0390089890ED010AB5
:40B00000B8EEC00A8DED020A0020DDE903219DED020AAEF023FC0A990870D0E00898007A032817D10FF06EFA04900898807A03900898808880B200EE100AB8EE400A8DED51
:40B04000020A0020DDE903219DED020AADF0C7FD0A990870F0E30898007A032817D10FF051FA04900898807A03900898808880B200EE100AB8EE400A8DED020A0020DDE95F
:40B0800003219DED020AAEF0BFFA0A990870D3E30898007A032805D1089800790121049007F0D5F906F0DBFBC6E30898007A032804D108980079049010F0C5FBBCE30898C4
:40B0C000007A032808D10898807A04900898007903900499AAF0D3F8AEE30898007A032815D1089890ED010AF8EEC00A9FEDA71A80EE810A8DED040AA34890F8A8050390E1
:40B100009DED040A13F0BEF90A9908703EE00898007A01281BD19C4890F8A81500F6580000EB8100D0ED000A9DED090AB8EEC00A30EE800A8DED030A934890F8A8050490CB
:40B140009DED030A13F09EF90A9908701EE00898007A02281AD18C4890F8A81500F6580000EB8100D0ED000A9DED090AB8EEC00A30EEC00A8DED030A834890F8A8050490AC
:40B180009DED030A13F07EF90A99087054E30898007A032813D17C4890F8A905012807D10898807A01460490002010F04BF806E00898807A01460490012010F043F83BE35B
:40B1C0000898406808B1012000E00020049010F085F831E30898007A032808D10898807A049008980079039004990DF08DFF23E30898007A032812D108984068012804D077
:40B20000022805D0032809D105E03BF0A4FF05E03CF080F802E03CF05DFC00BF00BF0BE30898007A03280ED1089890ED010AB8EEC00ADFED570A20EE200A8DED040A9DEDC8
:40B24000040A3CF0F3F8F7E20898007A032826D10898406805281DD2DFE800F003080D1217004FF4165007F008F813E04FF4964007F003F80EE04FF4164006F0FEFF09E037
:40B280004FF4614006F0F9FF04E04FF4E13006F0F4FF00BF00BF4FF4804006F05EFBCBE20898007A03280CD1089890ED010AB8EEC00ABCEEC00A10EE100AC0B2049007F0DB
:40B2C00082FFB9E20898007A032808D10898807A04900898007903900499B0F088FAABE2AAE20898007A03280AD1089890ED010AB8EEC00A8DED040A9DED040A09F0E8FAAF
:40B300009AE20898007A032804D108980079049018F0A7F890E20898007A03280AD108980079049008F0D4F80A9908704FF4007006F013FB80E200F04DFF20BB154800F088
:40B3400056FF00BB134801F03DFBE0B9114801F02EFBC0B90898007A032805D108980079049009F0C3FF2EE00898007A012817D109F047FE04280FDA09F043FE401CC0B29D
:40B38000049009F0B3FF1EE0602A002000007A446F12833A78170010012009F0A7FF12E00898007A02280ED109F02BFE012807DD09F027FE401EC0B2049009F097FF02E014
:40B3C000042009F093FF37E20898007A032809D10898807A0490089840680390049910F07EF826E00898007A01280FD1FE48B0F84A180122099802FB001003900898807AD3
:40B4000001460490039810F06AF812E00898007A02280ED1F448B0F84A180122099802FB101003900898807A01460490039810F056F801200690FFE10898007A03280ED14C
:40B440000898807A0490089890ED010AB8EEC00A8DED030A04989DED030AADF0D1F9EBE10898007A03280BD10898807A04900898808880B203900499AAF006FA0A9908700B
:40B48000DAE10898007A03280BD10898807A04900898808880B203900499AAF041F90A990870C9E10898007A03280BD10898807A04900898808880B203900499AAF09FF855
:40B4C0000A990870B8E10898007A032808D10898808880B2049057F0D7FD0A99087022E00898007A01280DD1BF48B0F84E170122099802FB001080B2049057F0C5FD0A995C
:40B50000087010E00898007A02280CD1B648B0F84E170122099802FB101080B2049057F0B3FD0A9908700120069085E10898007A032808D10898808880B2049057F0D3FDFE
:40B540000A99087022E00898007A01280DD1A648B0F850270121099801FB002080B2049057F092FD0A99087010E00898007A02280CD19D48B0F850170122099802FB101004
:40B5800080B2049057F080FD0A9908700120069052E10898007A032804D1089840680490A9F006F848E10898007A03280CD10898807A04900898808880B20390049959F0A3
:40B5C00043F90A99087024E00898007A01280ED10898807A04908448B0F85407401C80B20390049959F030F90A99087011E00898007A02280DD10898807A04907A48B0F8DB
:40B600005407401E80B20390049959F01DF90A99087011E10898007A03280BD10898807A04900898808880B20390049959F08FF90A99087000E10898007A03280AD108989D
:40B64000807A0490089800790390049959F028F80A990870F0E00898007A03280ED10898807A049008988088A0F51C50063800B20390049959F0EEF90A990870DCE00898DD
:40B68000007A03280ED10898807A049008988088A0F51C50063800B20390049959F072FA0A990870C8E00898007A03280AD10898807A04900898007903900499AFF086FFDC
:40B6C0000A990870B8E00898007A03280CD1089890ED010AB8EEC00A8DED040A9DED040A01F04CFD0A990870A6E00898007A032806D108980079049001F072FD0A9908709E
:40B700009AE00898007A032806D108980079049001F0FFFC0A9908708EE00898007A032807D10898808880B2049001F0AEFD0A99087081E00898007A03280AD10898406846
:40B7400008B1012000E00020049001F0D8FD0A99087071E00898007A032809D108980079049007F04FFD0A990870042006F0F5F862E00898007A032808D10898406808B197
:40B78000012000E0002004900AF065FC54E00898007A03280CD10898807A04900898406808B1012000E00020039004995EF08BFA00BF0898007A032804D10898007904904A
:40B7C00009F0F2FB38E00898007A032814D1089890ED010AF8EEC00A9FED041A80EE810A8DED040A04E00000602A002000007A449DED040A3CF058F91EE00898007A03287A
:40B8000004D10898007904903BF0C9FB14E0089890ED010AB8EEC00ADFEDA60A20EE200ADFEDA50A20EE200A8DED040A9DED040A59F0BAFB00E000BF00BF0898008804906C
:40B84000FCF7A3FE06980BB000BD86B04FF6FF740020009001900290039028219748B8F0D8F938219648DFF85CC200DF0221964880F884110C2284219448BEF08BF9002807
:40B8800071D10321904880F8841100BF224605A98B48DFF83CC200DF01284CD00020ADF800008DF80D0001208DF80C0000208DF80E0005980088002838D004AA012105981E
:40B8C000FCF76EFE05469DF8100068B100250599088850F0A9FE06460598C37A827A9DF81010304650F05AFF00F074FC08B1002504E00598007A032800D10025B5B19DF86B
:40B900000D0098B90598007A80B1059A07CA8DE8070001208DF80D008DF80C004FF47A649DF80E00401CC0B28DF80E0067480599FCF730FDAAE7BDF800000028A6DD9DF819
:40B940000E0000283DDD9DF80E00032803D102208DF80C000FE09DF80E00052804D106208DF80C0007E02FE09DF80E00072802D110208DF80C009DF80E00FF2805DA9DF83D
:40B980000E00401CC0B28DF80E009DF80C1004AA6846FCF705FE9DF8100078B100208DF80E000599088850F03FFE06460598C37A827A9DF81010304650F0F0FE4FF4FA64CD
:40B9C00064E74FF6FF7461E705213F4880F884110020DFF800C100DF00BFFEE72DE9F84305460C4616461F46DDF82080E0B23B463246002100902846FCF79CFDBDE8F8838D
:40BA00002DE9F04705460E4617469846DDF820904FF0010A2A48DFF8C0C000DFD0B900BF294890F8850140F00201274880F88511B0F890014FF6FF71884207DA2248B0F846
:40BA40009001401C81B22048A0F8901100BF4FF0000A2CE01D48FCF78DFC04466CB125806660277284F80A8084F80B900C2221461348DFF868C000DF19E000BF124890F820
:40BA8000850140F00401104880F88511B0F890014FF6FF71884207DA0B48B0F89001401C81B20948A0F8901100BF4FF0000A5046BDE8F087CDCCCC3D6DE2E43E50170010E3
:40BAC0001817001091A00C08F8FF00209416001021A20C08C5A90C0889A00C087DA10C0810B564F0D8FB044666480022D0F80016204662F0C7F910BD624890F83103022870
:40BB000001D1012070470020FCE74FF6FF7664F0C2FB07465B480022D0F80016384662F0B1F925F04AFD074664F060FB80460022394662F0A7F9DFF850C100DF07466423D7
:40BB40002122082166F07AFE30B1DFF83CC100DF0746082166F0AEFEDFF82CC100DF074639460420DFF824C100DF00BF002231460D20DFF81CC100DF0446012CF6D0022CCE
:40BB8000F4D1DFF810C100DF054605F0080090B10FF060FD10B100F08FF80AE025F09AFC10B126F000FC04E027F053FC08B127F082FB26F04EFC05F004000028D6D063F0A3
:40BBC0001EFE18B934480078012806D032480078032802D063F013FEA0B10FF03BFD20B100F097F825F07EFCC0E727F0ABF920B125F078FC27F0C0F8B8E727F006F925F056
:40BC000026FDB3E7244800780228AFD1FFF774FF30B127F0ECFB25F065FCFFF761FFA5E725F058FC20B127F0E2FB25F010FD9DE727F00FFC002899D025F054FC27F0E1FB3A
:40BC400094E701B50F4890F831039DF80010884216D000BF01226946104813F010FC20B99DF80000074981F8310300BF8A20FCF78CFC0B48D0F818130420DFF810C000DFF4
:40BC800008BD0000602A002031AB0C08099F0C08699F0C08B19E0C083005001031030068F8FF002010B5044621463848007863F0C3FE3748047010BD10B53648007848B9F4
:40BCC0003548D0F818130420DFF8D0C000DF0120304908704FF496713148006866F0DFFC40B100212948007863F0A6FE01202D4908700AE02B480078012806D10020294994
:40BD0000087023480078FFF7CDFF10BD2449086070471FB50020009001900290034601221A490390402063F001FF0020009001900290034603221C490390262063F0F6FE0B
:40BD40001FBD10B500241848007864F01FF800EE100AB8EE400ADFED150A20EE200ADFED140A80EE201A134880ED001A90ED000ADFED110AB4EEE00AF1EE10FA01DD01204A
:40BD800000E000200446204610BD00008C0500101C0000201E000020F8FF0020099F0C08180000201D0000208205001000404E3F9BB2263F2000002000803B4510B5A9F0EF
:40BDC00055FA10BD10B5A9F044FA10BD70B505460C4616462078A84203D0257066F042FC60602078217A884208D03146606866F056FC18B120782072012070BD0020FCE762
:40BE00000146887B704770B504460D461646607BA84204D0657366F025FC6060A66070BD0048704768E6001010B5B8F076F8001D10BD00BFB9ED0B002DF055BA000000004A
:40BE40000000000000000000000000000000000000000000000000000000000000000000000000000000000000000000526176656E20496E64757374726965732C20496E79
:40BE8000632E000000000000000000004175672D31382D32303138000000000032322E312E322E310000000000000000526176656E2047756964616E636520436F6E747262
:40BEC0006F6C6C6572000000000000003037373031373134343900000000000000000000000000000000000000000000FFFFFFFFFFFFFFFFFFFFFFFFFFFFFFFFFFFFFFFF30
:40BF0000FFFFFFFFFFFFFFFFFFFFFFFFFFFFFFFFFFFFFFFFFFFFFFFFFFFFFFFFFFFFFFFFFFFFFFFFFFFFFFFFFFFFFFFFFFFFFFFFFFFFFFFFFFFFFFFFFFFFFFFFFFFFFFFF41
:40BF4000FFFFFFFFFFFFFFFFFFFFFFFFFFFFFFFFFFFFFFFFFFFFFFFFFFFFFFFFFFFFFFFFFFFFFFFFFFFFFFFFFFFFFFFFFFFFFFFFFFFFFFFFFFFFFFFFFFFFFFFFFFFFFFFF01
:40BF8000FFFFFFFFFFFFFFFFFFFFFFFFFFFFFFFFFFFFFFFFFFFFFFFFFFFFFFFFFFFFFFFFFFFFFFFFFFFFFFFFFFFFFFFFFFFFFFFFFFFFFFFFFFFFFFFFFFFFFFFFFFFFFFFFC1
:40BFC000FFFFFFFFFFFFFFFFFFFFFFFFFFFFFFFFFFFFFFFFFFFFFFFFFFFFFFFFFFFFFFFFFFFFFFFF00C00008BFE31D0800900008FBBF000800800008F78F000833C43B92A2
:40C00000FC4890F8F805022802D19FEDFB1A01E09FEDFA1AF0EE410AB0EEC01AB4EEE01AF1EE10FA01DD012070470020FCE710B52DED028B17F0D5FD01280BD10AF040FCB9
:40C0400040B9EC4890F840040B2801D1012000E0002048B1E74890F84004072804D0E54890F84004062802D19FEDE58A09E0E14890F84206012802D19FEDE28A01E09FED72
:40C08000E28AB0EE480ABDEC028B10BD10B52DED028B06F097FFB0EE408AFFF7C8FFF0EE408AB4EEE88AF1EE10FA03D20120BDEC028B10BD0020FAE710B52DED028B17F0F2
:40C0C00090FD01280ED10AF0FBFB58B9C94890F840040B2801D1012000E0002010B99FEDC88A16E0C34890F84206012802D19FEDC48A0EE0BF4890F84004072804D0BD4890
:40C1000090F84004062802D19FEDC08A01E09FEDC08AC04824F08CFFB4EEC80AF1EE10FA03DD0120BDEC028B10BD0020FAE710B52DED028B17F055FD01280ED10AF0C0FB1A
:40C1400058B9AC4890F840040B2801D1012000E0002010B99FEDAB8A16E0A64890F84206012802D19FEDA78A0EE0A24890F84004072804D09F4890F84004062802D19FEDEA
:40C18000A28A01E09FEDA48A06F01CFFB4EEC80AF1EE10FA06DDFFF78FFF18B90120BDEC028B10BD0020FAE70146087A0B2804D1487A0A2801D1012070470020FCE7014634
:40C1C000087A042804D1487A022801D1012070470020FCE700B59148FFF7F1FF18B98F48FFF7E2FF08B1012000BD0020FCE70146087A042803D1487A012800D1704700203A
:40C20000FCE70146087A704710B58448FFF7F9FF0F283ED2DFE800F0092124202D1F3D3C083D252E223D0A0000BF00BF794824F008FF08B108240DE0764824F049FF30B9BB
:40C240007748C06C00F48020B0F5802F01D1012400E000241FE000BF00BF00BF01241AE000BF6C4824F038FF08B1052400E0022411E000BF6948FFF7BAFF08B1012406E01B
:40C28000644824F029FF08B1062400E0042402E000BF072400BF00BF204610BD10B517F0AAFC18B101205F49087002E000205D49087010BD01205C490870704710B50446C1
:40C2C000606866F00DFA10BD10B55448FFF7F6FF10BD54480078704710B5044600202060606020726072A0724E4908704E49087066F0B8F94D49086017F040FD10BD38B562
:40C300000446257A207A0F2873D2DFE800F008FB91F7F6F572727272F4F3B3F2F100206924F08FFE002863D1206924F0B3FE08B101255DE0206924F096FE58B12D4890F865
:40C340005308012804D02B4890F85308022801D105254DE0206924F08FFE08B1032547E004F09DFBA0B9A5F089FD88B9A4F012FA70B9A5F0D1FA58B9A3F0B1F940B918F0D1
:40C380003EFBFB2804D01B4890F85308012804D0184890F85308022801D1022528E0206924F061FE58B1134890F85308032804D0104890F85308022801D10C2518E004F006
:40C3C0006EFBA8B9A5F05AFD90B9A4F0E3F978B9A5F0A2FA60B9A3F082F948B918F00FFBFB2805D0034890F85308032800D10A25AAE2A7E2602A00200AD7A33C9A99193ED8
:40C40000E3A5AB403D0A8F4083C000413D0A0F418B6C4F4108000010B81E414178170010500F002000000010010000100400001004F035FBE0B9A5F021FDC8B9A4F0AAF9E6
:40C44000B0B9A5F069FA98B9A3F049F980B918F0D6FAFB280CD0F848007828B10425FFF7ADFC0020F44908700020F449087000E0002569E26946E06827F0FEFB68B100981A
:40C4800027F06EFA012804D0009827F06CFA012803D10D25FFF796FC33E06946E06827F0EBFB40B1009827F05BFA022803D10E25FFF788FC25E004F0F2FA08BB18F09FFA44
:40C4C000FB281DD0A4F066F928B9A5F025FA10B9A3F005F9A0B1D848007828B10B25FFF76DFC0020D44908700020D449087008E0ACE1E9E115E1C9E017E03CE028E001E0B5
:40C50000002521E2206924F0C5FD60B1CA48007828B10425FFF752FC0020C74908700020C649087000E000250EE2206924F09BFD60B1C148007828B10425FFF73FFC002035
:40C54000BD4908700020BD49087000E00025FBE1206924F091FD60B1B748007828B104250020B5490870FFF729FC0020B349087000E00025E8E1607A022842D1AF48007870
:40C58000E0B1206924F094FDC0B1AD4890F84108A0B1206924F051FD17280FD0206924F08CFD172803D1A64890F84E0430B100229FEDA40A03210F20A5F048F804F06FFA68
:40C5C000D8B9A5F05BFCC0B9A4F0E4F8A8B9A5F0A3F990B9A3F083F878B918F010FAFB280BD09648007810B3002094490870924908700225FFF7E6FB47E00025FFF7E2FBAD
:40C6000043E0607A012813D1206924F043FD58B18A48007858B1002088490870864908700125FFF7CFFB30E00025FFF7CBFB2CE0607A032813D1206924F01EFD58B17F48B3
:40C64000007810B300207D4908707B4908700325FFF7B8FB19E00025FFF7B4FB15E0607A052812D1206924F0FEFC58B17348007858B10020714908706F4908700525FFF7F4
:40C68000A1FB02E00025FFF79DFB5DE1607A10B1607A0E2843D104F002FA80BBA5F0EEFB68BBA4F077F850BBA5F036F938BBA3F016F820BB18F0A3F9FB282ED06946E06883
:40C6C00027F0DAFA68B1009827F04AF9012804D0009827F048F9012803D10D25FFF772FB17E06946E06827F0C7FA48B1009827F037F9022804D10E25FFF764FB09E00CE0CB
:40C700004D48007828B10B25FFF758FB00204A49087000204949087002E00E2500E0002512E1607A0A2843D16946474827F0A4FA68B1009827F014F9012804D0009827F0A4
:40C7400012F9012803D10D25FFF73CFB73E069463D4827F091FA40B1009827F001F9022803D10E25FFF72EFB65E004F098F9D8B9A5F084FBC0B9A4F00DF8A8B9A5F0CCF804
:40C7800090B9A2F0ACFF78B918F039F9FB280BD02A48007808B3002028490870264908700025FFF70FFB46E00E25FFF70BFB42E0607A0C283FD16946234827F05DFA68B19A
:40C7C000009827F0CDF8012804D0009827F0CBF8012803D10D25FFF7F5FA2CE069461A4827F04AFA40B1009827F0BAF8022803D10E25FFF7E7FA1EE004F051F9C0B918F0B3
:40C80000FEF8FB2814D0A3F0C5FF28B9A5F084F810B9A2F064FF58B10848007858B1002006490870044908700C25FFF7CBFA02E00025FFF7C7FA87E000000010010000103C
:40C84000602A002000000000604F0010607A0B2805D0607A0A2802D0607A0D2833D16946864827F009FA38B1009827F07FF818B90025FFF7A7FA26E06946804827F0FCF9C0
:40C8800068B1009827F06CF8012804D0009827F06AF8012803D10D25FFF794FA13E004F0FEF880B9A5F0EAFA68B9A3F073FF50B9A5F032F838B9A2F012FF20B918F09FF802
:40C8C000FB2800D00A253FE0607A0B2805D0607A0A2802D0607A0E2833D16946674827F0CBF938B1009827F041F818B90025FFF769FA26E06946614827F0BEF908B300984B
:40C9000027F02EF8E8B9009827F02DF8C8B904F0C6F898B9A5F0B2FA80B9A3F03BFF68B9A4F0FAFF50B9A2F0DAFE38B918F067F8FB2803D00A25FFF745FA02E00E25FFF79C
:40C9400041FA01E0002500BF00BF207AA84202D0207A60722572A07A217A884206D14FF47A714748006865F09AFE58B1207AA07265F078FE424908600B204AF0F3FF372016
:40C98000FBF703FE207A042804D03E4890F85308012807D0207A0B2807D03A4890F85308032802D165F05EFE6060207A38BD0146087A042804D1487A052801D10120704717
:40C9C0000020FCE70146087A042804D1487A032801D1012070470020FCE770B504460025FFF7F8FB38B92046FFF7ECFF18B92046FFF7DDFF38B1206924F06EFB08B106253F
:40CA00001FE004251DE02046FFF7F1FB08B1012517E0207A012808D0207A022805D0207A052802D0207A032807D1206924F054FB08B1052505E0022503E01348007800B107
:40CA40000325284670BD10B5104800BF0446104A1049B6F0BBFE104808490C4A002303604360037243728372C160026100BF0446074A0A49B6F0AAFE10BD0000604F001069
:40CA800004000010602A00200000001008000010008000086B650C0878170010A7640C0870B52DED028B05460C4608F079FA01282AD100EE104AB8EE400ADFEDFD0A80EEF5
:40CAC000201AB0EE418A012D04D0022D0ED0032D17D113E0B1EE480AB0EE408A3AF044FB0646B0EE480A3AF039FE0BE03AF03CFB0646B0EE480A3AF031FE03E03AF04BFFE2
:40CB000000E000BF00BF03E0214628463AF0DFF8BDEC028B70BDE7490870704770B505460E46E548FBF726FC044644B1257066700C222146E148DFF888C300DF17E000BFF8
:40CB4000E04890F8350340F00401DE4880F83513B0F840034FF6FF71884207DAD948B0F84003401C81B2D748A0F8401300BF70BD70B504460D4601221021D3481DF084FF15
:40CB800001280AD0D048447468B2CF498874012008740121CC481EF075F8CB4890F91100002806DDC84A517CC84A1078FFF7B6FF11E0C54890F9110000280CDAC24A92F90D
:40CBC0001160002E01DB324600E07242D1B2BF4A5078FFF7A3FF70BD70B505460C460D2D78D2DFE805F007111C27323D48535E69747576000CB1012200E00022B449885C45
:40CC00000121FFF78BFF65E00CB1012200E00022AF49091D885C0121FFF780FF5AE00CB1012200E00022AA49891D885C0121FFF775FF4FE00CB1012200E00022A449891CCA
:40CC4000885C0121FFF76AFF44E00CB1012100E000219F4A0A3A505C0121FFF75FFF39E00CB1012200E0002299490839885C0121FFF754FF2EE00CB1012200E000229449C2
:40CC8000891F885C0121FFF749FF23E00CB1012200E000228E49091F885C0121FFF73EFF18E00CB1012200E000228949891E885C0121FFF733FF0DE00CB1012200E000221B
:40CCC00083490831885C0121FFF728FF02E000BF00BF00BF00BF70BD70B50026002435E000252FE07B4800EB4400405D78490A3901EB440148550DF018FB98B974480A3889
:40CD000000EB4400405D032806D071480A3800EB4400405D022805D100206D490A3901EB440148556A480A3800EB4400405D38B167480A3800EB4400405D0C2800D00126E7
:40CD4000681CC5B2022DCDDB601CC4B2102CC7DB00201CE0002116E05E4A203202EB4002525C5A4B03EB40035A54584A02EB4002525C32B1554A02EB4002525C0C2A00D09F
:40CD800001264A1CD1B20229E6DB411CC8B20228E0DB304670BD10B524214848DFF838C100DFFFF799FF07F0ADFF4C4808F0E9F84B4808F0E9F810BD2DED028B82B04FF6DA
:40CDC000FF74FFF7E8FF022220213B48BCF0E2FE00286BD100BF224601A93848DFF804C100DF0128F7D0019800780D285FD2DFE800F007080F2131477D9AB282CAD2D300B0
:40CE0000CCE00120A8F05DF90120FFF784FEC5E0ABF0F2FCB1EE400AF2EE040A80EE201AB0EE418A0122B0EE480A03210A20A4F00DFCB3E0ABF0E0FCF2EE040A80EE201AEA
:40CE4000B0EE418A0122B0EE480A03210A20A4F0FDFBA3E00CF0B2FE2348D0EDD90AF2EE041A80EEA11A0198407800EE900AF8EE600A01EE200AB0EE408A0CF046FF8DE0A3
:40CE80000CF09CFE1848D0EDD90AF2EE041A80EEA11A0198407800EE900AF8EE600A01EE600AB0EE408A0CF030FF77E07CE074E000007A4406000020C0170010E0170010C7
:40CEC0007DA10C08F8FF0020AC17001000000020961700109E2D002091A00C08D9CB000871CB000821A20C08602A00209FEDF60A0CF00BFF52E0F54890EDD90AB2EE041A79
:40CF0000C0EE010A0198407800EE100AB8EE400A20EE800ABCEEC00A10EE105A29460320FFF7BEFD3AE0E94890EDD90AB2EE041AC0EE010A0198407800EE100AB8EE400ACD
:40CF400020EE800ABCEEC00A10EE105A29460120FFF7A6FD22E0DD4890EDD90AB2EE041AC0EE010A0198407800EE100AB8EE400A20EE800ABCEEC00A10EE105A29460220C8
:40CF8000FFF78EFD0AE000229FEDCF0A03211046A4F05CFB02E000BF00BF00BF00BFCC480199FBF7F7F916E70521CA4880F834130020DFF824C300DF00BFFEE70220C74925
:40CFC00008700A204870032008710A21C34841710720C24988710021C048C1710820BF4908720021BD4841720120BC4988740021BA48C1740420BA4908700520487006202E
:40D00000B64988700021B548C170704710B500BF2022B249B34812F032FA20B92022AF49B148B6F013FD00BF00BF0422AC49AD48203012F024FA20B9A448A9490968C0F869
:40D040005E1300BF10BD0020A8490978112905D0A249A64A127811F8120015E0A4490978032911D000209E49A14A127811F81210082901D10A2007E099499D4A127811F80B
:40D080001210042900D10B20704710B502460020022A22DA032920DA012902D0022912D108E008238E4C04F81230072304EB4204637010E004238A4C04F81230052304EB4A
:40D0C0004204637007E00023854C04F8123004EB4204637000BF00BF012010BD10B502460020102A14DA0B2912DA7C4B03F81210022901D0032905D10A23784C04EB42040D
:40D10000637004E00023754C04EB42046370012010BD70B5044600267448007811280AD02546092D01DD0025022629466F480078FFF7D4FF1BE06E480078032817D00CB94F
:40D1400000250EE00A2C02DA0025032609E00A2C01D1012505E00B2C01D1022501E000250226294662480078FFF78FFF00BFFFF74DFFF820FBF709FA304670BD10B52DED3D
:40D18000020B00249DED000A5FEDB70AB4EEE00AF1EE10FA05DD1FEDBA0A8DED000A02240BE09DED000AB5EEC00AF1EE10FA04D29FED450A8DED000A032400BF0422694607
:40D1C0004848263012F05BF920B99DED000A3F4880EDD90A00BFF620FBF7D7F920461CBD31B500249DF80000012803DD01200090022406E09DF80000002802DC0020009029
:40D20000032400BF012269463A4812F038F920B99DF800002D4981F8FA0000BFF720FBF7B4F9FA20FBF7B1F9204638BD00202F490978112902D02D49087807E02C490978AC
:40D24000032903D02A49097801F10A00704770B504462546012D00DD012525480570112022490870F820FBF790F970BD70B504462546092D00DD00251C48057003201C49D4
:40D280000870F820FBF781F970BD70B5044600250B2C01DB022500240A2C03DAE0B2FFF7E5FF04E0A4F10A01C8B2FFF7D0FF284670BD0F48007818B10D480078012801D116
:40D2C000012070470020FCE700000000602A0020C0170010F8FF0020C5A90C088C170010000000203E0300689E2D00200400002005000020FA00006810480078704731B5AA
:40D3000000240F4890F80B069DF8001088420FD000BF012269460B48006800F20B2012F0AEF820B99DF80010054880F80B1600BFFB20FBF72AF9204638BD000006000020A6
:40D34000602A00202001001010B504462046A0F085F90446204610BD70B504462046FFF7F3FF0546B9F0EAF970BD70B50546012406E0634B002221462846A0F023FA641CC4
:40D38000062CF6D370BD0021C16001610177704710B504462046A0F05BF90446594820602046FFF7F0FF564B052257492046A0F082F9204610BD10B55448007800F001008D
:40D3C00078B95248B9F00BFA58B15148FFF7E0FF0446504AAFF28F01B6F0F8F94B48AFF300804B4810BD70B50446208B85B24A48B0F85C0461690844A061A069A84205D0B2
:40D400003F4B002204212046A0F0DCF970BD70B50446A08A85B20CF08EFBD4E90321891A00FB01F60CF077FB96FBF0F0E168084460616069A84208D0314B00220321204670
:40D44000A0F0C0F92046FFF7CEFF70BD38B504460D46E068A8420ED0E560294B002201212046A0F0AFF92D4800902D4B03212D48E2684FF0F7FC38BD38B504460D4620693E
:40D48000A8420FD025611E4B002202212046A0F099F922480090224B03212248401E22694FF0E0FC38BD70B505460E46144631462846FFF7E1FF21462846FFF7C7FF284621
:40D4C000FFF7A5FF70BD0146C868704701460869704701464869704701468869704770B504460D46207FA84206D02577044B002205212046A0F066F970BD0146087F7047CF
:40D5000081640C08ECB21D086785000808000020B009002000800008602A0020406B0220985D0220AF040800012904D002290BD003291BD111E042F2107242436423B2FBED
:40D54000F3F2FE4B1A8012E042F2107242436423B2FBF3F2FA4B1A8009E042F2107242436423B2FBF3F2F74B1A8000E000BF00BF704710B50446F44800882044F249088096
:40D580000846008842F21071884202DB0020EE490880ED480088E9490988884205DA0121EA48007862F048FA04E00021E748007862F042FAE4480088E1490988884205DA7F
:40D5C0000121E348007862F037FA04E00021E048007862F031FADC480088DA490988884205DA0121DB48007862F026FA04E00021D848007862F020FA10BD70B5054665F0EE
:40D6000031F804460020D44988614FF47A71D248C1614462002180F8281003210020FFF783FF0020CC49C8624FF47A71CA4801638463002180F83C1002210020FFF774FF39
:40D640000020C54948604FF47A71C348816004610021017501210020FFF766FF0020BE4908644FF47A71BC484164C464002180F850100020B84948654FF47A71B6488165B6
:40D680000466002180F86410122D7DD2DFE805F009233D569CC1F1EFEEEDECEBEAE9E8E7E6E54FF4FA70AC4988610146AA48C1614462012180F82810014691ED080ABCEEAF
:40D6C000C00A10EE101A88B20321FFF72DFF0120A149087007E34FF4FA709F49C86201469D4801638463012180F83C10014691ED0D0ABCEEC00A10EE101A88B20221FFF764
:40D7000013FF012094490870EDE24FF4FA7092494860014690488160046101210175014691ED030ABCEEC00A10EE101A88B20121FFF7FAFE012088490870D4E2022086499C
:40D74000087032204860322183488160046100210175014691ED030ABCEEC00A10EE101A88B20121FFF7E0FE4FF4FA607A4948650021794881650466012180F86410002031
:40D78000FFF7D2FE032100E0ACE20020FFF7CCFE02210020FFF7C8FE02206F4981F8680002216D4880F8691080F86A1080F86B1080F86C10042180F86D10062180F8771095
:40D7C000002180F878108EE24FF4FA7062490864014661484164C464012180F85010014691ED080ABCEEC00A10EE101A88B20321FFF79AFE584991ED030ABCEEC00A10EE20
:40D80000101A88B20121FFF78FFE01205249087069E264205049086464214F484164C464012180F85010014691ED080ABCEEC00A10EE101A88B20321FFF776FE464991EDAC
:40D84000030ABCEEC00A10EE101A88B20121FFF76BFE01204049087045E213E2E1E1AFE169E123E1BDE0EEE086E04FE035E01AE0FFE74FF47A703849886100213648C16119
:40D880004462012180F82810014691ED080ABCEEC00A10EE101A88B20321FFF745FE01202D4908701FE24FF47A702B49C8620021294801638463012180F83C10014691ED83
:40D8C0000D0ABCEEC00A10EE101A88B20221FFF72BFE01202049087005E24FF47A701E49486000211C488160046101210175014691ED030ABCEEC00A10EE101A88B20121A7
:40D90000FFF712FE012014490870ECE14FF47A7011490864002110484164C464012180F85010014691ED080ABCEEC00A10EE101A88B20321FFF7F8FD07490FE00E000020C2
:40D94000100000201200002014000020660500108105001067050010D009002091ED030ABCEEC00A10EE101A88B20121FFF7DCFD0120FE490870B6E10220FC4908704FF4A0
:40D98000FA7088610021F948C161446280F82810014691ED080ABCEEC00A10EE101A88B20321FFF7C1FD4FF4FA70F049C8620021EE4801638463012180F83C1002210020DA
:40D9C000FFF7B2FD0120E94981F868000021E74880F86910022180F87710002180F8781081E10220E14908704FF4FA7088610021DE48C161446280F82810014691ED080A78
:40DA0000BCEEC00A10EE101A88B20321FFF78CFD4FF4FA70D54948600021D44881600461017501210020FFF77FFD0120CF4981F868000221CD4880F8691080F877100021EA
:40DA400080F878104FE10220C84908704FF4FA70C8620021C54801638463012180F83C10014691ED0D0ABCEEC00A10EE101A88B20221FFF759FD4FF4FA70BC4948600021F9
:40DA8000BA4881600461017501210020FFF74CFD0020B64981F868000221B44880F8691080F87710002180F878101CE10220AF4908704FF4FA7088610021AC48C1614462F5
:40DAC000012180F82810014691ED080ABCEEC00A10EE101A88B20321FFF726FD4FF4FA70A249C8620021A1480163846380F83C1002210020FFF718FD4FF4FA709B49486008
:40DB000000219A4881600461017501210020FFF70BFD0120954981F868000021934880F86910022180F86A10032180F87710002180F87810D7E002208C49087040F24D100B
:40DB4000886100218948C1614462012180F82810014691ED080ABCEEC00A10EE101A88B20321FFF7E1FC40F24D108049C86200217E480163846380F83C1002210020FFF7DB
:40DB8000D3FC40F24D10794948600021774881600461017501210020FFF7C6FC0120734981F868000021714880F86910022180F86A10032180F87710002180F8781092E0B3
:40DBC00002206A4908704FF4FA70886100216748C161446280F82810014691ED080ABCEEC00A10EE101A88B20321FFF79DFC4FF4FA705E49086400215C484164C464012126
:40DC000080F850100120594981F868000321574880F86910022180F87710002180F8781061E00220514908704FF4FA70C86200214E480163846380F83C10014691ED0D0A83
:40DC4000BCEEC00A10EE101A88B20221FFF76CFC4FF4FA7045490864002144484164C464012180F850100020404981F8680003213E4880F86910022180F87710002180F852
:40DC8000781030E00220394908704FF4FA70486000213648816004610175014691ED030ABCEEC00A10EE101A88B20121FFF73CFC4FF4FA702D49086400212C484164C46417
:40DCC000012180F850100220284981F868000321264880F86910022180F87710002180F8781000E000BF00BF2148057070BD20B1012806D002280CD107E01C4981ED0D0ADF
:40DD000008E01A4981ED080A04E0184981ED030A00E000BF00BF0121164A1170704770B5002515480078E0B980211048B5F071FF9FED120A0020FFF7DAFF9FED110A02201A
:40DD4000FFF7D5FF9FED0D0A0120FFF7D0FF0020064981F879000220FFF74FFC01200649087064F07FFC044600480BE0D00900200C0000200D000020160000200000A042EE
:40DD80000000C84290F87900002845D162F00CFAFF280ED1FD480078022803D1FC480078012805D10220FFF728FC0020F84908709BE0012048F084FF70B9F44800780528D0
:40DDC00003D1F34800780128F2D10520FFF715FC0020EF49087088E002F00BFF70B1EB480078042803D1EA48007801287DD10420FFF703FC0020E649087076E0E34800788A
:40DE000018B9E348007801286FD10020FFF7F5FB0020DF49087068E0DE4890F8790001280ED1DA4800780E2803D1D948007801285BD10E20FFF7E1FB0020D549087054E04C
:40DE4000D44890F87900022815D1D249C86F4FF47A6164F024FC70B9CC480078082803D1CB480078012840D10820FFF7C6FB0020C749087039E0C74890F87900042815D151
:40DE8000C449C86F4FF47A6164F009FC70B9BF480078072803D1BE480078012825D10720FFF7ABFB0020BA4908701EE0B94890F87900032815D1B749C86F4FF47A6164F047
:40DEC000EEFB70B9B1480078062803D1B048007801280AD10620FFF790FB0020AC49087003E00020AB4981F87900AA480078012802D002287DD1F9E0A64890F83C00E0B90B
:40DF0000A448C06AC8B1A348816B204664F0F7FBA049096B88422AD301219E4880F83C108463014691ED0D0ABCEEC00A10EE101A88B20221FFF7F8FA19E0964890F83C00A0
:40DF4000012814D19348006B88B19248816B204664F0D5FB8F49C96A884208D300218D4880F83C10846302210020FFF7DDFA8948007DD8B987484068C0B1864801692046FE
:40DF800064F0BDFB83498968884227D30121814801750461014691ED030ABCEEC00A10EE101A88B20121FFF7BFFA17E07948007D012813D17748806880B1764801692046ED
:40DFC00064F09DFB73494968884207D3002171480175046101210020FFF7A6FA6D4890F82800F0B96B488069D8B16A48416A204600E008E264F083FB6649C96988422AD35D
:40E000000121644880F828104462014691ED080ABCEEC00A10EE101A88B20321FFF784FA19E05C4890F82800012814D15948C06988B15848416A204664F061FB5549896928
:40E04000884208D30021534880F82810446203210020FFF769FA4F4890F8500038BB4D48006C20B34B48C16C204664F048FB4949496C884239D30121464880F85010C4648C
:40E08000014691ED080ABCEEC00A10EE101A88B20321FFF749FA3F4991ED030ABCEEC00A10EE101A88B20121FFF73EFA1DE0394890F85000012818D13648406CA8B13548B5
:40E0C000C16C204664F01BFB3249096C88420CD30021304880F85010C46403210020FFF723FA01210020FFF71FFA8CE1294890F878106830405C38BB264890F83C000128D9
:40E1000017D12448816B204664F0F9FA2149C96A88420DD300211F4880F83C10846302210020FFF701FA1B48006B002800D10125D2E01848816B204664F0E1FA1549096BF2
:40E140008842F5D30125C7E0124890F878106830405C02282BD10F48007D01281CD10D480169204664F0CBFA0A4949688842DFD3002108480175046101210020FFF7D4F983
:40E1800004488068002800D10125A5E00C0000200D000020D00900209C480169204664F0AEFA9A498968884200D3012594E0974890F878106830405C012826D1934890F8D4
:40E1C0002800012816D19148416A204664F097FA8E49896988427FD300218C4880F82810446203210020FFF79FF98848C06990BB012571E08548416A204664F080FA8349E3
:40E20000C969884268D3012566E0804890F878106830405C03282AD17C4890F8500001281AD17A48C16C204664F069FA7749096C884251D30021754880F85010C464032128
:40E240000020FFF771F901210020FFF76DF96F48406C00B901253FE06C48C16C204664F04EFA6A49496C884236D3012534E0674890F878106830405C04282DD1634890F877
:40E28000640001281ED16148016E204664F037FA5E49496D88421FD300215C4880F86410046602210020FFF73FF903210020FFF73BF901210020FFF737F95448806D58B9CA
:40E2C000012509E05148016E204664F018FA4F49896D884200D30125012D28D100254B4890F87800401CC1B2484880F8781090F8781090F87700814203DB0021434880F8D8
:40E300007810424890F878106830405C80B901213E4880F83C108463014691ED0D0ABCEEC00A10EE101A88B20221FFF7FDF869E0364890F878106830405C02280FD1012104
:40E34000324801750461014691ED030ABCEEC00A10EE101A88B20121FFF7E6F852E02B4890F878106830405C012810D10121274880F828104462014691ED080ABCEEC00A85
:40E3800010EE101A88B20321FFF7CEF83AE01F4890F878106830405C03281BD101211B4880F85010C464014691ED080ABCEEC00A10EE101A88B20321FFF7B6F8134991ED6B
:40E3C000030ABCEEC00A10EE101A88B20121FFF7ABF817E00D4890F878106830405C042810D10121094880F86410046602210020FFF79AF803210020FFF796F80121002044
:40E40000FFF792F800BF00BF70BD0000D009002070B5D4201CE0C41700EBD4646511E34C54F82540C51700EBD5656D11A0EB45160125B5402C40C51700EBD5656D11A0EB59
:40E4400045160125B540AC4200D103E0411EC8B20028E0DC00BF70BD10B50024D448006868B14FF47A71D248006864F018F930B180F033FF18B1CF48007800B90124204621
:40E4800010BD30B5C31700EBD3635C11C74B383353F824300246C41700EBD4646411A0EB44150124AC4023430146C41700EBD4646511BE4C383444F8253030BDBE4A5054B5
:40E4C000704730B5C31700EBD3635C11B74B53F824300246C41700EBD4646411A0EB44150124AC40A3430146C41700EBD4646511AE4C44F82530C31700EBD3635C11AB4B3D
:40E500001C3353F82430C41700EBD4646411A0EB44150124AC40A343C41700EBD4646511A24C1C3444F82530C31700EBD3635C119E4B383353F82430C41700EBD46464118E
:40E54000A0EB44150124AC40A343C41700EBD4646511964C383444F8253030BD30B50146CB1701EBD3635C11904B53F82430CC1701EBD4646411A1EB44150124AC40234094
:40E580000BB1012030BD0020FCE701468B48405C012800D170470020FCE713B5044600BF87490819012201A910F069FF20B9BDF80400C1B28348015500BF1CBD13B504465D
:40E5C00000BF814901EB4400022201A910F057FF20B9BDF804107D4820F8141000BF1CBD7CB504460D46E8B20190280A009000BF7149FF3960180122694610F040FF20B935
:40E60000BDF80000C1B27248015500BF00BF71496018012201A910F032FF18B99DF804106D48015500BF7CBD2DE9F0412DED028B04466A4890ED241BB0EE410AF0EE610A9F
:40E6400051EC100BBCF0A6FB08EE100A9FED640AC8EE000ABCEEE00A10EE100AC6B29FED610AC8EE000ABCEEE00A10EE100A80B23C2190FBF1F201FB1200C7B271025A480B
:40E6800090F8200041EA0010574991F8211008431FFA80F85048015D4D48005D41EA0025B5F57A7F01DA681C85B229462046FFF797FF41462046FFF781FF39462046FFF731
:40E6C0006CFFBDEC028BBDE8F081014641B1292905D02F2902D0302904D100BF00BF00BF002001E0012000BF00BF70470146A62914D006DC912909D0A32909D0A52911D153
:40E7000008E0B92908D0BA290CD109E000210BE01A2109E01B2107E01E2105E0252103E0282101E0084600BF00BF704770B58CB004460D4680F0D1FD48B32C4B2CA2232181
:40E7400002A80094B4F01EFD02A8B5F009F9461C324602A929489BF0EBFA2046FFF7C6FF2749087008460078FFF7AFFF40B13DB123480078FFF758FF2148007898F07EFA82
:40E78000A120F9F702FFE020F9F7FFFE00BF0CB070BD1B4800787047F0B52DED028B83B005460024682D2DD22DE00000540F002010000010E7220010FF0400683410002066
:40E7C000FE1E0068C2370020001D0068C4350020C4320020001C0068C4340020582000200000614500007042A01E002050E00C08257320636F64653A20256400BCDD00103B
:40E800000D000010FAE0DFE805F034FA353A3BF9F9F9F9F9F93C465B6D828396ACBFFFF7F6F5F4F3F9F9F9F9F9F2F1F0EFEEF9F9F9F9F9F9F9F9EDECEBF9F9EAF9E9E8E7B9
:40E84000E6E5E4E3E2E1E0DFF9F9F9F9F9F9F9DEDDDCDBDAD9F9F9F9F9F9D8D7D6D5F9F9F9F9D4D3F9F9F9D2F9F9F9F9F9F9F9D1D0CF90E261F0D1FD80F001048BE28AE2F3
:40E8800089E202F019FC28B963F0ECFEF849884200D901247FE202F00FFC80B104F000FC68B1F44890ED220ADFEDF30AB4EEE00AF1EE10FA02DC90F8900000B901246AE2E4
:40E8C00002F0FAFB68B104F0EBFB50B1E94890ED220ADFEDEA0AB4EEE00AF1EE10FA00D2012458E202F0E8FB80B104F0E2FB68B1E34890ED0C0ADFEDE30AB4EEE00AF1EE2B
:40E9000010FA02DC90F8380000B9012443E242E216F075F8FA280DD116F071F8FB2809D007F09BFC20B107F0DDFB08B1012000E0002004462FE216F062F8FA2810D116F05E
:40E940005EF8FB280CD007F08EFC38B107F0CAFB20B107F0D4FB08B1012000E00020044619E216F04CF8FA280DD116F048F8FB2809D007F07EFC20B107F0B4FB08B1012018
:40E9800000E00020044606E216F039F8FA283AD116F035F8FB2836D007F071FC80B307F0A1FB68B301202DE0E0E1CCE1C3E1BEE1B7E1B1E183E17EE178E172E16CE151E129
:40E9C0004BE145E13FE139E12BE11DE117E111E10BE105E1FFE0F9E0F3E0EDE0E7E0D0E0CAE0C0E0B6E099E074E18FE086E07DE069E055E041E02DE019E005E0CAE1C1E040
:40EA0000FFE700200446C6E115F0F9FFFA280DD115F0F5FFFB2809D007F037FC20B107F061FB08B1012000E000200446B3E115F0E6FFFA280DD115F0E2FFFB2809D007F024
:40EA400035FC20B107F04EFB08B1012000E000200446A0E115F0D3FFFA280DD115F0CFFFFB2809D007F028FC20B107F03BFB08B1012000E0002004468DE115F0C0FFFA2878
:40EA80000DD115F0BCFFFB2809D007F021FC20B107F028FB08B1012000E0002004467AE115F0ADFFFA280DD115F0A9FFFB2809D007F008FC20B107F015FB08B1012000E057
:40EAC0000020044667E115F09AFFFA280DD115F096FFFB2809D007F001FC20B107F002FB08B1012000E00020044654E102F01FFB08B9012000E0002004464CE104F09EFA2D
:40EB0000012800D100E00020044644E121F063FD08B9012000E0002004463CE115F06FFFFA2803D015F06BFFFB2812D15648D0ED020A5648B0F8F80000EE100AB8EE400A38
:40EB4000F4EEC00AF1EE10FA01D8012000E00020044620E14E4890F82D0108B9012000E00020044617E14A4890F8B90508B9012000E0002004460EE102F0C8FA80F001042F
:40EB800009E108E115F037F870B115F038FFFA280AD03F4890F84308012805D03D4858F0B7FA08B9012000E000200446F3E004F032FE00F00104EEE004F02DFEC0F3400423
:40EBC000E9E004F028FEC0F38004E4E004F023FEC0F3C004DFE004F01EFEC0F30014DAE004F019FEC0F34014D5E004F014FEC0F38014D0E004F00FFEC0F3C014CBE004F070
:40EC00000AFEC0F30024C6E004F005FE00F4007020B130F047FA08B1012000E000200446B9E004F0F8FD00F4806020B130F03AFA08B1012000E000200446ACE004F0EBFD97
:40EC4000C0F38044A7E004F0E6FDC0F3C044A2E004F0E1FDC0F300549DE004F0DCFDC0F3405498E004F0D7FDC0F3805493E00000E09304006816002000009643000048426A
:40EC8000A01E002000401C466032002058200020602A0020986C022004F0BDFDC0F3C05479E004F0B8FDC0F3407474E004F0B3FDC0F380746FE004F0AEFDC40F6BE002F03F
:40ECC000FBF930B10BF031FB18B146F0BFF900B1012460E0FDF7FDFAB0B9FDF77BFA58B9FC48FDF784FA38B9FA48FDF76BFE18B9F848FDF75CFE08B1012000E000200128D5
:40ED000002D007F0F1FA30B115F0F4FD08B1012000E0002004463EE010F046FB80F0010439E0002400BF00BF00BF00BF33E002F0C3FD04462FE021F07DFC08B9012000E0AD
:40ED40000020044627E007F0BBFD60B1E24890F840040B2807D007F0F2F910B906F055F908B1012000E00020044614E004F0EBFE78B1D94890F8430601280AD015F03FFE1E
:40ED8000FA2806D10BF0D1FA18B9012401200CF0C2FA00E000BF00BF15F031FEFB2801F00682CD4890F843080128F8D0702D7DD04ADC542D7BD026DC1C2D79D012DC092D2A
:40EDC00077D008DC052D75D0062D74D0072D61D0082D71D1B3E00A2D6FD01A2D6ED01B2DF7D15FE1252D6AD006DC1D2D68D01E2D67D0242DEDD1DFE1282D7DD02A2D69D0CD
:40EE00002B2DE6D111E2A5F155001B2854D2DFE810F03102430265025300530053005205BB00530025012D011B015300850290025300530053005300A702BF025300530040
:40EE4000D002E602FC021103A5F171002028DDD2DFE810F0300345036E0384039903AE03C303D803F60327043604450465047A048D04A204BD04D104DA041205F404510502
:40EE80009505C405F305240655068606B206DE060507190707F01CF9C8B906F081F8012802D13CF02BFB90B98C480BE0DCE2C4E125E14CE027E03AE0F2E3B7E0DEE086E086
:40EEC0003CE15AE158F024F908B9012000E00020044622E2804890F84508032810D07E4890F8450802280BD07B4890F84508012804D119F0F4FE00E073E108B9012000E056
:40EF000000200446E5E708F05CFE20B108F0E8FF08B1012000E0002004463CB1FFF739FC052803D000210520FFF700FCD1E707F06DFD08B9012000E000200446C9E709F037
:40EF400039FC08B1012000E000200446C1E76448FCF756FF98B96348FCF752FF78B96248FCF74EFF58B96148FCF74AFF38B96048FCF746FF18B95F48FCF742FF08B10120F4
:40EF800000E000200446A4E75548FCF739FF012818D05448FCF734FF012813D05248FCF72FFF01280ED05148FCF72AFF012809D04F48FCF725FF012804D04E48FCF720FF09
:40EFC000012801D1012000E00020044681E707F077FC50BB07F05DFC38BB07F06AFC20BB07F05FFC08BB3E48FCF70AFF022818D03C48FCF705FF022813D03B48FCF700FFAD
:40F0000002280ED03948FCF7FBFE022809D03848FCF7F6FE022804D03648FCF7F1FE022801D1012000E00020044652E708F058FF80F001043CB1FFF7ACFB0A2803D000217F
:40F040000A20FFF773FB44E707F068F828B105F0F5FF10B939F02AF804463AE705F0D5FF18B107F04CF980F0010432E707F067F818B107F044F980F001042AE707F020FCF7
:40F0800078B907F006FC60B907F013FC48B907F008FC30B9A6F085F808B9012000E00020044616E707F00CFC40B907F0F2FB28B907F0FFFB10B907F0F4FB20B1064890F8E2
:40F0C000530803281AD1A6F093F8012814D0012013E0000078170010602A0020986C022044D5022054D5022064D5022084D5022094D50220A4D5022000200446E9E615F02E
:40F100007EFCFA2819D115F07AFCFB2815D0FDF70EF880B1FDF75EF858B9FB48FDF767F838B9F948FDF74EFC18B9F748FDF73FFC08B1012000E000200446CAE615F05FFCC7
:40F14000FA2819D115F05BFCFB2815D0FCF7B4FF80B1FDF73FF858B9EB48FDF748F838B9E948FDF72FFC18B9E748FDF720FC08B1012000E000200446ABE615F040FCFA283C
:40F1800019D115F03CFCFB2815D0FCF77FFF80B9FDF720F868B9DC48FDF729F848B9DA48FDF710FC28B9D848FDF701FC08B9012000E0002004468CE615F021FCFA280FD139
:40F1C00015F01DFCFB280BD0D04890F80501012804D10FF0F8FA08B9012000E00020044677E607F06DFBF8B907F053FBE0B907F060FBC8B907F055FBB0B9FCF7EBFF58B976
:40F20000C148FCF7F4FF38B9BF48FDF7DBFB18B9BD48FDF7CCFB38B1A4F00CFA012801D0012000E00020044653E614F0E4FC08B9012000E0002004464BE607F041FBC0B97E
:40F2400007F027FBA8B907F034FB90B907F029FB78B9AF48C06800F40010B0F5001F06D09FEDAC0AABF06EFE08B1012000E0002004462EE607F024FB68B907F00AFB50B9DF
:40F2800007F017FB38B907F00CFB20B99FEDA20AABF058FE04461CE6FCF79CFF58B99A48FCF7A5FF38B99848FDF78CFB18B99648FDF77DFB88B1994890F8530802280CD086
:40F2C000964890F85308032807D003F07BFEB0EE408AFCF795FE80F00104FAE515F08FFBFA281AD115F08BFBFB2816D00FF0A0F978B907F0E5FA40B907F0CBFA28B907F041
:40F30000D8FA10B907F0CDFA28B14220A5F0FDF808B1012000E000200446FFE1A6F0B7F820B9A6F07FFB08B1012000E000200446F4E115F064FBFA2811D115F060FBFB2899
:40F340000DD005F02DFE012809D006F0F8FE20B146F038F908B9012000E000200446DDE10BF007F888B16D4890F8F90501280CD105F054FEF0EEC00A9FED690AF4EEC00A72
:40F38000F1EE10FA01DB012000E000200446C5E10CF00EFB20B121F013F908B1012407E00CF028FB20B121F00BF9012800D00124B4E15A4890F85604352110FB01F059498F
:40F3C00001EB001090F83600012800D100E0002020B90BF097F8012800D101249EE14F4890F85308022804D04C4890F8530803280AD102A94C4857F0DFF820B1029856F055
:40F4000089FC80F0010400BF88E1444890F85308022804D0414890F85308032809D102A9414857F0C9F818B1029856F021FC044600BF73E1394890F85308032813D137487B
:40F4400090F8120801280ED002A9374857F092F840B1029859F0F0FC20B9029859F00FFD80F0010400BF59E12C4890F8530803281FD12A4890F8120801281AD002A92A483C
:40F4800057F078F898B1029859F0F9FC78B101A9264824F0F1FB50B1019824F05EFA022805DD029859F0F4FC80F0010400E0002400BF33E1194890F8530803280ED1174855
:40F4C00090F81208012809D002A9174857F052F818B1029859F0C5FC044600BFFBE30F4890F85308022804D00C4890F85308032809D102A90C4857F05FF818B1029856F0BF
:40F5000056FC044600BFE6E37817001058200020500F00205677563D950A863E602A0020950A063FC0E60C08986C0220604F0010F74890F8530803280FD1F54890F81208F5
:40F5400001280AD002A9F34824F096FB20B1029824F036FA80F0010400BFBCE3EC4890F8530803280ED1EA4890F81208012809D002A9E84824F080FB18B1029824F00EFA9B
:40F58000044600BFA7E3E24890F8530803280ED1DF4890F81208012809D002A9DD4824F06BFB18B1029824F000FA044600BF92E3D74890F8530803280ED1D54890F81208D2
:40F5C000012809D002A9D34824F056FB18B1029824F0D2F9044600BF7DE3CD4890F8530803280ED1CA4890F81208012809D002A9C84824F041FB18B1029824F0C4F90446F2
:40F6000000BF68E3C24890F85308032817D1C04890F81208012812D0BD4890F840040B280DD0BD48007850B902A9BA4824F024FB20B101A9B94856F09DFF00BF00BF4AE3BB
:40F64000B34890F85308032829D1B14890F81208012824D0AE4890F840040B281FD002A9AC4824F009FBC8B1029824F0A9F998B1AA4857F098FB20B1A84857F094FB042893
:40F680000AD103F09FFCDFEDA60AB4EEE00AF1EE10FA01DD012000E00020044600BF1AE318E39B4890F85308032808D1984890F81208012803D09B4859F0C3FF04460AE383
:40F6C000934890F85308032808D1914890F81208012803D094485BF061F80446FBE28C4890F85308032819D1894890F81208012814D00021874824F0A4FA78B1894859F0F9
:40F7000080FF00F0010028B9864859F07AFF00F0020008B1012000E000200446DBE27C4890F8530803280ED1794890F81208012809D00021774824F084FA20B1794859F0B2
:40F7400060FFC0F3C004C6E2714890F8530803280CD16F4890F81208012807D072485AF0C4FE08B1012000E000200446B3E2684890F8530803280ED1654890F8120801287A
:40F7800009D002A9654856F0F5FE18B1029859F053FB044600BF9EE25D4890F85308022804D05B4890F8530803280FD1584890F840040B2809D002A9584856F0FDFE20B170
:40F7C000029856F011FB80F0010400BF83E220F01BFEDFED560A20EE200AB0EE408AB3EE0E0AB4EEC08AF1EE10FA01DD012000E0002004466FE24E48407B20B905F0D0FB7D
:40F80000012800D1012466E2414890F85308022804D03F4890F8530803280ED102A93F4856F0CAFE48B13A4890F840040B2804D0029856F0DEFA80F001044CE2344890F896
:40F840005308022804D0324890F85308032812D12F4890F840040B280CD002A92F4856F0ABFE38B12D4857F04FFC012800D100E00020044600BF2EE2254890F853080228E4
:40F8800004D0234890F85308032813D1204890F840040B280DD002A9204856F08DFE40B11E4857F031FC022801D1012000E00020044600BF0FE2164890F85308032819D1B7
:40F8C000134890F81208012814D00021114824F0B8F978B1134859F0BAFE164BC01A71F1050105D20F4859F0B6FC08B1012000E000200446EFE1064890F85308022804D04B
:40F90000034890F85308032816D1012015E00000602A0020604F0010E7220010986C02200AD7A33CA86E0220CCD10010E12E654274D50220529E5C1F002001281ED100213F
:40F94000EE4857F0BCFBC8B102A9EC4856F012FEA0B1EB4890F840040B2801D1012000E0002058B9029859F042FAB5EEC00AF1EE10FA01D1012000E000200446ABE1E048B8
:40F9800090F85308022804D0DD4890F85308032801D1012000E0002001281ED10021D74857F08DFBC8B102A9D44856F0E3FDA0B1D34890F840040B2801D1012000E0002055
:40F9C00058B9029859F016FAB5EEC00AF1EE10FA01D1012000E0002004467CE1C84890F85308022804D0C64890F85308032801D1012000E0002001281ED10021BF4857F08C
:40FA00005EFBC8B102A9BD4856F0B4FDA0B1BC4890F840040B2801D1012000E0002058B9029859F0E1F9B5EEC00AF1EE10FA01D1012000E0002004464DE1B14890F853089B
:40FA4000022804D0AE4890F85308032801D1012000E00020012820D10021A84857F02FFBD8B102A9A54856F085FDB0B1A44890F840040B2801D1012000E0002068B9029812
:40FA800059F0B5F9DFED9F0AB4EE600AF1EE10FA01D1012000E0002004461CE1984890F85308022804D0964890F85308032801D1012000E00020012820D100218F4857F0B2
:40FAC000FEFAD8B102A98D4856F054FDB0B18C4890F840040B2801D1012000E0002068B9029859F087F9DFED870AB4EE600AF1EE10FA01D1012000E000200446EBE08048A1
:40FB000090F85308022804D07D4890F85308032801D1012000E00020012820D10021774857F0CDFAD8B102A9744856F023FDB0B1734890F840040B2801D1012000E00020B2
:40FB400068B9029859F050F9DFED6E0AB4EE600AF1EE10FA01D1012000E000200446BAE0674890F85308022804D0654890F85308032801D1012000E0002001281BD102A92A
:40FB80005E4856F019FDB0B15D4890F840040B2801D1012000E0002068B9029856F0EAF838B1029856F0FEF8B0F5FA6F01DA012000E0002004468EE0514890F85308022841
:40FBC00004D04F4890F85308032801D1012000E0002001281BD102A9484856F0EDFCB0B1474890F840040B2801D1012000E0002068B9029856F0BEF838B1029856F0D2F8EE
:40FC0000B0F5FA6F01DB012000E00020044662E03B4890F85308022804D0394890F85308032801D1012000E00020012816D102A9324856F09FFC88B1314890F840040B2880
:40FC400001D1012000E0002040B9029859F0FCF8022801D1012000E0002004463BE0284890F85308022804D0254890F85308032801D1012000E00020012803D11F4857F0D5
:40FC80006CFA044627E01E4890F85308022804D01B4890F85308032801D1012000E00020012816D102A9154856F064FC88B1144890F840040B2801D1012000E0002040B9A4
:40FCC000029859F0A4F8022801D1012000E00020044600E000BF00BF06F0F2FD40B906F0D8FD28B906F0E5FD10B906F0DAFD58B1A5F15A007B287DD207E00000986C0220D0
:40FD0000602A002000F07F4551E2DFE800F03E7373737373734D73736273737373738094737373737373737373737373737373737373737373737373737373737373737343
:40FD4000737373737373A3F3F8FDECEBEAE9E8E7E6E5E4E3E2E1E0DFDEDDDCDBDAD9D8D7D6D5D4D3D2D1D0CFCECDCCCBCAC9C8C7C6C5C4C3C2C1C0BFBEBDBCBBBAB9B8B715
:40FD8000B6B5B4B3B2B1B0AFAE00A4F0AAFBF74BC01A71F1050104D207F032F908B1012000E00020044601E211F078FD06460F46A4F0F9FB301A8F4108D207F017F928B1D2
:40FDC000EB480078022801D1012000E000200446ECE111F063FD06460F46A4F0E4FB301A8F4111D207F002F970B15FF008FD28B9DF4800E0D9E10078012803D0DC48007899
:40FE0000032801D1012000E000200446CEE111F045FD06460F46A4F0C6FB301A8F4107D207F0E4F820B15FF0EAFC08B1012000E000200446BAE137F015FBB5EEC00AF1EE64
:40FE400010FA04D105F0ACF8012800D100E000200446ABE10120A4F058FB28B1C54857F057F908B9012043E041E099E193E18DE187E181E175E16FE169E163E15DE157E1BF
:40FE800051E14BE145E13FE139E133E12DE127E121E11BE115E10FE109E103E1FDE0F7E0F1E0EBE0E5E0DFE0D9E0D3E0CDE0C7E0C1E0BBE0B5E0AEE0A8E0A2E09CE096E0B9
:40FEC00086E080E07AE074E06EE068E062E05CE056E050E04AE044E03EE038E032E02CE026E020E01AE014E00EE008E002E0002004465BE10220A4F008FB044656E10320C3
:40FF0000A4F003FB044651E10420A4F0FEFA04464CE10520A4F0F9FA044647E10620A4F0F4FA044642E10720A4F0EFFA04463DE10820A4F0EAFA044638E10920A4F0E5FAAE
:40FF4000044633E10A20A4F0E0FA04462EE10B20A4F0DBFA044629E10C20A4F0D6FA044624E10D20A4F0D1FA04461FE10E20A4F0CCFA04461AE10F20A4F0C7FA044615E104
:40FF80001020A4F0C2FA044610E11120A4F0BDFA04460BE11220A4F0B8FA044606E11320A4F0B3FA044601E11420A4F0AEFA0446FCE01520A4F0A9FA0446F7E01620A4F09E
:40FFC000A4FA0446F2E01720A4F09FFA0446EDE0A4F087FA654B0522181A8A4106D207F00FF818B11820A4F090FA0446DEE01920A4F08BFA0446D9E01A20A4F086FA0446F9
:020000040801F1
:40000000D4E01B20A4F081FA0446CFE01C20A4F07CFA0446CAE01D20A4F077FA04460024C4E01E20A4F071FA0446BFE01F20A4F06CFA0446BAE02020A4F067FA0446B5E0E4
:400040002120A4F062FA0446B0E02220A4F05DFA0446ABE02320A4F058FA0446A6E02420A4F053FA0446A1E02520A4F04EFA04469CE02620A4F049FA044697E02720A4F0EA
:4000800044FA044692E02820A4F03FFA04468DE02920A4F03AFA044688E02A20A4F035FA044683E02B20A4F030FA04467EE02C20A4F02BFA044679E02D20A4F026FA044659
:4000C00074E02E20A4F021FA04466FE02F20A4F01CFA04466AE03020A4F017FA044665E03120A4F012FA044660E03220A4F00DFA04465BE03320A4F008FA044656E034205B
:40010000A4F003FA044651E03520A4F0FEF904464CE03620A4F0F9F9044647E03720A4F0F4F9044642E03820A4F0EFF904463DE03920A4F0EAF9044638E03A20A4F0E5F993
:40014000044633E03B20A4F0E0F904462EE03C20A4F0DBF9044629E03D20A4F0D6F9044624E03E20A4F0D1F904461FE0499E5C1F30050010986C02203F20A4F0C6F904460F
:4001800014E04020A4F0C1F904460FE04120A4F0BCF904460AE04220A4F0B7F9044605E04320A4F0B2F9044600E000BF00BF2846FEF7EBF980B154B9FB48007838B9FB48F3
:4001C0000078002808DDF9480078854204D1012003B0BDEC028BF0BD0020F9E710B5044662F040FA04EB8401F14A02EBC1018969884203D90120EF49085505E0ED48005DB0
:40020000012801D1EB49085510BD4FF00008C1464FF0500A0321E84880F8F410E421E748B3F0F7FC002436E10020E5490855E1490855E448005D04EB8401DD4A02EBC101A4
:400240008968087004EB8400114601EBC0008068007800287DDDE21704EBD2625311D74A121D52F823202146E31704EBD3635B11A4EB431C012303FA0CF31A432046E317A3
:4002800004EBD3634FEA631CCC4B1B1D43F82C20E21704EBD2625311C84A203252F82320E31704EBD3635B11A4EB431C012303FA0CF31A43E31704EBD3634FEA631CBF4B43
:4002C000203343F82C2004EB8400B94901EBC000007BE0B1E21704EBD2625311B74A3C3252F823202146E31704EBD3635B11A4EB431C012303FA0CF31A432046E31704EBCF
:40030000D3634FEA631CAD4B3C3343F82C2062F0A9F9AD4941F8240000BFE21704EBD2625311A64A583252F823202146E31704EBD3635B11A4EB431C012303FA0CF39A4377
:400340002046E31704EBD3634FEA631C9B4B583300E002E043F82C2000BF04EB8400944901EBC000407F01281CD1E21704EBD2625311924A743252F823202146E31704EB17
:40038000D3635B11A4EB431C012303FA0CF31A432046E31704EBD3634FEA631C874B743343F82C2004EB8400814901EBC000407F022806D004EB840001EBC000407F032842
:4003C0001CD1E21704EBD26253117C4A903252F823202146E31704EBD3635B11A4EB431C012303FA0CF31A432046E31704EBD3634FEA631C714B903343F82C2004EB840068
:400400006B4901EBC000407F04281CD1E21704EBD2625311694AAC3252F823202146E31704EBD3635B11A4EB431C012303FA0CF31A432046E31704EBD3634FEA631C5F4BA2
:40044000AC3343F82C2004EB8400594901EBC00090F8240001281CD0E21704EBD2625311564AC83252F823202146E31704EBD3635B11A4EB431C012303FA0CF31A4320462A
:40048000E31704EBD3634FEA631C4C4BC83343F82C20601CC4B2D52CFFF6C6AE96F070FC4FF47A60DFF824C100DF4348D0F820110120DFF81CC100DF4FF47A60DFF80CC14D
:4004C00000DF00BF002251460320DFF808C100DF0646022E50D1DFF800C100DF074607F0020078B3002442E0E31704EBD3634FEA631C324B1B1D53F82C304FEAE47C04EB7D
:40050000DC6C4FEA6C1CA4EB4C1B4FF0010C0CFA0BFC03EA0C034FEAE47C04EBDC6C4FEA6C1CA4EB4C1B4FF0010C0CFA0BFC634509D1012004EB84011D4A02EBC101896869
:40054000087008E018E0002004EB8401184A02EBC1018968087004EB8401154A02EBC101896808782146FDF7A9FF601CC4B2D52CBADB5420F8F709F8002458E22046FFF779
:400580002DFE2046FEF708F905462046FDF7E6FFA84240D03DB94FF000090948005D01281CD1814629E037E00E0000100F00001008BF0C0834100020F8FF0020500F002035
:4005C000790E0020FF040068500A0020A99E0C08099F0C08699F0C08B19E0C0804EB8400FE4901EBC000407B10B94FF0010904E0FB48007808B14FF00109B9F1010F0AD170
:400600000020F84908554FF001082046FDF759FF5420F7F7BAFFE3E0E31704EBD3634FEA631CF14B53F82C304FEAE47C04EBDC6C4FEA6C1CA4EB4C1B4FF0010C0CFA0BFC8A
:4006400003EA0C034FEAE47C04EBDC6C4FEA6C1CA4EB4C1B4FF0010C0CFA0BFC6345DAD00020E049085500BFFBF7B4FD58B9DF48FBF7BDFD38B9DD48FCF7A4F918B9DB48C6
:40068000FCF795F9E8B1E21704EBD2625311D64A543252F823202146E31704EBD3635B11A4EB431C012303FA0CF31A432046E31704EBD3634FEA631CCB4B543343F82C20AF
:4006C0001CE0E21704EBD2625311C74A543252F823202146E31704EBD3635B11A4EB431C012303FA0CF39A432046E31704EBD3634FEA631CBC4B543343F82C20E21704EB43
:40070000D2625311B84A52F823202146E31704EBD3635B11A4EB431C012303FA0CF31A432046E31704EBD3634FEA631CAE4B43F82C2061F097FFAE4941F8240000BF00BFBF
:40074000FBF748FD58B9A948FBF751FD38B9A748FCF738F918B9A548FCF729F908B1012000E0002001281DD1E21704EBD26253119D4A543252F823202146E31704EBD36338
:400780005B11A4EB431C012303FA0CF31A432046E31704EBD3634FEA631C934B543343F82C201CE0E21704EBD26253118E4A543252F823202146E31704EBD3635B11A4EB51
:4007C000431C012303FA0CF39A432046E31704EBD3634FEA631C844B543343F82C2000BF002D7CD0E21704EBD26253117E4A1C3252F82320E31704EBD3635B11A4EB431CAF
:40080000012303FA0CF31A40002A54D104EB8400724901EBC0000069F0BBE21704EBD2625311714A1C3252F823202146E31704EBD3635B11A4EB431C012303FA0CF31A438E
:400840002046E31704EBD3634FEA631C664B1C3343F82C204FF0010804EB84005F4901EBC000806800787E280DDA04EB840001EBC00080680078401C04EB8401574A02EBDB
:40088000C1018968087004EB8401544A02EBC10189680878214600E00EE0FDF70FFE04EB84004E4901EBC000007F032860D1012120467BF0DDFC5BE004EB8402474B03EB18
:4008C000C20211694A4A52F8240061F0E8FEE8B3E21704EBD2625311434A1C3200E09DE052F823202146E31704EBD3635B11A4EB431C012303FA0CF31A432046E31704EBF5
:40090000D3634FEA631C384B1C3343F82C204FF0010804EB8400314901EBC000806800787E280DDA04EB840001EBC00080680078401C04EB8401294A02EBC10189680870C8
:4009400004EB8401254A02EBC10100E010E0896808782146FDF7B2FD04EB84001F4901EBC000007F032803D1012120467BF080FC04EB8402194B03EBC202127BD2B3E21790
:4009800004EBD2625311184A383252F82320E31704EBD3635B11A4EB431C012303FA0CF31A403ABBFBF716FC58B91048FBF71FFC38B90E48FCF706F818B90C48FBF7F7FFB0
:4009C00030B304EB8400054901EBC0004069C8B104EB84020B4603EBC2020CE008BF0C08E7220010790E0020540F002078170010500A002019E05169F44A52F8240061F03A
:400A00004EFE90B12046FDF73CFD4FF001080CE02046FDF736FD4FF0010806E0792C04D17BF02CFD08B17BF05BF8601CC4B2D52CFFF6A4ADB8F1010F0BD1E548D0F820112E
:400A40000120DFF890C300DF4FF000085420F7F79CFDE148007848B9FDF7FEFC30B15420F7F793FD0120DC49087006E0DB48006818B961F0F7FDD9490860FDF7C9FC0446D5
:400A800020E5002107E0D64850F8210008B101207047481CC1B20729F5DB0020F8E70020002107E0CE4A383252F8212002B101204A1CD1B20729F5DB704770B5D4201DE07C
:400AC000C41700EBD4646511C54C383454F82540C51700EBD5656D11A0EB45160125B5402C40C51700EBD5656D11A0EB45160125B540AC4200D103E0411EC8B20028DFDC8A
:400B000000BF70BD70B50024FBF764FB58B9B548FBF76DFB38B9B348FBF754FF18B9B148FBF745FF68B3D42428E0E31704EBD3635D11AB4B1C3353F82530E51704EBD565E4
:400B40006D11A4EB45160125B5402B40E51704EBD5656D11A4EB45160125B540AB420BD104EB8403A04D05EBC3035B7B012B03D19E4B1B5D03B903E0601EC4B2002CD4DC57
:400B800000BF204670BD0121984A1154704701460020FF2906DA954A525C0AB1012200E000221046704700210CE08D4850F821008B4A703252F82120104008B101207047AC
:400BC000481CC1B20729F0DB0020F8E700210CE0834850F82100824A8C3252F82120104008B101207047481CC1B20729F0DB0020F8E7002200210CE0794850F82100784B00
:400C0000C43353F82130184008B101207047481CC1B20729F0DB1046F8E7002300210FE06F48C43050F8212009B922F002026C4850F82100104008B101207047481CC1B21D
:400C40000729EDDB1846F8E700B5002304E01846FFF799FF581CC3B2D52BF8DB00BD10B586B0044662A30FCBCDE90423CDE902013CB34AF071FB4EF0FAFE002201216048AD
:400C800099F085F80D2202A9FF204AF0B5FA5D4890F85308032810D15A4890F8120801280BD001A9584856F0CDF928B1019800680121026B0198904700BF0120534908704D
:400CC0001AE0504890F85308032810D14D4890F8120801280BD001A94B4856F0B3F928B1019800680021026B0198904700BF0020464908704AF0AAFA06B010BD43480078E7
:400D00007047014601EB8100374A52F830007047014601EB8100344A02EBC000007970473B490870704710B504463A480470E320F7F72BFC10BD10B5044600212046FDF760
:400D40004FFC00212046FDF739FC00212046FDF724FC10BD2DE9F0472F480078002832D100F0D4F900282ED02C4890F82180A8F108044FF00009012C00DA0C34002514E0DC
:400D8000274810F8150000F00F06A64200DA0C360027301B082800DD012727B12846FFF7CAFF4FF00109681CC5B2FF2DE8DBB9F1000F04D0012095F062FE95F0E1FF0120A6
:400DC0001549087000BFBDE8F0870000500A0020F8FF0020099F0C081400001010000010540F00207817001008BF0C08790E002001020A0B111214181921242A2B000000F3
:400E0000BCDD0010602A0020986C02200C0000100F0000100E00001015000010A01E0020C435002070B504460025FE4890F8F0050A2818D2DFE800F017050C071712171714
:400E4000060D00BF00BF204630F073FD05460CE000BF204633F0E4FF054606E020462BF0C3FD054601E0002070BD00BF2846FBE710B5ED48007800F0010080B10120FFF7E4
:400E8000D1FF01280AD1E848006840F00800E64908600846006820F0010008600BE1E248007800F0020080B10220FFF7BBFF0128F4D1DD48006840F00800DB4908600846B8
:400EC000006820F002000860F5E0D748007800F0400080B14020FFF7A5FF0128DED1D248006840F00800D04908600846006820F040000860DFE0CC48007800F0800080B1DC
:400F00008020FFF78FFF0128C8D1C748006840F00800C54908600846006820F080000860C9E0C148007800F0040080B10420FFF779FF0128B2D1BC48006840F00800BA49C4
:400F400008600846006820F004000860B3E0B648007800F0080058B10820FFF763FF01289CD1B148006820F00800AF490860A2E0AD48006800F4003060B14FF40030FFF761
:400F800051FF01288AD1A848006820F40030A649086090E0A448007800F0100058B11020FFF740FF012805D19F48006820F010009D4908607FE09C48007800F0200008B3E6
:400FC0002020FFF72FFF07220421984819F05CFD012810D09548006940F04000934908619348816C4FF48060DFF848C200DF07218E4819F047FE8C48006820F020008A49C3
:40100000086058E08848008800F4807060B14FF48070FFF707FF01284DD18348006820F480708149086046E07F48008800F4004060B14FF40040FFF7F5FE01283BD17A48C7
:40104000006820F400407849086034E07648008800F4007060B14FF40070FFF7E3FE012829D17148006820F400706F49086022E06D48008800F4804060B14FF48040FFF74D
:40108000D1FE012817D16848006820F480406649086010E06448006800F4803058B14FF48030FFF7BFFE012805D15F48006820F480305D49086010BD5F48007B052801D128
:4010C000012070470020FCE710B55C49D1F8FC0061F006FB10BD00B5584890F8FA10FFF7EBFF00B90021084600BD00B5FFF7F3FF022801D1012000BD0020FCE700B5FFF7F6
:40110000EAFF012800D100BD0020FCE710B5FFF7F5FF10B9FFF7E9FF30B1FFF7D5FFB0F57A7F01D9012400E00024204610BD434890F80601012804D13F48007808B901203E
:4011400070470020FCE710B53D49C86F61F0C8FAB0F5FA7F2BD33A4890F8900038B30020374981F89000354981F806019FED350A084680ED170A0021314880F84A109FED39
:40118000310A80ED130A00202C4981F80201A1F8F8009FED2D0A2A4880ED140A002081F8FA0081F8FB004FF48B70F7F7EEF92749C86A61F095FA43F69821884207D323486B
:4011C00090F8380018B10020204981F838002049D1F8D40061F084FA42F21071884207D31B4890F8E00018B10020194981F8E0001849D1F8D40461F073FA43F69821884213
:4012000007D3144890F8E00418B10020114981F8E0041149886C61F063FAB0F57A6F24D30D481BE0602A00208800001090210020F8FF0020099F0C0870210020582000206C
:40124000681600200000000000007F43A01E002044180020801900202819002090F8540018B10020FE4981F85400FE49C86A61F037FA44F62061884207D3FA4890F8380065
:4012800018B10020F74981F83800F74890F8060138B921F057FE20B11FED160A21F0CCFD08E0F14890F8060120B920F013F908B120F00EFAFFF73BFF60B1EC4890ED140AD2
:4012C0005FED1F0AB4EE600AF1EE10FA12D1FFF71DFF78B9E6A20321E4486630B1F052FFE3A20321E1485630B1F04CFF0021DF48A0F8541010BD10B561F0B4F90446DB4879
:40130000C467C06F6438D94988670846C06F896F401A00EE100AB8EE400AD44880ED220A0120D24981F89000D248C462C06A6438D04988620846C06A896A401A00EE100A0F
:40134000B8EE400ACB4880ED0C0A0120C94981F83800002081F83900C748C0F8D440D0F8D4006438C449C1F8D0000846D0F8D400D1F8D010401A00EE100AB8EE400ABE489D
:4013800080ED360A0120BC4981F8E000BB48C0F8D444D0F8D4046438B849C1F8D0040846D0F8D404D1F8D014401A00EE100AB8EE400AB34880ED360A0120B04981F8E00458
:4013C000A7488464806C6438A54948640846806C496C401A00EE100AB8EE400AA04880ED130A01209E4981F854009E48C462C06A64389C4988620846C06A896A401A00EE18
:40140000100AB8EE400A974880ED0C0A0120954981F8380010BD01B500BF0122694699480EF02DF820B99DF80000974981F8300300BF08BD00218D4880F84A101FED7F0A9D
:4014400080ED130A9FED910B80ED0C0B9FED8F0B80ED0E0B80F849101FED850A80ED140A704731B5002400BF042269468948006800F5FA700EF003F818B983480099C0F8C0
:40148000F41500BF204638BD10B501208249087382A1874898F05CFC10BD10B561F0E2F87249C86761F0DEF87249C8626F4890ED140A5FED9B0AB4EE600AF1EE10FA07D049
:4014C0001FED9F0A80ED140A40F2E7307CF0CBF96D4890F8F0050B287ED2DFE800F07D068D08B15BF3F20788F10000BF00BF6A48407B20B9FFF79EFF00206E4988800822DE
:4015000010216548103019F0BFFA012810D05E4B93F8F825604B597B5B4BD3F8F4052FF044FF5D49487308215B48103019F0AAFB6048808801282CDD5EF061F918B95E480A
:401540000078012803D05C480078032801D1012000E00020012817D14B4890F8300398B95648007880B90020524988800120FFF752FF4F4898F092FC58B90120FFF74BFF74
:4015800002204C49888004E0FFF77EFF002049498880EEE04048407B20B9FFF74BFF002044498880082210213B48103019F06CFA012810D0344B93F8F825374B597B324BEC
:4015C000D3F8F4052BF0D6F83349487308213248103019F057FB00E0C7E036488088052804DDFFF751FF002032498880C1E04FF46140FFF736FF00BF2748407B30B9FFF74D
:4016000019FF32F077FC00202A498880082210212148103019F038FA012810D01A4B93F8F8251D4B597B184BD3F8F40533F0A7FA1949487308211848103019F023FB98E061
:401640001548407B18B9FFF7F5FE2DF045F8082210211148103019F017FA012843D032E028190020641E002058200020681600202D2D2D00A01E002044180020801900200F
:40168000801D002030030068602A0020000000000000000020010010702100204750532052656365697665722052657365740000BCDD001060210020300500108E000010B7
:4016C00012E031E050E05EF072FD0446002221464FF4E1302DF01CF8F84948730821F748103019F0CFFA44E0F448407B18B9FFF7A1FE2CF0F1FF08221021F048103019F0C3
:40170000C3F901280FD05EF052FD0446002221464FF461402CF0FCFFE84948730821E748103019F0AFFA24E0E448407B18B9FFF781FE2CF0D1FF08221021E048103019F05B
:40174000A3F901280FD05EF06BFD0446002221464FF4E1302CF0DCFFD84948730821D748103019F08FFA04E000BF0820D349487300BF00BF10BD10B5D048007B06286CD24A
:40178000DFE800F0031F2C414F6A5EF038F818B9CB480078012803D0C948007803280CD1C84800785EF08CFC38B10320C349087360F058FFC449086002E00120BF49087330
:4017C0004BE00021C14800785EF036F90220BB49087360F047FFBC4908603EE0BA48006860F07EFF41F2883188420BD30121B74800785EF021F90320B049087360F032FFF9
:40180000B149086029E0B048006860F069FF42F21071884204D30420A8490873002048731BE0FFF73AFEA548407B082813D10020FFF7F1FDFFF75FFD0520A049087301207F
:401840004870A348D0F818130420DFF888C200DF0120A149087000E000BF00BF10BD10B5082210219548103019F00EF901280AD00020924948730420087308218F4810301B
:4018800019F000FA17E007220421944819F0FCF8012810D09148006940F020008F4908618B48816C4FF48060DFF828C200DF07218A4819F0E7F910BD10B50024884890F8B7
:4018C000F0050B2814D2DFE800F013060C080F121011070D0E0000BF00BF32F0D3FA044608E000BF00BF00BF00BF00BF00BF00BF002400BF00BF204610BD10B5002079493E
:4019000008702DF0CFFB10B92DF0A5FB20B132F0BFFA7449087003E02BF013FB714908707048007810BD10B500246F48007830B901206D49087060F095FE6C4908606B48A3
:40194000006860F0CDFE41F28831884203D90124002065490870204610BD654909680143634A1160704710B55D4991F8F0150B2916D2DFE801F015060B08110F1213070C29
:401980000D0000BF00BF32F06FFA0BE000BF00BF002007E0002005E000BF00BF002001E0002000BF00BF10BD10B54D4991F8F0150B2916D2DFE801F015060B08110F121382
:4019C000070C0D0000BF00BF2DF0F9FB0BE000BF00BF002007E0002005E000BF00BF002001E0002000BF00BF10BD10B53C4991F8F0150B2916D2DFE801F015060B08110FDF
:401A00001213070C0D0000BF00BF2DF064FB0BE000BF00BF012007E0002005E000BF00BF012001E0002000BF00BF10BD00202C4991F8F015042900D10120704710B52849D7
:401A400091F8F0150B2916D2DFE801F015060B080F131011070C0D0000BF00BF2DF009FB0BE000BF00BF002007E000BF00BF012003E0002001E0002000BF00BF10BD10B5B1
:401A8000174991F8F0150B2934D2DFE801F033060B080F131011070C0D0000BF00BF2DF00EFB29E000BF00BF002025E000BF00BF012021E02AF0ECFD1EE0000070210020F5
:401AC000300500104A050010900000106C050010F8FF0020099F0C088E00001090210020602A00208C000010990000109C00001088000010002000BF00BF10BD10B5FE4935
:401B000091F8F0150B2917D2DFE801F016060B080F131011070C0D0000BF00BF2DF05BFB0CE000BF00BF002008E000BF00BF012004E02AF0B8FD01E0002000BF00BF10BDAF
:401B40002DE9F04106460F46062F7DD2DFE807F003115F311F4816B90024002508E0022E01D0012E02D10124032501E0002402259CE016B90024002508E0022E01D0092E00
:401B800002D10124032501E0002402258EE0FFF7B5FF10B9002401250AE016B90024002506E0022E02D10124032501E0002402257CE0FFF764FF10B9002401250FE0022E63
:401BC00002D1022406250AE016B90024002506E0052E02D10124032501E00024022565E0FFF72CFF10B9002401250FE016B9002400250BE0022E02D10224062506E0052E82
:401C000002D10124032501E0002402254EE0FFF70DFF20B316B90024002543E0042E02D1032501243EE0012E03D1B34890F8DB0578B1022E04D1B04890F8DB05012808D0B5
:401C4000052E09D1AC4800E02DE090F8DB05022802D10224062525E00024022522E0FFF7C4FE10B9002401251CE016B90024002518E0022E02D10224062513E0042E0AD143
:401C8000FFF792FE20B1FFF76EFE08B1052500E00325012406E0052E02D10224042501E00024022502E00024002500BF00BF934890F8FA00A04203D19148007801280AD1E3
:401CC00060F0D0FC8D49C1F8FC00084680F8FA4000208B490870894880F8FB50BDE8F0810020854991F8F015052900D1012070470020814991F8F015012909D07E4991F809
:401D0000F015082904D07C4991F8F015032900D10120704710B5794890ED0E1BB0EE410AF0EE610A9FED771B53EC112B51EC100BB9F062FD2FD3714890ED0E1BB0EE410AD0
:401D4000F0EE610A9FED711B53EC112B51EC100BB9F070FB1FD3694890ED0C1BB0EE410AF0EE610A9FED6B1B53EC112B51EC100BB9F042FD0FD3614890ED0C1BB0EE410ABD
:401D8000F0EE610A9FED651B53EC112B51EC100BB9F050FB07D20020584981F802010120604908703BE0FFF7A3FF60B15E4890F82C00524981F802015B4890F82C105B4870
:401DC00080F8481028E0FFF78BFFF8B14A4890F8F805032813D1554890F84800042802D005280AD104E00521504880F8481005E001214E4880F8481000E000BF00BF4B4879
:401E000090F848003D4981F8020105E0474890F848003A4981F8020100204249087010BD10B5364890F805014149097888420FD0324890F805013E490870032045F092FD2A
:401E400040F275207BF00FFD40F252207BF00BFD10BD10B52DED028B274890F84044102C28D2DFE804F02720212217161508252727272324272607F062FEF0EE408A07F070
:401E80004EFEF0EE000A80EE201A38EEC18A17E000BF00BF07F053FEF0EE408A07F03FFE38EEC08A0CE000BF00BF00BF00BF00BF00BF00BF1F481FF04CF9B0EE408A00BFC5
:401EC00000BFB0EE480ABDEC028B10BD10B52DED068BF0EE408AF0EE609AB0EE41AA9FED160AF4EEC08AF1EE10FA27D2B0EE680ABDEC068B10BD0000602A002058200020A4
:401F00008F000010000000000080664000000000008066C0000000000080564000000000008056C070210020DC1E00206816002098000010584900102FDDE43E29EE8A0AEF
:401F4000B0EE409A29EE090AB0EE409A28EEA88AB4EEC89AF1EE10FA06D278EE49AAB0EE6A0AB6F0FAFF01E09FEDFD0AB0EE408AB0EE480ABDEC068B10BD70B52DED0A8B89
:401F800082B005460E46144695ED140AF0EE40BAB0EE6B0AB4F02EFBB0EE408AB0EE6B0AB4F06FFBF0EE408A1EF019FAB0EE40CAB0EE4C0AB4F065FBB0EE409AB0EE4C0A40
:401FC000B4F018FBF0EE409A9FEDE50AB0EE40AAE44890F85604912809D0E24890F85604922804D0DF4890F8560471280BD19FEDDC0AB0EE409A9FEDDA0AF0EE409A9FED19
:40200000D80AB0EE40AA07F0EAFDF1EE40AA07F0ADFDB1EE40BA28EE290A68EE8A0A00EE890A20EE2A0A84ED010A28EE090A68EE8A0A00EEE90AD4ED010A40EE0B0AC4ED2F
:40204000010AB1EE680A20EE290A68EE0A0A00EE890A20EE2A0A84ED000A28EE890A68EE0A0A00EEA90AD4ED000A40EE4B0AC4ED000A142306F1200205F1B001684624F0E5
:40208000C1FB9DED000AD4ED000A30EE200A8DED000A9DED010AD4ED010A30EE200A8DED010A0922102105F1A00018F0EDFC01280BD0142305F11002AB49684624F032FC01
:4020C000092105F1A00018F0DDFD02B0BDEC0A8B70BD31B5002400BF01226946A348006800F502700DF0CBF928B9BDF80000C1B29C4880F8081600BF7A20F6F746FA20469C
:4021000038BD31B5002400BF012269469748006800F206200DF0B3F920B99DF80010914880F8061600BF7A20F6F72FFA204638BD8C4991F8F815062911D2DFE801F00F0509
:40214000030C080B7F200DE040F6EC100AE040F6EC1007E000BF40F2FA2003E000BF40F6EC1000BF00BF704710B501247D4890F8F0050B2815D2DFE800F014090E0B11061E
:4021800012130A0F10002AF0BCFA0CE000BF00BF2EF011F807E000BF00BF00BF00BF00BF00BF012400BF00BF204610BD10B52DED020B0024FFF7BCFF00EE100AB8EE400A80
:4021C000DDED000AB4EEE00AF1EE10FA08D2FFF7AFFF00EE100AB8EE400A8DED000A0224634890ED020ADDED000AB4EE600AF1EE10FA14D000BF042269465C48006800F500
:4022000081600DF03CF920B99DED000A584880ED020A00BF6C20F6F7B8F9FFF7A5FF20461CBD31B52DED028B00244E4890F8F8059DF8081088421CD000BF012202A94B48F4
:40224000006800F5FC700DF01AF920B99DF80810444880F8F81500BFFFF76AFF00EE100AB8EE400AB0EE408AFFF7A0FF4D20F6F78CF92046BDEC028B38BD31B5002400BFA2
:40228000042269463948006800F500700DF0F7F818B934480099C0F8001600BFCE20F6F774F93448D0F818130420DFF8CCC000DF204638BD31B5002400BF022269462B4815
:4022C000006800F501700DF0DAF820B9BDF800102448A0F8041600BF204638BD31B5002400BF012269462148006800F5FE700DF0C6F820B99DF800101A4880F8FC1500BFB9
:402300004E20F6F742F9204638BD31B5002400BF022269461548006800F5FD700DF0AFF820B9BDF800100F48A0F8FA1500BF204638BD31B5002400BF012269460B48006839
:4023400000F211400DF09BF820B99DF80010054880F8111800BF7C20F6F717F9204638BD00000000602A0020082100202001001060320020F8FF0020099F0C0810B50120DC
:40238000FFF7BFFE0020FFF7A4FE0020FFF7D1FF0420FFF7A3FF4FF6FE70FFF7B6FF0420FFF79CFF4FF6FE70FFF784FF0120FFF738FF012010BD10B5FB4890F8F0050B28DD
:4023C00017D2DFE800F016060C0816121616070D0E0000BF00BF31F0A7FC04460DE000BF00BF33F00FFD044607E02AF032FC044603E0FFF7C3FF044600BF00BF4D20F6F7F1
:40240000C4F87A20F6F7C1F87C20F6F7BEF84E20F6F7BBF84F20F6F7B8F807220421E34818F032FB012810D0E048006940F02000DE490861DE48816C4FF48060DFF874C3DB
:4024400000DF0721D94818F01DFC204610BD73B50C46002500BF01226946D748006800F5F8700DF00CF820B99DF80010CE4880F8F01500BFC120F6F788F88120F6F785F8A2
:402480003CB1FFF798FFFEF7FFFF4FF4E130FFF7F4FE28467CBD2DED068B86B04FF0C8084FF0000940F25451C448B1F0B2FB9821C348B1F0AEFB4FF4A271C248B1F0A9FBB0
:4024C000E421C148B1F0A5FB5821C048B1F0A1FB40F2E441BE48B1F09CFB3C21BD48B1F098FB3C21BC48B1F094FB3821BB48B1F090FB9821BA48B1F08CFB4FF48471B9486F
:40250000B1F087FB2021B848B1F083FB1421A748B1F07FFB6821B548B1F07BFB3821B448B1F077FBB3480021016041608160C1600020AD49087360F095F8AA49C1F89C00FE
:40254000002081F807019E4981F89100A24981F83A00A34981F891001421A248B03024F00DF801F0CFFB904890F85604912809D08D4890F85604922804D08B4890F856041C
:40258000712808D100210620FFF761FF4FF4E130FFF773FE48E05DF032F940B100210420FFF755FF4FF4E130FFF767FE3CE07E4890F85604702804D07B4890F856049328F2
:4025C00008D100210720FFF742FF4FF4E130FFF754FE29E05DF013F918B987480078012803D085480078032808D100210120FFF72EFF4FF4E130FFF740FE15E06A48D0F8CC
:402600000006B0F5966F05D36748D0F80006B0F5E13F04D94FF4E130FFF72FFE04E06249D1F80006FFF729FE4FF4E130FEF719FF5D4890F8F805072808DB0120FFF7F1FD5F
:402640000120FFF75EFD0020FFF743FD06F02FFC0321574880F84C1000BF0022414640F6FC70DFF898C100DF0546012D7ED0022D7CD1DFF88CC100DF044604F00400002811
:4026800075D0FEF719FD0028FAD00B2210214C4818F0FAF901286BD06822494910315348B1F05BFA0B21464818F0ECFA4D4B4F4E203647CE47C34D4890ED0C0A494880ED21
:4026C000180A5FF0CFFF3E49C867012081F89000084690F89100052806DA084690F89100401C81F8910014E0354A916FD06F60F006F8444908603248C06F31498867022150
:402700002F4888303F4A92ED000AB8EE400A23F048FA2B48D0F880003A490968884204D9384800682649C1F880002548D0F8840034490968884204D2324800682049C1F8E2
:402740008400FEF7DBFC68BB264890F8B00048B31423264A20322349B03104A824F052F82848016804A810F040FB02E0A7E3F4E124E114231D4A20321A49B03104A824F0FB
:40278000D1F810F07BFC48B110F081FC064602F077FA10F07CFC064602F018F8002010F070FC44E030E00000602A002090210020F8FF0020099F0C0820010010101100206E
:4027C0006816002000170020441800202819002080190020641E0020A01E0020DC1E0020181F00205820002070210020A8210020102200206021002030050010699F0C08F7
:40280000B19E0C081800001010F03EFC78B910F040FC8DED040ACDED050A04A802F030FA04A801F0D3FF012010F02BFC00BFFE4890F8B000E8B1FC4890F80401C8B11DF069
:4028400006FEB0B104AAF949F748FFF796FBF74890ED0C0AF44880ED190AB9F1000F07D104A802F00DFA04A801F0B0FF4FF0010920E0ED4890F8B00030B91422EB492031C3
:40288000E948B03023F09DFEE748E84E20364ECE10304EC0E54890ED0C0AE34880ED190AE34890F8900018B10120DF4981F806014FF00009DC4890F8B00001287ED1142292
:4028C000D949B031A1F1A00024F008F88246BAF1000F25D11423D44A103202F1A001684623F090FF9DED010AFFEE000A20EE200A8DED010A9DED000AFFEE000A20EE200A90
:402900008DED000A1422C849103101F1A00023F058FE684602F0B4F9684601F057FF00BFC24890ED040ADFEDC30A20EE200ABDEEC00AC14880ED000A0068C0490968401AF8
:40294000BF490860BC480068BC490860BC480068002807DABA4800684EF660210844B849086006E0B6480068142802DA1420B4490860AE4890F838601423AB4A02F1B001D2
:4029800004A823F03FFFAE483146026804A802F098F81423A44A103202F1A00102A823F031FFA7483146026802A801F0DBFF07F0BCFC07469C4890ED160A00E0C1E0B0EE4C
:4029C000401A3B469F4802689D4801683046DDED030A9DED020A01F026FC99480068DDED030A9DED020A01F091F901F012FFF0EE408A9FED950AB0EE408AFFF72AFAB0EE41
:402A0000409A1DF0DCFCF0EE409A02F025F9B0EE40AAB0EE491AF0EE690AFFF757FAB0EE408A20F08FFA18B1B0EE480A20F004FA7D4890F8040120B901F030FF08B1012001
:402A400000E00020834609220C217748A03018F01BF8012865D001F014FF80F00100724981F8030101F01AFF6F4981F8040101F074FA6D4981F805010846C0ED1A8A80EDA0
:402A80001B8A02F00FF9F7EE000A80EE801AB6EE000A31EE000ABCEEC00A10EE100A87B20A2F00DD0A27C7F10A015F484830B0EE480A23F076F8C7F11E015B484030B0EEC2
:402AC000480A23F06EF8FFF7ABF902F0CDF8564880ED1D0A02F0CCF8534880ED1E0A5CF08EFE18B959480078012803D057480078032805D102F0B4F84B4880ED1C0A02E026
:402B0000494880ED1C8ABBF1000F04D04648C0ED168A80ED178A09214348A03018F0B2F800BF434890F89000012809D13E4981F806014748816F4FF48050DFF818C100DFB5
:402B400000BF1EF0C5FDFFF7E5F8434A92F8F815354A92F80201FEF7F3FF04F01000F8B1FEF7AAFAE0B15FF07DFD3C49C862012081F83800084690F8390028B9012081F831
:402B800039000004FEF7E9FE344890F83A00052807DA324890F83A00401C304981F83A0014E02E4A916AD06A5FF0A9FD2549086001212A483030234A92ED000AB8EE400AA6
:402BC00022F0EFFF2548C06A2449886204F0200018B3FEF771FA00B35FF044FD2049C1F8D400012081F8E0000A46D2F8D010D2F8D4005FF084FD1349086001211848D8303F
:402C0000104A92ED000AB8EE400A22F0CAFF1448D0F8D4001249C1F8D00004F48070E8B3FEF74AFAD0B31DE058200020A82100206816002000007A44200000101C00001095
:402C400024000010180000100000000030050010F8FF0020099F0C08602A0020A01E0020441800205FF0FEFCF949C1F83401012081F840010A46D2F83011D2F834015FF0DF
:402C80003EFDF44908600121F348F24A92ED000AB8EE400A22F085FFED4800E008E0D0F83401EB49C1F830014FF48B70F5F76DFC04F0400010B3FEF7FFF9F8B15FF0D2FC37
:402CC000E649C1F8D404012081F8E0040A46D2F8D014D2F8D4045FF012FDDE4908600121DF48DC4A92ED000AB8EE400A22F059FFDA48D0F8D404D949C1F8D00404F008004A
:402D0000F0B1FEF7D9F9D8B15FF0ACFCD549C862012081F838000A46916AD06A5FF0EFFCCC4908600121CF483030CA4A92ED000AB8EE400A22F035FFCA48C06AC9498862B1
:402D400004F40070D0B3FEF7B7F9B8B35FF08AFCC5498864012081F854000A46516C906C5FF0CDFCBB4908600121BF484C30B94A92ED000AB8EE400A22F013FFBA48806CDB
:402D8000B9494864084690ED0D0AB84880ED1F0A084690ED0E0AB54880ED200A084690ED0F0AB24880ED210A084690ED100ABCEEC00A10EE100AAD49A1F8F80004F4806030
:402DC00000287CD007220421A94817F05DFE0128F7D0A748007C00F0020070B15120F5F7D4FB7220F5F7D1FB8120F5F7CEFBA048006920F002009E4908619D48007C00F080
:402E0000080040B18420F5F7C0FB9948006920F00800974908619648007C00F00400F8B1944890F8F80504280ED0924890F8F805032809D08F4890F8F805052804D08D48AC
:402E400090F8F805022805D1B620F5F79EFB1F2044F088FD8648006920F00400844908618348007C00F0100040B15020F5F78DFB7F48006920F010007D4908617C48007C1E
:402E800000F0800040B15020F5F77FFB7848006920F08000764908617548007C00F0200038B1FEF7DCFC7248006920F02000704908616F48007C00F04000E8B100E05AE070
:402EC000FEF731FDC0B1FEF718FD02280ED1FEF7F3FC10B1FEF7C3FC08E06748006840F40040654908608120F5F74FFB6048006920F040005E4908615D48007C00F00100EF
:402F0000A8B3FEF7D9F890B30A2210215B4817F0BBFD01282BD02022584910315848B0F01CFE0A21554817F0ADFE544890ED070A4E4880ED1F0A514890ED080A4B4880EDD4
:402F4000200A4E4890ED090A484880ED210A4B4890ED0A0ABCEEC00A10EE100A4349A1F8F8004348006920F001004149086107213F4817F087FEFEF7FEFBFEF7E4F8FEF725
:402F80009BF808B1FDF774FF11F0BFFC022808D13C48007828B99B20F5F7F7FA0120394908703249D1F89C0042F210715FF077FB18B100202D4981F807015020F5F7E5FA9E
:402FC000FFF74BBB294890ED170A70472748D0ED170AB0EE600A90F80501012805D1FFEE000A60EE200AB0EE600A70471F48D0ED100AB0EE600A90F80501012805D1FFEE3F
:40300000000A60EE200AB0EE600A7047174890ED100A70471548D0ED120AB0EE600A90F80501012805D1FFEE000A60EE200AB0EE600A70470D4890ED120A704700B50B48FC
:4030400090F8FB10FEF738F800B90021084600BD00170020180000103818002080190020581E0020641E0020281900205820002090210020602A002088000010DC1E0020CD
:40308000102200208D00001000B5FEF724F808B9012000BD0020FCE7FE4890F802017047FD4890F89100052801DB012070470020FCE7FA4890F83A00052801DB012070470A
:4030C0000020FCE7F648007B012800D170470020FCE7F348007B032801D1012070470020FCE7EF48407B082801D1012070470020FCE710B52DED028BEA4890F84044102C1D
:4031000028D2DFE804F02720212217161508252727272324272606F012FDF0EE408A06F0FEFCF0EE000A80EE201A38EEC18A16E000BF00BF06F003FDF0EE408A06F0EFFC47
:4031400038EEC08A0BE000BF00BF00BF00BF00BF00BF00BF06F0F3FCB0EE408A00BF00BFB0EE480ABDEC028B10BD31B5002400BF01226946CC48006800F207200CF07FF959
:4031800020B99DF80010C74880F8071600BF7A20F5F7FBF9204638BD31B5002400BF01226946C148006800F2FD100CF068F920B99DF80010BB4880F8FD1500BF4F20F5F7CC
:4031C000E4F9204638BD31B50024B64890F8DB059DF80010884213D000BF01226946B248006800F2DB100CF04AF920B99DF80010AC4880F8DB1500BF4FF48870F5F7C5F948
:40320000204638BD31B50024A64890F8DC059DF8001088420FD000BF01226946A248006800F5EE700CF02BF920B99DF800109D4880F8DC1500BFFC20F5F7A7F9204638BDA0
:4032400010B50124974890F8F0050B2813D2DFE800F012060B080E0F1011070C0D0000BF00BF30F013FB08E000BF00BF00BF00BF00BF00BF00BF002400BF00BF204610BD0E
:4032800038B504462046B0F06BFB052832D3052286A12046B0F014FB28B9864896F087FE10F052FC26E0052283A12046B0F008FB00BBFFF7C5FF00BF3C2281A181480CF0FB
:4032C000DEF820B977487EA1097880F8C01100BF8120F5F75AF9FF2003460322012100904D20F8F78DFB4FF48070FEF736FB8120F5F74BF938BD10B56A4890F8F005012879
:4033000006D0032806D005285CD0082870D100E000BF00BF6C48FFF7B3FF40216B48B0F078FC062268496948B0F09AFC2C20674988710622644909316448C01DB0F090FC91
:403340002C206249487306225F4912315F480E30B0F086FC2C205D49087506225A491B315A481530B0F07CFC2C205849C87606225549243155481C30B0F072FC2C205349D7
:4033800081F8220050482D30B0F0EAFAC4B2621C4D492D314D482330B0F062FC4A4890F8380070B14948B0F0DBFAC4B22C2047490855601CC4B20819072243493831B0F032
:4033C0004FFC50E029F09EFD98B129F0B7FD80B940213E48B0F01DFC3B484130B0F0C0FAC4B2621C384941313848B0F039FC38E038E040213548B0F00CFC0822324933484F
:40340000B0F02EFC08223049093130480830B0F027FC08222C4912312C481030B0F020FC082229491B3129481830B0F019FC08222549243125482030B0F012FC08222249DD
:403440002D3122482830B0F00BFC1F483830B0F087FAC4B2621C1C4938311C483030B0F0FFFB00E000BF00BF2020FEF776FA10BD10B504462046FFF703FF2046B0F070FAC8
:40348000402803D821461148B0F046FA2020FEF764FA10BD5820002068160020A01E002070210020602A0020200100104345535452000000BCDD001043454750530000008D
:4034C00000000000C0010068F01F0020B01F002031B500249DF80000032802DD032000900224FE4890F860089DF80010884212D000BF01226946FA48006800F58C600BF065
:40350000BEFF20B99DF80010F44880F8601800BFDC20F5F73AF8204638BDF248704770B50546EE4890F8F005012804D0032804D0082807D100E000BF00BF284630F007FBEA
:40354000044602E0AFF2880070BD00BF2046FBE770B50546E14890F8F0050B2821D2DFE800F020060D0819141A1B070E0F0000BF00BF284630F079FB044615E000BF00BFD1
:40358000284632F099FB04460EE0284629F01EFB044609E000BF00BF284627F079FC044602E0AFF2E40070BD00BF2046FBE710B5CA4991F8F0150B2916D2DFE801F015062A
:4035C0000B08110F1213070C0D0000BF00BF2BF0DCFD0BE000BF00BF002007E0002005E000BF00BF002001E0002000BF00BF10BD10B5BA4890F8F0050B2813D2DFE800F06F
:4036000012060C080F0B1011070D0E0000BF00BF30F031FC09E000BF00BF00BF00BF00BF00BF00BF9FEDB00A00BF00BF10BD10B50024AA4890F8F0050B2815D2DFE800F05A
:4036400014060C0814101414070D0E0000BF00BF30F0FBFB044609E000BF00BF002405E029F032F8044601E0002400BF00BF204610BD10B5994991F8F0150B2912D2DFE809
:4036800001F011060B08110F1111070C0D0000BF00BF30F0C6FB07E000BF00BF002003E0002001E0002000BF00BF10BD10B58B4991F8F0150B2913D2DFE801F012060B0837
:4036C000120F1212070C0D0000BF00BF30F095FB08E000BF00BF002004E028F001FF01E0002000BF00BF10BD2DE9F04781460E4614464D460027B84610E04FF02C0A5146F3
:403700002846B0F0C1F807461FB9B04500DA002506E0B04500DA7D1C08F10108B045ECDD45B117B1781B207006E02846B0F018F9207001E0002020702078102801DC20784F
:4037400010B90025002020702846BDE8F08700B5FDF7EDFC18B16548B0F8F80010B94FF6FF7102E06148B0F8F810084600BD5B4890F81F08704701B500BF012269465848C5
:40378000006800F21F400BF07AFE20B99DF80010524880F81F1800BF9C20F4F7F6FE002008BD4E48B0F8AA0500EE100AF8EE400A9FED4F1A80EE810A70474C4890F80701E9
:4037C000704701B500BF012269464A480BF057FE20B99DF80000414981F8000100BF9B20F4F7D3FE08BD01463C20052911D2DFE801F00305070A0D0000200AE03C2008E09C
:403800004FF4967005E04FF4167002E04FF4B46000BF00BF7047384840687047364948607047364800787047344908707047324890ED020A7047304880ED020A70472E4835
:40384000407B70472C48007B7047F0B52DED0C8B85B0B0EE408AF0EE608A01279FED280B53EC102B51EC180BB7F0E4FD0AD2BF1EB0EE480AF0EE680AB3F0EEFEB0EE408A3C
:40388000F0EE608AB0EE480AF0EE680AB3F0F0FEB0EE409AF0EE609A51EC190BB7F0FCFC44B22046B7F055FD53EC182BB7F0DAFF9FED150B53EC102BB7F0F8FD41EC1A0BB4
:4038C000B0EE4A0AF0EE6A0AB3F0D2FEB0EE409AF0EE609A51EC190B1AE00000602A002020010010B01F0020000000005820002000007A44000100687021002028000010F4
:4039000000000000000000000000000000004E40B7F0C2FC45B2C5EB05118800B7F019FD41EC1A0B2046B7F014FD53EC182BB7F099FF9FEDD40B53EC102BB7F0B7FD53ECE2
:403940001A2BB8F067F8B7F025FA06463046B8F04BF941EC190B8DED029B04FB07F3CBA20F21CD480095AFF00DFCCB4805B0BDEC0C8BF0BD10B5044600BF0B222146C74811
:403980000BF07DFD40B9C648216801606168416021890181A17A817200BF10BD10B5044600BF0B222146BD480B380BF068FD48B9BB480B38216801606168416021890181A0
:4039C000A17A817200BF10BD10B5B64991F8F0150B2916D2DFE801F015060B080F131011070C0D0000BF00BF30F049FA0BE000BF00BF002007E000BF00BF002003E0002084
:403A000001E0002000BF00BF10BD10B5A54991F8F0150B2916D2DFE801F015060B080F131011070C0D0000BF00BF30F028FA0BE000BF00BF002007E000BF00BF002003E0E3
:403A4000002001E0002000BF00BF10BD0020954991F8F015022909D0924991F8F015092904D0904991F8F0150A2900D10120704710B50446A06860605EF0F4FDA060D4E9C5
:403A80000110401A206010BD10B5874B87A20C218748AFF077FB864810BD10B58248663890ED140ABCEEC00A10EE100A80B2FF2805D1804A7DA18048AFF04EFB0DE07A481C
:403AC000663890ED140ABCEEC00A10EE100A83B27AA204217848AFF055FB774810BD00B5FEF706F900BD10B52BF0DCFA10B9FEF7F7F808B1012010BD0020FCE710B52BF0FD
:403B0000AAFA10BD00B5FEF7F3F810B9FEF7E8F808B1012000BD0020FCE710B5FEF7E8F820B1FDF762FF08B1012010BD0020FCE710B52BF090FA20B1FDF757FF08B101207E
:403B400010BD0020FCE710B501245D4890ED0C1BB0EE410AF0EE610A9FED5A1B53EC112B51EC100BB7F048FE20D2554890ED0E1BB0EE410AF0EE610A1FED9D1B53EC112BA9
:403B800051EC100BB7F056FC10D24D4890ED0E1BB0EE410AF0EE610A9FED4C1B53EC112B51EC100BB7F028FE00D200E00024204610BD70B504460D4634B1012C09D0022CEE
:403BC0000CD0032C14D10EE042A12846AFF0A4FE0FE042A12846AFF09FFE0AE041A12846AFF09AFE05E041A12846AFF095FE00E000BF00BF324890F8060130B304EB440183
:403C00003C4800EB011090F82C0064281DDA04EB440000EB0411384800EB0110807B642813DA04EB440000EB0411334800EB0110837B04EB44012F4800EB011090F82C2087
:403C40002EA1281DAFF088FA05E000231A462BA1281DAFF081FA70BD0021194890F8060168B1002009E000EB4003224A02EB031292F82C200A44D1B2401C0428F3DB084635
:403C800070470000000000000020AC4025642A256427252E32662200482200200D0100686D2B0020602A0020CE16002025730000572200207016010894000010257500006D
:403CC000582000200000000000003E400000000000003EC06770730D00000000676C6F0D0000000067616C0D000000006265690D00000000541800209019002025642F255A
:403D0000640000000020FE490870704731B52DED020B2DED068B0446FA4890ED000AB0EE409A06F02FFB002879D0002C7ED0F6480078002875D09DED070AF448D0ED010A79
:403D400030EE600AF0EE408A9DED060AD0ED000A30EE600AB0EE408A68EEA80A48EE080AB0EE600AB2F0B6FCF0EE409AE8480078012811D1B1EE680AF0EE408AB1EE480A01
:403D8000B0EE408A68EEA80A48EE080AB0EE600AB2F0A0FCF0EE409A9FEDDE0AF4EEC09AF1EE10FA10DDDC48007868B9B0EE691AF0EE480AB0EE680A23F0A3FEB0EE409A7D
:403DC000D248DDE9061206C0CE48D0ED000AB0EE490A25F04FF9F0EE400A00EE104AB8EE401ADFEDCE1A81EE210A80EE80AA04221021CB4816F048FE012810D0C94890ED37
:403E0000000A7AEE400A90ED000A9FEDC71A01EE200A80ED000A0421C14816F033FF05E0FFE79FEDC20ABF4880ED000AB54880ED009ABDEC068B3EBD10B5FCF75FFF0028C4
:403E40007BD0BB4890ED000ABA48007800EBC000B94901EB800080ED000AB84890ED000AB448007800EBC00001EB800080ED010AB34890ED000ADFEDA90A80EE201AAD483B
:403E8000007800EBC00001EB800080ED021AAD4890ED000AA748007800EBC00001EB800080ED030AA84890ED000AA248007800EBC00001EB800080ED040AA44890ED000A98
:403EC0009C48007800EBC00001EB800080ED050A9F4890ED000A9748007800EBC00001EB800080ED060A9B4890ED000A9148007800EBC00001EB800080ED070A964890EDCF
:403F0000000A8C48007800EBC00001EB800080ED080A88480078401C8649087008460078032801DB00200870432043F01BFD442043F018FD452043F015FD10BD10B58748E0
:403F4000007840B14FF47A71854800685EF0A7FB08B9012010BD0020FCE710B5FFF7EEFF10B18048007810BD69480078FBE710B506F0DBF910B19FED7C0A10BD9FED7B0A12
:403F8000FBE710B50446754804705EF06BFB7449086010BD31B52DED040B2DED028BB0EE408A0446FFF7CAFF70B3594800786D490978884208D1B0EEC80ADFED6D0AB4EEA7
:403FC000E00AF1EE10FA1BDD5348007838B96948DDE9031206C001204F49087072E0FFF7C6FFD4ED000AB4EEE00AF1EE10FA69D25C4800784649087000204749087061E05B
:404000000020454908705DE00020FFF7BAFF42480078F8B9B0EEC80ADFED550AB4EEE00AF1EE10FA4EDD1CF00CFA534908700846007837490978884204D04F480078344949
:4040400008703FE04B48DDE9031206C001203249087037E0FFF78BFFD4ED000AB4EEE00AF1EE10FA14D2B0EEC80ADFED410AB4EEE00AF1EE10FA07DD2548007808B90120FD
:4040800000E000202249087000202349087019E0B0EEC80ADFED360AB4EEE00AF1EE10FA10DD1CF0CEF9344908700846007818490978884206D0304800781549087000204C
:4040C00015490870BDEC028B05B030BD10B52DED068BB0EE408AF0EE608AB0EE419AB0EE48AAF0EE680AB0EE480A24F0C3FFF0EE409AB0EEE90ADFED210AB4EEE00A3FE068
:4041000034000020980000203500002090000020590000209A99193E5800002000007A446422002080000020CDCCCC3E000000007C000020840000207422002044000020F2
:404140008C000020880000206C000020400000203C000020480000204C000020280000202C0000205B0000209A99193F9A99993ED80FC93F600000205A0000203333B33EEB
:40418000F1EE10FA17D2F1EE000A69EE200AB0EE600AF7EE000AB4EEE00AF1EE10FA03DDF7EE000AB0EE600AF0EE680A49EE800AB0EE60AA00BFB0EE4A0A23F035FEBDEC27
:4041C000068B10BD10B52DED020B00BF04226946FE48006800F514700BF051F920B99DED000AFB4880ED940A00BF00201CBD10B52DED028B1FED330AB0EE408A042210218E
:40420000F44816F041FC012808D0F34890ED000AB0EE408A0421EF4816F034FDB0EE480ABDEC028B10BD2DE9FF432DED040B2DED0A8B81B00546F0EE41AA0C4616461F46C6
:4042400000EE106AB8EE400AE44880ED000AE4480078A84202D1B4F5FA7F15D9E04805700020E0490870DA4890ED940ADE4880ED000A90ED000ADD4880ED000ADA4890EDD8
:40428000000ADB4880ED000AD648007840BBD948DDE90B1206C0D848DDE90B1206C00020D6490870D6490870D64908701FED610AD54880ED000A1FED630AD44880ED000A3A
:4042C0000020D34908600120C64908705EF0CAF9D049086001B0BDEC0A8B08B0BDE8F0839DED0C0AC448D0ED010A70EE608A9DED0B0AD0ED000A30EE608A68EEA80A48EEB9
:40430000080AB0EE600AB2F0E5F9C34880ED000AC2480078012800D017B11FED820A01E09FEDBF0AF0EE40BA06F02CF810B1FFF75EFF01E01CF043F800EE904AB8EE601A3A
:40434000B248D0ED000A40EE010A1FED8C0A80EE801A80ED001AAC48D0ED000A00EE104AB8EE400A30EE800A80ED000AAA4890ED000AB4EEEB0AF1EE10FA3ED2A24890ED90
:40438000000ADFEDA80AB4EEE00AF1EE10FA20DD9E48D0ED000A9C4890ED001AC0EE811AB0EE610A994890ED001A00EE904AF8EE600A00EE601A80ED001A934890ED001A98
:4043C00000EE904AF8EE600A71EE600AC0ED000A00BF41F28831944800685EF060F958B1FCF78CFE40B1804890ED000AFFF7EAFE5EF038F98C4908606CE781480078D8B112
:404400009DED0C0A7B48D0ED010A30EE600AF0EE408A9DED0B0AD0ED000A30EE600AB0EE408A68EEA80A48EE080AB0EE600AB2F051F9794880ED000A774890ED001AF0EE1B
:40444000480AB0EE680A23F05CFB684880ED000AFDF7FFFC8DED000A7048007820B19DED000AB1EE400A01E09DED000AB0EE409A1FEDD30AB4EEC09AF1EE10FA0DD2664810
:4044800090ED001A5A48D0ED000A584890ED000AFFF71CFE554880ED000A58480078E8BB5448554A06CA06C05348DDE90B1206C01BF085FFF0EE400A00EE104AB8EE400AF2
:4044C0001FEDEA1AC0EE011A20EEA10AB0EE40CA9DED000A6CEE000A4F4890ED001A80EE810A4248D0ED000A30EEC00A3E4880ED000A3E4890ED000A3D4880ED000A012003
:404500003E4908701FEDF70A3F4880ED000A1FEDF90A3E4880ED000A002000E002E03C490860D7E6304890ED000A404880ED000AD0ED000A2D4890ED000A24F09BFDB0EECE
:4045400040AA364890F8008033489DED0C1ADDED0B0AB0EE4A0AFFF71DFD2748DDE90B1206C02748007850B19FED310A264880ED000A9FED2F0A254880ED000AAAE627486B
:404580000078804566D01F48007838B99FED290A3AEE800A144880ED000A05E0134890ED000A114880ED000A0F4890ED000A23F03BFC0D4880ED000A9FED1D0A124880ED6F
:4045C000000A9FED1B0A114836E0000020010010602E002064220020800000208C0000206800002034000020400000207C000020440000206000002050000020350000203F
:40460000580000205C000020700000206C000020740000202C0000208800002059000020CDCCCC3D0000FA43300000203C00002000000000DC0F494080ED000A0020AF49DB
:404640000860FFF78AFC81461BF0FEFE0020AC4908703FE6AB4890ED000AAB4880ED000A1CF04CF9A74880ED000AA748D0ED000AA44890ED000A24F0FDFCA44880ED000AA2
:404680009FEDA30AB4EEC09AF1EE10FA05D327B9A04890F84004072818D19F48D0ED000A89EE200A9D48D0ED000A20EE200AB0EE40CAB0EE4C0A23F000FA9948D0ED000AD4
:4046C00030EEC00A974880ED000A12E000BFB0EE4A0AB4F03DFB9048D0ED000A60EE200A80EE890A8F48D0ED000A30EE200A80ED000A8C4890ED000A8B4880ED000A8B4810
:40470000D0ED000A884890ED000A24F0B3FCF0EE409A7E4890ED000AF0EEC00A9FED840A30EE80BAD0ED000A39EEE00AF0EEC00A9FED7F0AF4EEC00AF1EE10FA21DD6F489A
:40474000006805281DDA05F0F0FDD0B1F5EEC09AF1EE10FA01DD012001E04FF0FF3000EE100A7248D0ED000AB8EEC01A41EE0B0A6C48C0ED000A61480068401C5F490860A1
:4047800008E0694890ED000A664880ED000A00205A490860634890ED000A23F045FB614880ED000AFFF748FB1FED5F0A5B4880ED000A1FED610A5F4880ED000A584890ED6A
:4047C000000A5D4880ED000A00BF83E55B4991ED010AD0ED010A30EE200A81ED010A91ED000AD0ED000A30EE200A81ED000A544991ED010AD0ED010A30EE200A81ED010AF8
:4048000091ED000AD0ED000A30EE200A81ED000A7047444890ED000A704710B5FFF78EFB48B14848007848490978884201D0012010BD0020FCE745480078F9E7414800781F
:40484000704770B50446FFF779FB48B13E48007808B1012000E0002005463B4804700FE03848007808B1012000E00020054635480470A54201D0012000E0002020490870DE
:4048800070BD3348007828B13248007810B12F48007808B1012070470020FCE72C48007820B12C48007808B1012070470020FCE725490870704710B5FFF74FFB08B100240D
:4048C00000E00124204610BD234890ED000A7047214880ED000A704700EBC0021F4B03EB820202EB810292ED000A70471C490978491EC8B2032800DB0220704774000020CD
:404900005C000020480000204C00002078000020CDCCCC3E602A0020880000206C0000207C00002040000020380000203C000020C7B8B23D7000002044000020600000207C
:4049400050000020590000205B00002058000020340000203500002024000020742200208400002070B52DED028B84B004460E461546D0480078B04202D1B5F5FA7F08DDBE
:40498000CC4806700020CC49087004B0BDEC028B70BDC948007838B9C848D4E9001206C00120C5490870F0E70A2D00DAEDE700EE105AB8EEC00ADFEDC20AC0EE808A94ED8E
:4049C000010ABE48D0ED010A30EE600A20EE280A8DED030A94ED000AD0ED000A30EE600A20EE280A8DED020A9DED030AB548D0ED010A30EE600A8DED010A9DED020AD0ED33
:404A0000000A30EE600A8DED000AAF4890ED000AB0EEC00ADFEDAD0A30EE200AAC4880ED000A90ED000ADFEDAB0AB4EEE00AF1EE10FA03DD9FEDA70A80ED000AA14890EDCD
:404A4000010ADDED010AA24890ED001A00EE810A9C4880ED010A90ED000ADDED000A9C4890ED001A00EE810A964880ED000A23F064FAB0EE408AB0EE480AF7F7C1FA10B129
:404A8000B0EE480A01E09FED940AB0EE408A9FED930AB4EEC08AF1EE10FA02DD9FED8E0A01E0B0EE480A884880ED000A94ED010A824880ED010A94ED000A80ED000A00BFEB
:404AC00063E770B52DED048B84B005460E46144683480078B04202D1B4F5FA7F08DD8048067000207F49087004B0BDEC048B70BD7C48007838B97C48D5E9001206C0012003
:404B000078490870F0E70A2C00DAEDE700EE104AB8EEC00ADFED6A0AC0EE808A95ED010A7148D0ED010A30EE600A20EE280A8DED030A95ED000AD0ED000A30EE600A20EE8B
:404B4000280A8DED020A9DED030A6848D0ED010A30EE600A8DED010A9DED020AD0ED000A30EE600A8DED000A614890ED000AB0EEC00ADFED560A30EE208A9FED560AB4EEDE
:404B8000C08AF1EE10FA03DD9FED520AB0EE408A564890ED010ADDED010A00EE880A80ED010A90ED000ADDED000A00EE880A80ED000A23F0C2F9B0EE409AB0EE490AF7F728
:404BC0001FFA10B1B0EE490A01E09FED430AB0EE409A9FED420AB4EEC09AF1EE10FA02DD9FED3D0A01E0B0EE490A414880ED000A00EE104AF8EEC00A9FED311A81EE200A0F
:404C0000D0ED000A3B4890ED001A70EEC10A20EE200A394880ED000A90ED000A3748D0ED000A70EE600A90ED000AB6EE001A00EE810A80ED000A95ED010A2B4880ED010AF8
:404C400095ED000A80ED000A294890ED000A294880ED000A00BF47E71B4890ED000A7047234890ED000A7047234890ED000A7047224890ED000A704700200F490870704722
:404C80000E4991ED010AD0ED010A30EE200A81ED010A91ED000AD0ED000A30EE200A81ED000A70470A4890ED000A7047144890ED000A7047B9000020B8000020A400002026
:404CC00000007A44AC000020B4000020CDCC4C3E9C000020CDCC4C3F00000000CDCC3242DD000020DC000020BC000020C4000020CC000020D0000020D4000020D8000020C5
:404D0000A00000200120A2490870704770B505460C46601B46B29F48006820B1E1B230469C4A1268904770BD70B506460C461546AC4207DA9848006820B100213046964A39
:404D400012689047AC4207DD9348006820B101213046914A1268904770BD2DE9F04107460C4615469846069E05F0DFFA38B94AF09CFF20B1894890F8FA00002875D0082DEE
:404D800074D1834844602A4641680830AEF098FD00286BD07E480078002868D17C484068007800F0030008B1012000E0002002467748007A00F0030008B1012000E00020BA
:404DC00001460020FFF7B0FF714840680078C0F3810008B1012000E0002002466C48007AC0F3810008B1012000E0002001460120FFF79AFF664840680078C0F3011008B1FA
:404E0000012000E0002002466148007AC0F3011008B1012000E0002001460220FFF784FF5B4840680078800908B1012000E0002002465748007A800908B1012000E000207C
:404E400001460320FFF770FF51484068C07800F0030008B1012000E0002002464C48C07A00F0030020B1012003E085E087E079E0002001460420FFF757FF45484068C078D6
:404E8000C0F3810008B1012000E0002002464048C07AC0F3810008B1012000E0002001460520FFF741FF3A484068C078C0F3011008B1012000E0002002463548C07AC0F378
:404EC000011008B1012000E0002001460620FFF72BFF2F484068C078800908B1012000E0002002462A48C07A800908B1012000E0002001460720FFF717FF25484068007921
:404F000000F0030008B1012000E0002002462048007B00F0030008B1012000E0002001460820FFF701FF1A4840680079C0F3810008B1012000E0002002461548007BC0F3E3
:404F4000810008B1012000E0002001460920FFF7EBFE0F4A5268B2F801100D4AB2F80900FFF7D4FE0A482A4641680830AEF06EFD00200749087002E0012005490870BDE8E5
:404F8000F081054908607047024908607047000004180010E4000020E0000020602A0020FE4890F85706704701B5FC4890F857069DF80010884213D000BF01226946F848EB
:404FC000006800F257200AF05AFA20B99DF80010F24880F8571600BF40F20910F3F7D5FA08BD10B57D231A46D900012036F0E4FE10BD10B57D231A469900012036F0DCFE5A
:4050000010BDE64991F86108704700B5FFF7F9FF042801D1012000BD0020FCE7DFEDE10AB0EE600A032808DAC0EBC001DE4A02EB8101D1ED010AB0EE600A7047DB48007857
:405040007047DFEDD80AB0EE600A032808DAC0EBC001D54A02EB8101D1ED000AB0EE600A704770B52DED028BF7F7B4F858B9D048F7F7BDF838B9CE48F7F7A4FC18B9CC4889
:40508000F7F795FC08B1012000E000200446C9480578FFF7B6FF06287ED2DFE800F003040FC01ABFBFE0C048406B18B90120C149087002E00020BF490870B4E0BA48006DE5
:4050C00018B90220BB49087002E00020B9490870A9E0B548406B00287ED10220FFF79EFFB0EE401A0120FFF799FF31EE400AF0EE408AB1F0EAFAB0EE408AFFF79FFF68BB0C
:405100009FEDAD0AB4EEC08AF1EE10FA26D20120FFF784FFF0EE408AB1F0D7FADFEDA70AB4EEE00AF1EE10FA18D20120FFF789FFF0EE408AB1F0C9FAA148D0ED000AB4EED2
:40514000E00AF1EE10FA09D29E480068052811D29C480068401C9B4908600BE0002099490860FFF76BFF08B1002001E09648007895490870DCB18C48006DC0B9924800787B
:4051800018B990480068052811D302208949087001208D49087000E041E08348D0ED070AB0EE600A1921894820F0FBFC31E0FFF745FF00BB794890F81308E0B184480078FF
:4051C000C8B17948006DB0B90120FFF727FFF0EE408AB1F07AFA00E01CE0DFED770AB4EEE00AF1EE10FA06D20220724908700120754908700DE001206E4908706A4890ED17
:40520000070A7248D0ED000A30EE600A664880ED070A02E000206749087004E000BF00206449087000BF00BF14B362480078A8421AD0FFF7EAFE88B1584890F8620701280A
:405240000CD15C480078012802D1FFF7D2FE05E058480078022801D1FFF7C3FEDD20F3F794F90B2042F07EFB00205949087015E00020544908609FED4B0A544880ED000A31
:405280000020524948609FED470A524880ED000A00204D49087001204D4908704E48D0F898110120DFF834C100DFBDEC028B70BD2DE9F04104460D4616460027FFF770FE3F
:4052C00010B101280ED106E032462946204631F041FA074606E032462946204632F0B7FC074600BF00BF3846BDE8F08131B500249DF80000052801DB02241FE09DF8000040
:40530000002801DC032419E000BF012269462448006800F261400AF0B2F820B99DF800101E4880F8611800BFDE20F3F72EF940F20910F3F72AF90B2042F014FB204638BDEA
:4053400010B51D20F3F721F96A20F3F71EF91E20F3F71BF91F20F3F718F92A2042F002FB10BD01211C4880F8641030F079FD074631F0C3FE32F0A4FDFFF7E2FF00200D4999
:405380000870FFF73EFE18B1FFF73BFE052802DB0120FFF7ABFF5421034821E0602A0020200100100000000014180010B000001078170010A0000010C7B8323E39FA0E3D2C
:4053C000B8000010BC000010C0000010A4000010C1000010AC000010F8FF0020099F0C08AEF017FCFE48002101604160002408E00020C4EBC401FB4A02EB81010875601CCE
:4054000084B2032CF4DBDFF8E0C300DF80466923042201215DF012FA30B1DFF8CCC300DF804601215DF046FADFF8BCC300DF804641460220DFF8B4C300DFA7BB0321EC48C6
:4054400080F8641000BF00224FF6FF710720DFF8A4C300DF0546022DF5D1DFF89CC300DF0646304631F079F8304631F0A7FC304632F02AFD06F001000028E4D0D94A243278
:40548000111F081FFFF714FFD649486301F140023C31081F32F054FDD249086531F0F8FFFFF7DFFDCFE7FFE70020DFF850C300DF00BFFEE72DE9F05F2DED028BB0EE408A78
:4054C00005460F46914698460C9E4FF0000BDA460FFA89F446E0A21905EBC20105EBC40022F003FDF0EE408AF4EEC88AF1EE10FA30DDC8EE280AB0EE600AA01905EBC00038
:40550000D0ED010A05EBC40090ED011A30EEC11A05EBC400D0ED010A41EE000AC7ED010AA01905EBC000D0ED000A05EBC40090ED001A30EEC11A05EBC400D0ED000A41EECC
:40554000000AC7ED000AC8F8004078EE680AB0EE608A10E038EE680AB0EE408AA01904B20AF1010A04FB06F0D8F80010884202DABAF1280FAFD3B5EEC08AF1EE10FA01DD0B
:405580004FF0010B5846BDEC028BBDE8F09F2DE9F04F2DED028B83B006460F4690469A46F0EE408ADDE90EB900200290DBF80040A9F10100A04201D2044602E0002C00DA96
:4055C000002407EBC401304622F08FFCB0EE408AB4EEE88AF1EE10FA2BD2109858B9BAF1000F03D000200190451E0FE0A9F10100019001250AE0BAF1000F04D0A9F10100AD
:405600000190012502E000200190451E38EEC80AF0EE408A01AB224641463846B0EE680A0095FFF747FF029001982844CBF8000020E0C8EE880AB0EE600A07EBC400D0ED06
:40564000010A96ED011A30EEC11AD6ED010A41EE000AC8ED010A07EBC400D0ED000A96ED001A30EEC11AD6ED000A41EE000AC8ED000A00BF029803B0BDEC028BBDE8F08F83
:405680002DE9F05F2DED048B06460F4690461D46DDE90EB9F2EE020AB2EE040AB2F0C0FFF0EE408A4FF0000A9FED550AB0EE409A4A46102105F1B80015F0E6F9012843D097
:4056C00000243AE008EBC401384622F00EFC05F5A76000EB840080ED000A4A4890ED161AF0EE410A05F1D80000EB840090ED001AB0EE410A23F0BEFCF0EE409AB0F0E5FF05
:40570000B0EE408A05F5A76000EB840090ED000AB4EEE80AF1EE10FA0DD2B4EEC98AF1EE10FA08D2A24605F5A76000EB840090ED000AF0EE408A601C04B2B442C2DB49461B
:4057400005F1B80015F09EFA5046BDEC048BBDE8F09F2DE9FF4F2DED020B2DED0E8B8FB00E469046B0EE40AA9A4600200A901FEDF30AF0EE408A08F1100408F1C807002568
:4057800081461FEDF80AF0EE409A09F0D7FD04902C99049843463246CDE900010FFA8AF01F99FFF76DFF05460995AAF1010000B2079009990798814202D10998401E099008
:4057C000099A521C06EBC201099A06EBC20008F1640222F0FEFEF0EE408AF5EEC08A13E0A40000101418001031AB0C08099F0C08F8FF0020699F0C08B19E0C08C5A90C08A5
:40580000792C494058200020F1EE10FA01D2012000E00020E070E07810B14FF0FF3000E001208346BDB96A1C06EBC20106EBC5001F9A22F0E3FEF0EE408AF5EEC08AF1EE5E
:4058400010FA03D20A9840F480700A90E07880B3681C05B22DE00798854217D16A1E06EBC20106EBC5001F9A22F0C8FEF0EE408AF5EEC08AF1EE10FA03D20A9840F48070EC
:405880000A90E078A8B9681E05B212E005EB0B0206EBC20106EBC5001F9A22F0AFFEF0EE408AF5EEC08AF1EE10FA02D2A5EB0B0005B2A94606EBC90003C8C4E9060109EB87
:4058C0000B0006EBC00106C9C4E9081204F1200204F1180104F1280022F073FD09EB0B00207084F8019084F802A0257105A904F1280022F049FE05AA04F118011F9822F097
:405900009AFEB0EEC00AF0EE408A102108F1B8002C9A15F0B9F801280BD0C7ED038AA7F804905CF09FFEB86008F1B8002C9915F0A9F994ED070AD4ED0B0A08EEA00A84ED52
:40594000030A94ED060AD4ED0A0A08EEA00A84ED020A94ED090AD4ED070A30EE600A84ED050A94ED080AD4ED060A30EE600A84ED040AD4E90601C4E90C01D4E90212C4E9C2
:405980000E12D4E90812C4E910129FEDF90A84ED120A9FEDF70A84ED130ABAF1020F7DD90A9800287AD198F8080000EE100AB8EE400AF0EE000A20EE200AF0EE40BA98F8AB
:4059C000080000EE100AB8EE400AF0EE000A20EE200AB0EE40CA0020049000BF102108F1B8002C9A15F050F8012811D00498012806D187F84405B888401CA7F8480502E09F
:405A0000002087F8440508F1B8002C9915F03AF9CDF82490012009A9CDE9001A0290E378B0EE6B0A0BAA314604F10800FFF7AFFD10B14FF4007000E000200A9908430A90ED
:405A400009EB0B000990002109A8CDE901A10090E378B0EE4C0A0DAA314604F10800FFF796FD10B14FF4806000E000200A9908430A909DED0E0ADDED0C0A30EE600A84EDEA
:405A8000050A9DED0D0ADDED0B0A30EE600A84ED040AB5EEC0AAF1EE10FA00E012E102D2B7EE000A01E0BFEE000AF0EE40CA98ED010A60EE0A0AB6EE001AB0EE6C0A00EED2
:405AC000810AF0EE409A0020039009EB0B000990F5EEC09AF1EE10FA15D219EE900AB6F083F841EC1E0B9FEDA30B53EC102BB5F0DDFC41EC1D0BB5F04DF909EE900A0120CF
:405B00000390CDF824900998089009A90398CDE9001A0290E378B0EE690A04F13802314604F10800FFF733FD10B14FF4006000E000200A9908430A90BAF1030F08D197ED36
:405B4000550A84ED120A94ED120A84ED130AB8E0099818B10999079881420DD107F5A870099900EB810090ED000A84ED120A94ED120A84ED130AA4E004F1400104F1080012
:405B800022F0B3F9B0EE409A07F5A870089900EB810090ED000AB0EE40BAB1EE080AB4EEC09AF1EE10FA07DD9FED710AB0EE40BAB1EE080AB0EE409A04F1300104F108000A
:405BC00022F093F9B0EE408A0898A0EB0B0107F5A87000EB8100D0ED00AAB1EE080AB4EEC08AF1EE10FA07DD9FED610AF0EE40AAB1EE080AB0EE408A29EE2A0A08EE0B0AE9
:405C000079EE080A80EE201A84ED121A099806EBC00106C9C4E9101204F1400104F1380022F063F9B0EE409A07F5A870099900EB810090ED000AB0EE40BAB1EE080AB4EED8
:405C4000C09AF1EE10FA07DD9FED490AB0EE40BAB1EE080AB0EE409A0998A0EB0B0006EBC00003C8C4E90C0104F1300104F1380022F03BF9B0EE408A0998A0EB0B0107F5BB
:405C8000A87000EB810090ED000AF0EE40AAB1EE080AB4EEC08AF1EE10FA07DD9FED340AF0EE40AAB1EE080AB0EE408A29EE2A0A08EE0B0A79EE080A80EE201A84ED131AE7
:405CC00000BF00BF94ED130AD4ED120A30EE600A20EE290A84ED140A0A980FB0BDEC0E8B06B0BDE8F08F10B52DED028BF0EE408A044694ED001AF0EE410A94ED011AB0EE7A
:405D0000410A21F06CFFB0EE408A38EE680AB0EE408A05E09FED190A38EE000AB0EE408A9FED170AB4EEC08AF1EE10FAF2D305E09FED120A38EE400AB0EE408A9FED110AB5
:405D4000B4EEC08AF1EE10FAF2DCB0EE480ABDEC028B10BD10B50C49086E01215CF0E8FD0948016E0120DFF824C000DF10BD000000000000000000000000F0BFDC0F49403F
:405D8000D80FC9BFD80FC93FF8FF0020099F0C085FED090AB0EE600A032808DAC0EBC001FE4A02EB8101D1ED020AB0EE600A70470146002003290ADAC1EBC102F74B03EB7C
:405DC000820292690AB9012200E00022104670470146F348B0F8AA0500EE100AB8EE400ADFEDF00A30EE600ADFEDEE0A80EE201A81ED001AEA4890F8A82500F2AC5000EBBC
:405E00008202E74890F8A90532F8100000EE100AB8EE400ADFEDE40A80EE201A81ED011ADF4890F8B4050872DD4890F8B6054872DB4890F8100600EE100AB8EE400AF2EEBF
:405E4000040A80EE201A81ED031A01207047D7480078704731B50024BDF90000B0F57A7F04DD4FF47A700090022406E0BDF90000002802DA00200090032400BF0222694690
:405E8000CB48006800F5D57009F0F9FA28B9BDF8000081B2C248A0F8AA1500BF1D20F2F774FB2A2041F05EFDC248016E0220DFF808C300DF204638BDF7B50C4615460026F7
:405EC000BDF90000B0F5FA7F04DD4FF4FA700090022606E0BDF90000002802DA002000900326B64800EB840030F81500BDF90010884222D000BFAE49096801F5D67101EB93
:405F0000840101EB45000222694609F0B8FA38B9BDF8000081B2A94800EB840020F8151000BF6A20F2F731FB2A2041F01BFDA148016E0220DFF880C200DF3046FEBD31B53D
:405F40000024BDF800000A2803DD0A200090022406E0BDF80000012802DA01200090032400BF022269469248006800F5DA7009F086FA20B9BDF800108948A0F8B41500BFC3
:405F80001E20F2F702FB2A2041F0ECFC8948016E0220DFF824C200DF204638BD31B50024BDF800000A2803DD0A200090022406E0BDF80000012802DA01200090032400BF19
:405FC000022269467A48006800F5DB7009F057FA20B9BDF800107248A0F8B61500BF1F20F2F7D3FA2A2041F0BDFC7248016E0220DFF8C4C100DF204638BD31B50024BDF8D7
:406000000000FA2802DD0A200090022400BF012269466748006800F5047009F030FA28B9BDF80000C1B25E4880F8101600BF2320F2F7ABFA2A2041F095FC5E48016E02202B
:40604000DFF874C100DF204638BD5D480068401C5B490860704700B50246002359480270FFF7F3FF184600BD002055490860704710B5554C47F013F9012827D0204690F8E4
:406080004202FE2802D004F510741FE04E4890F80203FE2806D0424890F85308032801D14A4C13E048488078FE2801D0464C0DE0454890F88201FE2801D0454C06E0424888
:4060C00090F8C200FE2801D03F4CC034204610BD10B5FFF7CDFF8078FE2801D0012010BD0020FCE700B5FEF78CFF042803D0FEF788FF012801D1012000BD0020FCE710B5F5
:40610000274890F85308032804D13248F6F779F80B2801D1012010BD0020FCE700B5FEF770FF042803D0FEF76CFF022801D1012000BD0020FCE7284890ED000A704700B587
:40614000FEF75FFF022801D1012000BD0020FCE700B5FEF725FF08B9012000BD0020FCE700B5FFF774FE022801D1012000BD0020FCE701B500BF012269460D48006800F28F
:40618000134009F07CF920B99DF80010044880F8131800BF7120F2F7F8F908BD14180010602A00200000C84200009642A000001020010010F8FF0020099F0C080C300020EA
:4061C000B4000010B0000010D84A0220D84D0220584C022078170010A400001001B500BF012269467C48006800F2623009F047F920B99DF80010794880F8621700BF7020C8
:40620000F2F7C3F908BD012809D0022813D003281DD19FED730A734A82ED000A18E0714AD2ED000A00EE101AB8EE400A30EE800A82ED000A0CE06B4AD2ED000A00EE101A66
:40624000B8EE400A30EEC00A82ED000A00E000BF00BF70476448406B704700B5FFF7FAFF00F0010000BD00B5FFF7F4FFC0F3400000BD00B5FFF7EEFFC0F3800000BD00B5CD
:40628000FFF7E8FFC0F3C00000BD00B5FFF7E2FF00F08001FFF7DEFF00F01002802901D0102A01D1012000BD0020FCE700B5FFF7D1FFC0F3401000BD00B5FFF7CBFFC0F335
:4062C000002000BD00B5FFF7C5FFC0F3802000BD00B5FFF7BFFFC0F3402000BD00B5FFF7B9FFC0F3C02000BD00B5FFF7B3FF08B9012000BD0020FCE73B48006D70473A482E
:40630000006D08B9012070470020FCE73748006808B1012070470020FCE710B52DED028BB0EE408A324880ED008A6F20F2F72DF9BDEC028B10BD2E4890ED000A704710B57A
:406340000024264890F85308032804D005F082F908B9012400E00024204610BD7FB50546284601A90EC93AF07EFB0446FE2C32D0012068701F4A4FF6A071284640F0E9FD59
:4063800004461D4A4FF63F71284640F0E2FD04431A4A4FF45041284640F0DBFD0443184A4FF45941284640F0D4FD0443144A4FF45841284640F0CDFD0443114A4FF457416A
:4063C000284640F0C6FD04430E4A4FF6FF71284640F0BFFD04437FBD20010010602A002000000000A400001014180010B4000010B80000104B9E02086F480B08133A0B0897
:40640000A93205084771050810B50220FE490870002008715CF026F9FB498860002088600120487041F288304880012008750021F54801765CF016F9F349C8610021F248B7
:40644000C1610121417541F28831C182152141620220EE49087010BD10B5ED480078ED490870ED4800784870EC4800788870EC480078C870FFF7C8FF10BD0421018000211E
:406480004180012181800021C1800181704770B50446042C01DD002070BD44BBE148B0F8460828B9DF48B0F8480808B9012523E0D748007859F06AFC00EE100AB8EE400A4D
:4064C000DFEDD90A20EE200ABCEEC00A10EE106AD448B0F84608B04206D8D248B0F84808B04201D3012000E00020054604E0C949085D59F0E5FD054694B925B15CF0B2F8B9
:40650000CA4908600CE05CF0ADF8C8490968401A41F65831884201D2012000E0002005460DB10120B8E70020B6E770B504460025012C11DA84B9B648007859F027FC00EE6A
:40654000100AB8EE400ADFEDB80A20EE200ABCEEC00A10EE100A85B2284670BD2DE9F04106463007070E042F02DD0020BDE8F0810025002410E03819042805DAA549085DDE
:4065800059F09EFD804601E04FF00308610008FA01F00543601CC4B2102CECDB2846E5E72DE9F0470746884615461E464FF00009002448E004EB8400934911F82000B8420E
:4065C00040D104EB840001EB80000079404539D14FF00109012D00D05EB104EB84008A4901EB8000457004EB840001EB8000468028E086480078401EA04206D1002004EBCD
:406600008401814A02F8210017E0804A1278521E02EB82027C4B03EB820104EB840203EB82001422ADF099FA002178480078401E00EB8000744A02F8201074480078401EA4
:4066400072490870641CB9F1000F03D16F4800788442AFDBB9F1000F2ED16C480078202802D10120BDE8F087012D00D016B36748007800EB8000644901F82070634800786D
:4066800000EB800001EB800080F804805F48007800EB800001EB800045705C48007800EB800001EB8000468058480078401C5749087001E00220D5E70020D3E77CB5002627
:4066C00000250024CEE0002604EB84004E4911F8200000B9C9E004EB84004B4901EB80004088B0B104EB84020B4603EB8202518804EB840203EB8202D0685BF0D0FF40B111
:406700005BF0B0FF04EB84013F4A02EB8101C86001263EB904EB84003B4901EB80004078012819D104EB8400374911F82000022809D104EB8401344A02EB81010879FFF787
:406740000DFF054608E004EB84012F4A02EB81010879FFF79CFE0546A6B904EB84002A4901EB8000407801280CD104EB840001EB80008068A84205D004EB840001EB80004E
:4067800085600126F6B304EB84001F4911F82000022816D104EB840001EB800001799DF8000061F387108DF800009DF8000020F03E008DF80000CDF80150684640F083FFD3
:4067C0004EE004EB8401104A02EB81010879C11700EB117109119DF8042061F347128DF8042004EB8401084A02EB81010879C11700EB11710911A0EB01119DF8042061F380
:40680000440215E02CE0000068180010EC00002084050010E8000020830500108205001085050010602A002000404E3FF00000208DF804209DF8050065F301008DF805005E
:4068400004EB84000F4901EB8000007C9DF8051060F387018DF8051001A840F03CFF00BF601CC4B2202CFFF62EAF00BF7CBDFFF7F3FD05E0FFF722FF2820DFF80CC000DFBF
:40688000F8E7000068180010A99E0C08FC4908707047FC480078092801D1012070470020FCE7F84800780B2801D1012070470020FCE7F4480078012800D170470020FCE700
:4068C000F0480078062801D1012070470020FCE770B58CB004460D46E21704EBD2625311E94A02EB830212682146E31704EBD3635B11A4EB43160123B3401A432046E317C2
:4069000004EBD3635E11E04B03EB86031A60DF480470FFF7D5FF40B9FFF7BBFF28B9FFF7C8FF10B9FFF7BDFF40B1FFF7B2FF28B9272D03D10120FFF7A9FF14E0D44BD5A296
:40694000232102A80095ACF01DFC02A8ADF008F8461C324602A9D24893F0EAF901212846F7F7E4FE00BF282D04D02A460021CC4893F00DFAECB302220421CA4814F084F8A2
:40698000012818D0C74890F82E1090F82E00401CC44A82F82E0002F110004454103890F82E001E2803DB0020114681F82E000221BC4814F067F903220421BB4814F064F816
:4069C000012816D05BF04EFEB84941F83400084600EBC4000079FF2807DA084600EBC4000079401C01EBC40108710321AE4814F049F9232040F0B6FF0CB070BDAC4890F81C
:406A00002000012800D170470020FCE7A84890F8210008B9012070470020FCE710B503F084FC00B910BD9FF009F8A24908709FF015F8A1490870A14890F84E04A049097871
:406A4000884206D19D4890F8F9059E490978884212D001209C4908709C4908705BF002FE9B490860954890F84E0495490870934890F8F905934908700DF039FF02287DD115
:406A80004FF4FA71924800685BF009FE60B18948007810B900208C49087087480078012802D10020894908708248007801284DD18848007801280CD0FFF716FC48B18248B6
:406AC000007830B95BF0CEFD83490860012083490870F5F77FFB58B98148F5F788FB38B97F48F5F76FFF18B97D48F5F760FF08B1012000E00020C8B978480078002862D0F7
:406B00006E4890F84F0458B16C4890F84F04642210FB02F1704800685BF0C1FD002852D0F5F7BCFB00206D4908704CE0F9F7B7FF40B1F9F7C2FF044621460920FFF7C8FE3A
:406B4000F5F7B8FB0020654908703CE05A480078012838D16348007848B95C48007830B95BF080FD60490860012060490870F5F731FB68B95A48F5F73AFB00E02CE038B9AB
:406B80005748F5F71FFF18B95548F5F710FFD0B156480078B8B1494890F8D50450B1474890F8D504642210FB02F14F4800685BF076FD40B1F5F77EFB28210220FFF788FE62
:406BC00000204A4908703C48007846490870394800784049087004E001203C4908703A49087000BF1EE710B59EF002FB01280FD19EF0D7FA60B19CF01DFD012808D1A4F0A7
:406C0000CBFA012804D1FFF701FF08B1012010BD0020FCE710B5044603F087FB08B1022C01D1012010BD0020FCE770B504460D46607B01285CD1A06868B1D4E901015BF0A5
:406C40002EFD002806D0002211462046F5F7DBF80120E073A1E02846FFF7DCFF00280ED04FF4FA6160685BF01AFD002807D00220A07325210820FFF72BFEF5F71BFB8CE01C
:406C800000010020F5000020811D0010F7000020DEE00C08257320636F64653A20256400BCDD0010501D0010401D0010401B0010E81A00101401002015010020602A0020AC
:406CC00018010020190100201A0100201B0100201001002016010020080100201C01002078170010170100200C0100201D010020A07B022802D10020A0734EE0207B01285D
:406D00004BD10020E073F5F765FA38B9F948F5F74EFE18B9F748F5F76AFA30B1F5F7CAFA26210320FFF7D4FD37E0FFF75CFF48B1F9F7B5FE30B9F5F7B1FA29210020FFF709
:406D4000C7FD2AE09CF076FC012804D028210420FFF7BEFD1FE09EF04BFA012804D01B210320FFF7B5FD16E09EF01BFA20B91A210120FFF7ADFD0EE0F9F791FE38B1F9F7A2
:406D80009CFE064631460920FFF7A2FD03E027213120FFF79DFDF5F78DFA207B617B884202D04620F1F7F1FBE07B08B9607B207370BD70B504460225152C02DA0025CE4847
:406DC00004709F20F1F7E1FB284670BD10B50020FFF7EFFF0121C948006839F0C0FE0220C549487010BD0020C54908707047F0EE400A9FEDC41A20EE811AB0EE410A9FEDF4
:406E0000C21A30EE011AB0EE410AB1EE001A20EE011AB0EE410AB6EE001A30EE011AB0EE410A9FEDBA1AB4EEC10AF1EE10FA03DD9FEDB61AB0EE410ABCEEC01A11EE100A31
:406E400080B2704700B52DED028B81B0B04890F8260001281DD1AE4890F82700012818D1FFF72EFD40B9FFF714FD28B9FFF721FD10B9FFF716FD38B10120A54981F82800A7
:406E80005BF0F0FBA24948600020A14981F827005BE09F4908685BF023FCB0F57A7F54D39B4890F8260001284FD1192204219848083013F0E9FD012847D05BF0D3FB95492B
:406EC0000860DFED950A9FED940AA3F09FF8B0EE408AFFF78CFF8E494883DFED8F0A9FED8E0AA3F093F8B0EE408AFFF780FF88490883012081F82400022081F82300002064
:406F000081F82000022081F8220091F822009CF027FB00207E4981F821005620F1F735FB00207B4981F82600012081F82700FFF75AFF19217648083013F0A4FE7748D0F8A4
:406F400088120120DFF8D8C100DF714890F82700012812D103F06EFF78B16E4800685BF0BFFB43F69821884207D3FFF72FFF48F07EFD5BF077FB67490860654890F8280048
:406F800080B3634948685BF0ABFB40F6C411884228D3644800680090634890F8A825574803210368614845F05DFF5E48006800905D4890F8A9255148032103685B4897304A
:406FC00045F050FF574800680090574890F853284A4803210368564845F044FF00204C4981F8280001B0BDEC028B00BD44480078C0F38000704742480078C0F34000704709
:407000003F48007800F0010070473D480078072801D1012070470020FCE74649087070477FB545484FF0A3FE042825D0002421E0012504B90025002204EB44003F4901EB5A
:40704000801005EB85013E4B03EBC101CDE90041CDE902020522002337484FF02AFF38B104EB4400354901EB80103649086003E0601CC4B2022CDBDB7FBD10B503F0E9FD5F
:4070800030B10022134660212F4839F04DFD9BE003F098FE30B10022134627212B4839F043FD91E003F0C6F930B100221346D221274839F039FD87E003F09CFE30B100224E
:4070C00013460621234839F02FFD7DE003F03CFE30B10022134631211B4839F025FD73E003F03FFEC0B3002213460621164839F01BFD69E078170010F5000020C80200204C
:407100000101002000007A440000FB4500FF7A47141B00102001002000000000F8FF0020099F0C08DC020020602A002058010800AE040800F4000020986C0220D8620220C3
:40714000186B0220CC020020985A0220585B0220D8590220185C0220FFE703F0AAFD30B100221346FC21FE4839F0DEFC2CE003F051FE30B1002213460321F94839F0D4FC60
:4071800022E0F84890F844041C2806D1002213462721F54839F0C8FC16E003F065F950B1002213461321EE4839F0BEFCEFA1F54892F0CEFD08E003F059FE28B10022134605
:4071C0009021F14839F0B0FC10BD10B503F041FD88B903F0F7FD70B903F02CF958B903F009FE40B903F0B0FD28B903F062FD10B903F010FE20B10121D94839F0B0FC08E032
:40720000D84890F844041C2803D10121D64839F0A6FC10BD10B5002403F01BFDE0B903F093FDC8B903F09DFDB0B903F042FD98B903F000F980B903F0DDFD68B903F0EAFD77
:4072400050B9C84890F844041C2805D003F00CF910B903F00BFE00B10124204610BD10B503F0F7FC88B10820FFF7A3FD002213461321C64839F058FCC448C5490860C548DB
:40728000C54908600020C549487003F09AF888B10D20FFF78EFD002213461321BB4839F043FCBA48BA490860BA48BB4908600020BA49487003F062FDA0B103F0CFFD88B993
:4072C0000E20FFF776FD00221346F021AF4839F02BFCAE48AE490860AE48AF4908600020AE49487003F052FDA0B10F20FFF761FD002213462721A548C03039F015FCA348CF
:40730000C030A3490860A3482830A34908600120A249487003F0C5FCA0B11120FFF749FD0022134627219948C03039F0FDFB9748C0309749086097482830974908600120D0
:407340009649487003F09DFC88B11320FFF731FD0022134614218D4839F0E6FB8B488C4908608C488C49086000208C49487003F090FC88B10420FFF71CFD00221346132163
:40738000824839F0D1FB81488149086081488249086000208149487010BD10B5002403F058FC88B903F0F2FC70B903F0E7FC10B103F054FD40B103F004F828B903F071FC31
:4073C00010B903F05EFC00B10124204610BD74480078704710B50121724839F0C0FB10BD6E480078122801D1012070470020FCE7F0EE400A9FED6C1A9FED6C0A00EE810A67
:4074000070476B48C08B00EE100AB8EE400A704700B5FFF7F6FFDFED650A70EE600A1FEDC71A80EE810A00BD6148808B00EE100AB8EE400A704710B52DED028B0024FBF7BD
:40744000C1FDB0EE408AF4F7DBFD00283BD15948008890B1F4F7BEFE58B95748F4F7C7FE38B95548F5F7AEFA18B95348F5F79FFA08B1012000E0002010BB07F011FF18B1F6
:4074800000204C4908801BE007F001FF40B1FFF7CBFFBCEEC00A10EE100A464908800FE007F007FF40B1FFF7B3FFBCEEC00A10EE100A4049088003E03D48408B3D490880E6
:4074C0003C48048802E000203A49088033480078152844D2DFE800F0FD7AD10B0C437B0D0EB90F8D161012111314FC15170000BF00BF00BF00BF00BF00BF00BF00BF00BF96
:4075000000BF00BF00BFF4F765FE58B92A48F4F76EFE38B92848F5F755FA18B92648F5F746FAD8B1FBF74EFDB0EE408AF4F768FD48B9FBF747FDB0EE408A99F053F968B1D4
:407540009AF0EAF950B19EF0EAFCDFED1C0AC0EE208AA1F078FA38EE800A31E035E0E3E0985A0220602A0020D859022043542D353620666F7263652072656769737465724F
:4075800065640000BCDD0010586A022058520220C8020020186B0220DC020020F5000020F4000020D85C02200000C84200401C46141B0010040100207817001000007A452F
:4075C000B0EE408AFFF713FC0446B0E000BFF4F701FE68B1FBF7F6FCB0EE408AF4F710FD30B107F067F8B0EE408AFFF700FC04469DE0F4F7EFFD38B3FBF7E4FCB0EE408AEA
:40760000F4F7FEFC00B307F035FE38B107F052F8B0EE408AFFF7EBFB044615E007F049FE38B107F047F8BCEEC00A10EE100A84B20AE007F03FF8B0EE408AFFF7D9FEBCEEC5
:40764000C00A10EE100A84B271E0F4F7C3FD98B1FBF7B8FCB0EE408AF4F7D2FC60B107F029F8F0EE408AA3F0FCF938EE800AB0EE408AFFF7BCFB044659E09AF0F1FC07289F
:407680000FD2DFE800F00508040F06070B0000BF00BF00BF00BF4FF6FF742CE0F848048B29E000BFF4F796FD58B9F648F4F79FFD38B9F448F5F786F918B9F248F5F777F950
:4076C000C0B1FBF77FFCB0EE408AF4F799FC01E013E028E070B19EF022FC5FED480AC0EE208AA1F0B0F938EE800AB0EE408AFFF77EFB044600BF00BF19E0E148048BFFF7F5
:407700007DF901280ED19EF00AFC5FED540AC0EE208AA1F098F938EE800AB0EE408AFFF766FB044603E000BF4FF6FF7400BF00BF2046BDEC028B10BD00B50020FFF76DFCE5
:4077400000BD0EB5D048002101802C21CF48ACF060FA2C21CA48ACF05CFA4FF40071CC48ACF057FA3021CB48ACF053FACA480021016081800D21C948ACF04BFA0D21C8482F
:40778000ACF025FA4FF050080025A9460121C54880F8CC11BB48F4F79FFD0020B84981F82600012081F82700002081F82800FFF700FB0220B44948700020FFF72EFC9DF07E
:4077C0000EFF0020B8490870B84839F0EBF90321B44880F8CC1100BF002241460F20DFF8D0C200DF84B2022C30D1DFF8C8C200DF054605F0020038B1FFF71DFEAE49088022
:40780000012040F0AFF821E005F00800F0B10021AA481CF016FA06469A48F4F7F2FC824606F04CFF8DED010AFBF7CCFB8DED020A534601AA02A9A24800964EF0EFFE9F482D
:407840001CF07CF99F4852F0FCFD00BF012C7CD19D4890F84D04092803D150209AF087FC00E000BF00BFFFF7BBFD08B198F0AAFB02F0A7FD60B101209449487098F06DF9AF
:4078800030B998F0BCFA98F068F908B1FFF7A2FD0CF0B1F920B3FFF79AFD08BBF4F79AFCF0B97848F4F7A3FCD0B97648F5F78AF8B0B97448F5F77BF890B9FFF76EFD18B181
:4078C000FFF784FAFFF7CBFCFFF7A4FC18B1FFF77CFCFFF7D2FBFFF7A3FB0120FFF79DFBFEF7EEFF40B9FEF7D4FF28B9FEF7E1FF10B9FEF7D6FF10B1FFF787FB38B1012154
:407900006F484FF022FBE8B352F075FCD0BB48465AF0E6FE42F2107188423BD3FFF770FB40B96B4803686B48002102684FF6DA603DF0A7FDFFF75FFB50B9654803686548EE
:40794000002102684FF6C55000E038E13DF099FDFFF74CFB40B95E4803685E48792102684FF46F403DF08DFD012155484FF0EDFA68B152F040FC50B9544B2833564800218E
:40798000026800E006E04FF6DA603DF07AFD5AF069FE8146192210213948083013F074F8012809D02C2236493848ACF0D6F819213348083013F066F9FFF744FA9DF06CFD36
:4079C0009EF009F800214548FFF72FF901214448FFF72BF902214348FFF727F903214248FFF723F904214148FFF71FF905214048FFF71BF906213F48FFF717F907213E480A
:407A0000FFF713F9FFF70AF899F0E2FF98F01AFBF4F7E0FB58B91B48F4F7E9FB38B91948F4F7D0FF18B91748F4F7C1FF08B1012000E000200746002F21D001202F490870FD
:407A4000FEF7E4FF30B1FEF7D9FFB0B92C480078142812DBF4F72EFC9DF0CAFB012804D01B213420FEF734FFA6E09DF09AFB28B91A213420FEF72CFF9EE06DE042E093E04E
:407A8000141B001078170010F5000020E81A0010401B0010501D0010F8000020801D00108D1D0010F8FF00200101002039770108699F0C08B19E0C08FE000020604F00100C
:407AC000986C0220CCD10010602A0020186B0220DC020020C8020020CC02002044D5022054D5022064D5022084D5022094D50220A4D50220B4D50220C4D502200301002082
:407B0000020100209BF096FD012804D028213420FEF7DEFE50E0FA48F4F749FFB8B9F848F4F750FF98B9F648F4F761FB78B9F8F7B6FF60B1F8F7C1FF064606EB8601F14A9F
:407B400002EBC101887B3146FEF7C2FE34E027213420FEF7BDFE2FE0E948F4F728FFC8B9E748F4F72FFFA8B9E548F4F740FB88B9F8F795FF70B1F8F7A0FF0646F4F79AFBB9
:407B800006EB8601DF4A02EBC101887B3146FEF79FFE11E0DC48007814280DDADA480078401CD949087007E0D848007820B10020D5490870D5490870D148F4F7A0FB0025C9
:407BC0000AE6D34890F8260008B9012070470020FCE710B50D21CF48ACF01BF810BD70B50023012115E0CC1701EBD4646511C94C641C04EB85042468CD1701EBD5656D11AD
:407C0000A1EB45160125B5402C4004B10B46481CC1B24029E7DB184670BDBF4890F822007047BD4890F823007047BC480078022801D1012070470020FCE710B5FFF7F5FF72
:407C400018B19AF013FA044602E0B34890F82540204610BDB24800887047B0F57B4F01DB4FF6FF2000EE900AF8EE600AB1EE001AC0EE811AB0EE610ADFEDAA0A70EE600A4A
:407C8000B0EE600ADFEDA80A80EE201AB0EE410A7047F0EE400A9FEDA51A20EE811AB0EE410A9FEDA31A30EE011AB0EE410A9FEDA11A20EE011AB0EE410AB6EE001A30EE51
:407CC000011AB0EE410ABCEEC01A11EE100A80B270478F48408B7047F0EE400A9FED960A30EEC01ADFED951A81EE210A704700B5FFF79AFBB0EE402AFFF7EEFF00BD10B5DC
:407D00000024FFF76DFB18B198F0CFF9044612E0F4F760FA58B97A48F4F769FA38B97848F4F750FE18B97648F4F741FE08B1012000E00020044644F0FC0010BD774800780B
:407D40000D2801D1012070470020FCE7734800780E2801D1012070470020FCE72DE9F0472DED048B07460C4692469846DDF8309002F060FB30B1A078FD2803D1BDEC048BB4
:407D8000BDE8F087FFF7E2FF28B16D480068C078404500D0F2E70025FFF7D0FF18B1204697F010FF24E0B7F56F4F0AD12078AA2807D12046A4F05EF80121624819F0FDF91F
:407DC00016E0B7F52C4F04D1A4F021F908B900250EE0B7F56F4F0AD1FEF763FD38B12078AC2802D02078AE2801D1012500E0C5E7192250214648083012F046FE01286DD03E
:407E0000615D681C205C41EA00264148068303F05FFC30B13E48868300203D4981F8240028E003F063FC30B13948C6830020384981F824001EE0B6F57B4F15DBFBF7C6F8CA
:407E4000F0EE408A18F0BBFAB0EE409AF0EE680AA2F0DCF8B0EE408AFEF7C9FF2C494883012081F8240005E0294846830020284981F82400A81C205C00F00300244981F8E6
:407E80002300A81C205CC0F3810081F82000A81C205CC0F3011081F82200A81C205C800981F8210091F822009BF05AFB5AF0DAFB17490860012081F82600E81C205C400995
:407EC00081F8250019211248083012F0DBFE1E48D0F888120120DFF874C000DF00BF4DE70E48007808B1012070470020FCE770B504460025164890F85604FF282AD12AE114
:407F00007817001008BF0C080201002003010020141B0010801D0010E81A0010F5000020FE0000200000FB4500007A44E12E6542D7A320430000484300401C460000C84287
:407F4000C802002058490010F8FF0020099F0C08602A0020092C06D1FE4890F84C04032801D00125F7E0012C06D1FA4890F84C04032801D00125EEE0062C06D1F54890F8EA
:407F80004C04032801D00125E5E00C2C0BD1F14890F85308022804D0EE4890F85308032801D10125D7E0042C14D1EA4991F8560402F042FE07280BD0E64890F844041728C5
:407FC00008D1E44991F8560402F036FE012801D10125C0E0072C14D1DE4991F8560402F02BFE08280BD0DB4890F84404172808D1D84991F8560402F01FFE012801D101252A
:40800000A9E0022C1ED1D34890F85308022819D0D04890F85308032814D0CE4991F8560402F00AFE09280BD0CA4890F84404172808D1C84991F8560402F0FEFD012801D1A9
:40804000012588E00A2C14D1C24991F8560402F0F3FD0B280BD0BF4890F84404172808D1BC4991F8560402F0E7FD012801D1012571E0032C14D1B74991F8560402F0DCFD98
:408080000A280BD0B34890F84404172808D1B14991F8560402F0D0FD012801D101255AE0122C14D1AB4991F8560402F0C5FD19280BD0A84890F84404172808D1A54991F8C0
:4080C000560402F0B9FD012801D1012543E0102C14D1A04991F8560402F0AEFD16280BD09C4890F84404172808D19A4991F8560402F0A2FD012801D101252CE00E2C14D128
:40810000944991F8560402F097FD14280BD0914890F84404172808D18E4991F8560402F08BFD012801D1012515E0142C13D1894991F8560402F080FD1C280BD0854890F81B
:408140004404172807D1834991F8560402F074FD012800D10125284670BD10B5012402F078FD00B10024204610BD70B504460E460025FFF7F2FF00284BD002F0D6F850B1A7
:408180000B2C06D0734890F840040B2841D1062C3FD101253DE0D6B9012C03D0092C01D0062C08D12046FFF7A2FE054615B30020694948702DE068484078D8B12046FFF7CE
:4081C00096FE0546B5B100206349487021E06248407878B1012C05D0092C03D0062C01D00C2C08D12046FFF782FE054615B10120594948700DE002F01DFE10B9FFF770FE7D
:4082000038B92046FFF773FE054615B1012052494870012D04D1FFF763FE08B1FEF7D6FD284670BD03B58FB000200E900F9800287AD0F220012102220023CDE90532CDE999
:408240000710042010210193CDE90231049097201A46194600900AA838F06DFA0AA90F9837F037FE0C900C9800F0F2000C900F9838F0A9FC0D900C98F2280ED10D98022849
:408280000BD10E9848B90B201099FFF76EFF20B10B20FEF78EFD01200E90F220012102220023CDE90532CDE9071010220193CDE9023297201A461946049300900AA838F06D
:4082C0003AFA0AA90F9837F004FE0C900C9800F0F2000C900F9838F076FC0D900C98F2280FD10D9801280CD10E9850B909201099FFF73BFF28B10920FEF75BFD01200E9023
:4083000024E00C98F22810D10D9802280DD10E9858B901201099FFF728FF30B10120FEF748FD01200E9011E0D3E10C98F2280DD10D9858B90E9848B906201099FFF715FFDD
:4083400020B10620FEF735FD01200E909A200121022203E0602A0020F50000200023CDE90532CDE9071051210193CDE9023197201A461946049300900AA838F0DCF90AA9B3
:408380000F9837F0A6FD0C900C9800F09A000C900C989A280BD10E9848B910201099FFF7E4FE20B11020FEF704FD01200E909620012100220592CDE90621089010210192CC
:4083C000CDE90221392013461146049200900AA838F0B1F90AA90F9837F07BFD0C900C9800F096000C900C9896280BD10E9848B904201099FFF7B9FE20B10420FEF7D9FC78
:4084000001200E9096210122002305931846CDE90632089110211A460123CDE90132CDE90310392000231A46194600900AA838F082F90AA90F9837F04CFD0C900C9800F082
:4084400096000C900C9896280BD10E9848B907201099FFF78AFE20B10720FEF7AAFC01200E909220012102220023CDE90532CDE9071086210193CDE9023121201A4619464C
:40848000049300900AA838F056F90AA90F9837F020FD0C900C9800F092000C900C9892280BD10E9848B902201099FFF75EFE20B10220FEF77EFC01200E909A20012202234F
:4084C0000021CDE90632059108900846862219460023CDE90131CDE9032066201A46194600900AA838F027F90AA90F9837F0F1FC0C900C9800F09A000C900C989A280BD121
:408500000E9848B903201099FFF72FFE20B10320FEF74FFC01200E909E20012202210023CDE90531CDE9072086210193CDE9023166201A461946049300900AA838F0FBF865
:408540000AA90F9837F0C5FC0C900C9800F09E000C900C989E280BD10E9848B90A201099FFF703FE20B10A20FEF723FC01200E909A20012102220023CDE90532CDE90710ED
:4085800086220193CDE902325E201A461946049300900AA838F0CFF80AA90F9837F099FC0C900C9800F09A000C900C989A280BD10E9848B912201099FFF7D7FD20B1122083
:4085C000FEF7F7FB01200E90B221012202200023CDE90530CDE907211146842201939720CDE90232049100901A4619460AA838F0A2F80AA90F9837F06CFC0C900C9800F02E
:40860000B2000C900C98B2280BD10E9848B90C201099FFF7AAFD20B10C20FEF7CAFB01200E90BA2000220221CDE90521CDE90720012010210023CDE90130CDE90310662080
:40864000194600900AA838F076F80AA90F9837F040FC0C900C9800F0BA000C900C98BA280BD10E9848B90E201099FFF77EFD20B10E20FEF79EFB01200E90B22001210222CB
:408680000023CDE90532CDE9071086210193CDE902316F201A461946049300900AA838F04AF80AA90F9837F014FC0C900C9800F0B2000C900C98B2280BD10E9848B91420E4
:4086C0001099FFF752FD20B11420FEF772FB01200E900E9810B18020EFF757FF0E9811B000BDF84800780C2801D1012070470020FCE7F4480078102801D1012070470020B0
:40870000FCE7F0480078082801D1012070470020FCE7EC4800780F2801D1012070470020FCE7E8480078032801D1012070470020FCE7E44800780A2801D101207047002019
:40874000FCE7E0480078042801D1012070470020FCE7DC480078072801D1012070470020FCE7D8480078132801D1012070470020FCE710B5D4484EF0D6FB0121D348006810
:4087800038F0EDF910BD10B5CF484EF0A4FC0121CF48006838F0E3F910BD10B5CD481BF05CFA0121CC48006838F0D9F910BDC54800787047C94890F824007047C74890F8CB
:4087C000260008B1012070470020FCE7C4487047F0B504460D460027C24890F84C6490F8561490F85308022804D0BE4890F85308032802D1212900D1042634B1012C0FD061
:40880000022C16D0032C26D11CE035204843DFF8D8C20CEB00103C3000EB861002781CE035204843DFF8C0C20CEB001090F87C2113E035204843DFF8B0C20CEB001090F837
:408840007D210AE035204843DFF89CC20CEB001090F87E2101E0FF2200BF00BF35B1012D0FD0022D16D0032D26D11CE035204843DFF874C20CEB00103C3000EB8610037826
:408880001CE035204843DFF860C20CEB001090F87C3113E035204843DFF84CC20CEB001090F87D310AE035204843DFF83CC20CEB001090F87E3101E0FF2300BF00BFFF2A2B
:4088C0001BD0FF2B19D0002015E0DFF820C20CEB800C1CF804C0944509D1DFF810C20CEB800C1CF805C09C4501D1012705E000F1010C0CF0FF001E28E7DB3846F0BD10B5E8
:40890000784890F84404122805D100221346D721774838F009F910BD10B503F07EF840B9FFF783F928B9FEF75BFD10B901F09CFD08B1012000E000200446204610BD6D4947
:40894000097801436B4A117070472DE9F04781460C4692461D46DDF8208067480068C078A84240D100232022644920464AF047F818B920216148ABF02AF9012320225F496D
:40898000203120464AF03BF820B920215B482030ABF01DF9022320225849403120464AF02EF820B9202155484030ABF010F9032320225249603120464AF021F828B920215C
:4089C0004E486030ABF003F90AE010214B48603008F065FB06469BF089FD0120FFF7AFFF5220EFF7D2FDBDE8F0872DE9F04107460C4690461D46069E3F480068C078A842EB
:408A00005ED1002320223E4920464AF066F818B920213B48ABF0DBF8012320223849203120464AF05AF820B9202135482030ABF0CEF8022320223249403120464AF04DF870
:408A400020B920212E484030ABF0C1F8032320222B49603120464AF040F820B9202128486030ABF0B4F8042320222549803120464AF033F820B9202121488030ABF0A7F83C
:408A8000052320221E49A03120464AF026F820B920211B48A030ABF09AF8062320221849C03120464AF019F820B920211448C030ABF08DF80220FFF742FF5220EFF765FDD5
:408AC000BDE8F081F5000020986C0220CC020020D0020020604F0010D8020020141B0010E81A0010602A0020C0E60C0866E00C08D85C022001010020C80200209A1D001054
:408B00001A1E00100B480078704710B501F00DFC18B1094890F84E0408B1012010BD0020FCE70648006890F8200008B9012070470020FCE700010020602A0020DC0200204B
:408B40000146002009B9012000E0002070472DE9F04106460C4690461D46069FE1488078A8424BD0A6F57040223868B3A0F6266010B1012840D113E059F074FDDA490860FC
:408B80002078617840EA0120D749886008464571E17901F00300FFF7D3FFD34908742CE059F060FDD14908602078617840EA0120CE49886008464571E17901F00300FFF708
:408BC000BFFFCA49087418E059F04CFDC84908602078617840EA0120C549886008464571E079C0F382000871E17901F00300FFF7A7FFBF49087400E000BF00BFBDE8F08186
:408C00000720BC4A9268B2F57B4F01DA092073E0B74A12790B2A1CD2DFE802F00D061415161B1B1718191A00B14A9268B2F57B4F00DA0A200DE0AE4A9268B2F57B4F00DA5F
:408C40000A2006E000BF00BF00BF00BF00BF00BF00BF00BF07284FD1A34A9268B2F57B4F06DAA24A9268B2F57B4F01DB002043E09D4A9268B2F57B4F06DB9C4A9268B2F535
:408C80007B4F01DA012037E0974A9268B2F57B4F06DB964A9268B2F57B4F01DB07202BE0914A9268B2F57B4F26DA904A9268B2F57B4F21DA8C4A92ED020AB8EEC00ADFED2E
:408CC0008E0A20EE200ABDEEC00A10EE101A92680AB9002010E0854A9268834B9B685B1A9A4208DD814A92687F4B9B680B449A4201DA012000E0002070472DE9F0412DED99
:408D0000028B0446FF2559F0ADFC06469FED7B0AB0EE408A02270B2C4CD2DFE804F037284648494B4B474A06150072484579066890ED020AB8EEC00ADFED710A80EE201A02
:408D4000B0EE418A077C35E06948007902280DD067484579066890ED020AB8EEC00ADFED680A80EE201AB0EE418A077C22E05F484579066890ED020AB8EEC00ADFED600A17
:408D800080EE201AB0EE418A077C13E056484579066890ED020AB8EEC00ADFED590A80EE201AB0EE418A077C04E000BF00BF00BF00BF00BF00BF53480471457106600774A1
:408DC0000146086840F2DC5159F069FC70B1FF204C4948710720087159F044FC494908609FED460AB0EE408A0220087401214648B0EE480A1CF006FF424880ED030A02F075
:408E00007EFC90B13F48007C012805D1FBF750FD0120FBF7B6F808E03A48007C28B90020FBF746FD0120FBF7ACF8BDEC028BBDE8F08110B52C49086840F2DC5159F02FFCD9
:408E400018B14FF6FF70284988602849086840F2DC5159F024FC18B14FF6FF70234988602349086840F2DC5159F019FC18B14FF6FF701F4988601F49086840F2DC5159F0BC
:408E80000EFC18B14FF6FF701A498860FFF7B8FE0446FFF732FF10BD10B5164C60712360A160227410BD174890ED030A704710B514211448AAF0ADFE14210C48AAF0A9FE12
:408EC00014210948AAF0A5FE14210948AAF0A1FE14210848AAF09DFEFF210B481CF0E6FE10BD0000586702205422001040220010682200107C220010CDCCCC3E0000000042
:408F000000007A442C220010FC1E001038B504460020FE490880FE4908809FEDFE0AFE4880ED000A0020FD490870FD4890F85604352110FB01F0FB4901EB001090F87C0109
:408F400069460090F8484DF015FFF54890F85604352110FB01F0F34901EB001090F87D0169460090F0484EF063F8ED4890F85604352110FB01F0EB4901EB001090F87E01C2
:408F800069460090E9481AF017FE38BD70B5E44890F8564490F84C54352114FB01F1E14A02EB011101F5157101EB45110888002211464AF0E8FF352114FB01F1D94A02EBC2
:408FC000011101F5157101EB45114888002211464BF081F8352114FB01F1D24A02EB011101F5157101EB4511888800214BF0D6F9352114FB01F1CB4A02EB011101F5157152
:4090000001EB4511C88800214BF005FA352114FB01F1C44A02EB011101F5157101EB4511088900214BF010FC352114FB01F1BD4A02EB011101F5157101EB451148894BF001
:4090400027FA352114FB01F1B64A02EB011101F5157101EB451188894BF050FA352114FB01F1B04A02EB011101F5157101EB4511887B4BF079FA352114FB01F1A94A02EB2F
:40908000011101F5157101EB4511087C4BF0D4FA352114FB01F1A34A02EB011101F5157101EB4511C87B4BF093FA352114FB01F19C4A02EB011101F5157101EB4511487C89
:4090C00000214AF0A3FD352114FB01F1954A02EB011101F5157101EB4511887C00214BF0DFFA002108469CF045FA002108469CF05BFA002108469CF009FA0A2049F0C4FF9B
:409100000A2049F0F0FF70BD33B581B00C460025834890F84C0403280CD0814890F84C04042804D17E4890F84D041B2802D0FFF7D8FAA8B100BF012201A97D4800684D30C9
:4091400006F09DF920B99DF80410754880F84D1400BFCB20EFF719FA31203EF003FC5CE0BCB9FDF7ADFB40B9FDF793FB28B9FDF7A0FB10B9FDF795FB58B16E4800680090EE
:409180006D489DF80420032103686C4843F06AFE43E0FCB168480068C078A0421AD0FDF78FFB58B9FDF775FB40B9FDF782FB28B9FDF777FB10B9FDF76CFB58B15D48006899
:4091C00000905D489DF80420032103685B4843F049FE22E0FDF774FB40B9FDF75AFB28B9FDF767FB10B9FDF75CFBB0B152480068C078A04211D100BF012201A94C480068FC
:409200004D3006F03CF920B99DF80410444880F84D1400BFCB20EFF7B8F928463EBD31B5002400BF012269464148006800F2454006F025F920B99DF80010394880F845180A
:4092400000BF204638BD70B5354890F8565490F84C44352115FB01F1324A02EB011101F53D7104EB440211F81200FFF7D8FF352115FB01F12B4A02EB011101F53D7104EBF5
:40928000440201EB42014878012144F013F8352115FB01F1234A02EB011101F53D7104EB440201EB42018878002144F003F8002652E01B4890F84004072815D100223146C7
:4092C00010469FED1F0AA0F0C9FA0022314610469FED100AA0F098F90022314610469FED190A9FF07CFC35E00022314610469FED160AA0F0B3FA0022314610469FED050A3E
:40930000A0F082F90022314610461FE02601002028010020000000002C01002030010020602A0020C0E60C08986C0220604F001020010010DC020020C80200208C00080010
:409340009E9240BF9E92403FF966DFBE9FEDFB0A9FF045FC701CC6B2032EAADB032C01D0042C24D135216943F54A02EB011101F2123111F8340000219BF081FF35216943F2
:40938000EF4A02EB011101F2123101EBC401487800219AF03CF835216943E94A02EB01113C3101EB841108780021FFF7ADFE70BD2DE9F04104460F4632F059F8804672F0DD
:4093C00092F9E04890F8565490F84C64352115FB01F1DB4A02EB011101F5C07106EBC60201EB8201891C085D3A46214605F054FA352115FB01F1D24A02EB011101F5C071B7
:4094000006EBC60201EB8201091D085D3A46214605F080FA352115FB01F1C94A02EB011101F5C07106EBC60201EB8201891D085D3A46214605F0EAFA352115FB01F1C04A3D
:4094400002EB011101F5C07106EBC60201EB82010831085D3A46214605F09AFA352115FB01F1B74A02EB011101F5C07106EBC60201EB82010A31085D3A46214605F004FB6E
:40948000352115FB01F1AE4A02EB011101F5C07106EBC60201EB82010C31085D3A46214605F030FB352115FB01F1A54A02EB011101F5C07106EBC60201EB82010E31085D2C
:4094C0003A46214605F05CFB352115FB01F19C4A02EB011101F5C07106EBC60201EB82011031085D3A46214605F093FB352115FB01F1934A02EB011101F5C07106EBC60289
:4095000001EB8201085D3A46214605F076F9352115FB01F18A4A02EB011101F50D7106EB460201EB4201891C31F8141008B23A462146FCF7C1FC352015FB00F0804901EBB8
:40954000001000F5C07006EBC60100EB8100143000EB8400D0ED000AB0EE600A204604F091FF352115FB01F1754A02EB011101F5C07106EBC60201EB820191ED070ABCEE88
:40958000C00A10EE101A88B205F088FD352115FB01F16B4A02EB011101F50D7106EB460231F8121008B2FCF755FC0320FCF7F6FC0220FCF7C4FC0020FCF71FFD0020FCF7E4
:4095C000D8FD0120FCF70AFEBDE8F0812DE9F84304460F46FDF774F940B9FDF75AF928B9FDF767F910B9FDF75CF9B0B1FDF751F998B9554800680090544803221146036884
:40960000534843F02FFC4F4890F84C04042803D100210120A1F0BDFB81E04A4890F8565490F84C6490F8900408B1012000E000208046B8F1000F0DD04649C85D0022394634
:409640009EF0E9F94349891CC85D002239469EF088FA1BE035216943394A02EB01113C3101EB86110A31085D002239469EF0D3F935216943324A02EB01113C3101EB8611FC
:409680000C31085D002239469EF06BFA352169432B4A02EB01113C3101EB8611091D085D00233A4621469DF0E7FA35216943244A02EB01113C3101EB8611891D085D00237E
:4096C0003A4621469DF027FC352169431C4A02EB01113C3101EB86110831085D00233A4621469DF0D9FC35216943154A02EB01113C3101EB8611491C085D00233A4621464E
:409700009DF0E9F9352169430D4A02EB01113C3101EB8611C87800219DF05BFB00BFBDE8F88370B504460D4629462046FFF74EFF29462046FFF73CFE70BD0000F966DF3EC7
:40974000C0E60C08602A0020DC020020C802002072000800EC2E002070B500240BE0002505E029462046FFF723FE681CC5B2022DF7DB601CC4B2022CF1DB70BDF8B5FDF709
:409780009FF840B9FDF785F828B9FDF792F810B9FDF787F8B0B1FDF77CF898B9FB4800680090FB48032211460368FA4843F05AFBF94890F84C04042841D100210120A1F09A
:4097C000E8FA3CE0F44890F8566490F84C74002419E0002505E029462046FFF7F7FE681CC5B2022DF7DB35217143EC4A02EB01113C3101EB87112431085D00222146A1F0BE
:4098000031FC601CC4B2022CE3DB35207043E34901EB00103C3000EB8710D0ED080AB0EE600A00209EF051FB9EF0E5F800210846A1F0AFFA002108469FF05DF800BFF8BD53
:4098400010B5FFF79BFFFFF787FF10BD08B5FDF720F890B1CD4800680090CD48042203210368CC4843F0FEFACB4890F84C04042803D100210120A1F08CFA08BDF8B504462A
:40988000FDF71EF840B9FDF704F828B9FDF711F810B9FDF706F868B1FCF7FBFF50B9BB4800680090BA48012203210368B94843F0D9FA9EE0B84890F8565490F84C6490F8E7
:4098C000900408B1012000E000200746002120469FEDB30A9DF08BFD002120469FEDB10A9DF088FF7FB3B04800EB8400D0ED000AB0EE600A002120469DF090FCAA481030AC
:4099000000EB8400D0ED000AB0EE600A002120469DF06DFDA448083000EB8400D0ED000AB0EE600A002120469DF07BFE9E48183000EB8400D0ED000AB0EE600A0021204689
:409940009DF058FF54E0FFE735206843934901EB00103C3000EB86100E3030F9140000EE900AF8EEE00AB0EE600A002120469DF055FC35206843894901EB00103C3000EBBF
:409980008610163030F9140000EE900AF8EEE00AB0EE600A002120469DF029FD352068437E4901EB00103C3000EB8610123030F9140000EE900AF8EEE00AB0EE600A002144
:4099C00020469DF02EFE35206843744901EB00103C3000EB86101A3030F9140000EE900AF8EEE00AB0EE600A002120469DF002FF00BFF8BD38B5FCF763FF40B9FCF749FFBC
:409A000028B9FCF756FF10B9FCF74BFF68B1FCF740FF50B95D48006800905D480122032103685C4843F01EFA08E0002404E02046FFF724FF601CC4B2022CF8DB38BD2DE953
:409A4000F0415548B0F82278B0F82448B0F82658B0F82868B0F8348890F840040A2828D1A74207DB002C05DD611E88B2002211464AF089FAAE4204DA691C88B200214AF059
:409A8000CAFCBD4203DA002138464AF087FCA64203DD002120464AF0BEFCB04503DD002130464AF08FFEA84503DA002128464AF089FEBDE8F08110B5012043F0A3FC014603
:409AC0003A4880F83910002043F09CFC37494874012043F097FC04462146012036F0EAF9002043F08FFC04462146002036F0E2F910BD10B5FFF7A7FBFCF7CBFE08B1FFF7F5
:409B0000A5FEFFF79DFEFFF775FFFFF7D4FF01209BF099FB10BD2049B1F85404704700B5FFF7F9FF00EE100AF8EE400A9FED201A80EE810A00BD1849D1F85804704700B547
:409B4000FFF7F9FF00EE100AB8EEC00AF0EE400A1848B0F9000000EE100AB8EEC00A30EE801ADFED131A81EE210A00BD0A48B0F85C041149B1F90010084400EE100AF8EE26
:409B8000C00A9FED0B1A80EE810A7047DC020020C802002072000800602A0020C0E60C080000C8C20000C842CC2E0020186B022000007A442801002026010020FE4890ED50
:409BC000000A704700B5FFF7F9FFFC4890ED181A30EE010AF0EE400AB0EE600A00BD00B5FFF7F0FF1FED0E1AC0EE010AB0EE600A00BD30B502460B460024F148B0F9000028
:409C0000824204D1EF48B0F90000834221D0EC480280EC480380FFF78EFFE949B1F90010E84DB5F90050491B01EB8101490000FB01F5FFF770FF95FBF0F0E249098801EB5D
:409C4000810100EB410000B2DF4908800020DF490880204630BD33B581B00C460025BDF8040041F65831884202DD08460190022500BF022201A9D6480068543005F0FFFB73
:409C800020B9BDF80410D348A0F8541400BF0920EEF77BFC24203DF065FEACB1CE480068C078A04210D0CB4890F84C0403280BD0CA4800680090C848BDF804200321036887
:409CC000C74843F0CFF817E0B4B9FCF7F9FD40B9FCF7DFFD28B9FCF7ECFD10B9FCF7E1FD50B1BE4800680090BB48BDF8042003210368BB4843F0B6F8BA48D0F8981102200C
:409D0000DFF8E4C200DF28463EBD10B52DED028BB0EE408A00249FEDB50AB4EEC08AF1EE10FA04DD9FEDB10AB0EE408A02249FEDB00AB4EEC08AF1EE10FA04D29FEDAC0A5D
:409D4000B0EE408A03249C4880ED008A0C20EEF71CFC2046BDEC028B10BD31B500240098B0F5FA4F04DD4FF4FA400090022406E0009810F5FA4F02DA9E480090032400BF3F
:409D80000422694692480068583005F078FB18B990480099C0F8581400BF0D20EEF7F5FB24203DF0DFFD8F48D0F898110220DFF838C200DF204638BD31B50024BDF80000F4
:409DC00041F65831884202DD08460090022400BF022269467E4800685C3005F050FB20B9BDF800107B48A0F85C1400BF0E20EEF7CCFB24203DF0B6FD204638BD10B52DED0A
:409E0000020B00249DED000ADFED780AB4EEE00AF1EE10FA05DD9FED750A8DED000A02240DE09DED000ADFED720AB4EEE00AF1EE10FA04D29FED6E0A8DED000A032400BF81
:409E40000422694662480068603005F018FB20B99DED000A594880ED180A00BF0C20EEF794FB24203DF07EFD20461CBD31B5002400BF0422694656480068403005F0FFFA3A
:409E800018B954480099C0F8401400BF1020EEF77CFB24203DF066FD204638BD31B5002400BF022269464A480068563005F0E7FA20B99DF800104748A0F8561400BF0F2027
:409EC000EEF763FB7320EEF760FB24203DF04AFD204638BD31B5002400BF042269463C480068443005F0CBFA18B93A480099C0F8441400BF1120EEF748FB24203DF032FDCD
:409F0000204638BD33B581B00C4600259DF8040003282AD100BF012201A92D4800684C3005F0ADFA20B99DF804102A4880F84C1400BF1220EEF729FB31203DF013FD254934
:409F400091F85614352211FB02F12B4A02EB011101F53D711F4A92F84C2402EB420201EB4201487904F037FCE0E01CBBFCF7A8FC40B9FCF78EFC28B9FCF79BFC10B9FCF70A
:409F800090FCB8B100BF012201A9114800684C3005F075FA20B99DF804100E4880F84C1400BF0E48006800900B489DF804200321036823E03BE000002C010020602E00200E
:409FC0003201002034010020260100202801002020010010602A0020C8020020DC02002004FA0700F8FF0020099F0C080000FA460000FAC60083FFFFC0E60C08FA4842F0DF
:40A0000031FFFA4991F85614352211FB02F1F84A02EB011101F53D71F44A92F84C2402EB420201EB4201487904F0D5FB7EE0FCB1F0480068C078A0421AD0FCF741FC58B972
:40A04000FCF727FC40B9FCF734FC28B9FCF729FC10B9FCF71EFC58B1E74800680090E5489DF8042003210368DF4842F0FBFE5DE0FCF726FC40B9FCF70CFC28B9FCF719FCB9
:40A0800010B9FCF70EFC60B3DA480068C078A04227D100BF012201A9D84800684C3005F0EEF920B99DF80410D04880F84C1400BFCE4991F85614352211FB02F1CC4A02EB2B
:40A0C000011101F53D71C94A92F84C2402EB420201EB4201487904F07EFB1220EEF755FA24E01CBB00BF012201A9C44800684C3005F0C5F920B99DF80410BC4880F84C1441
:40A1000000BFBA4991F85614352211FB02F1B84A02EB011101F53D71B44A92F84C2402EB420201EB4201487904F055FB28463EBD31B5002400BF01226946B048006800F2BC
:40A140003E4005F09CF920B99DF80010A74880F83E1800BF204638BD31B5002400BF01226946A648006800F23F4005F088F920B99DF800109D4880F83F1800BF204638BD5E
:40A1800001460020704710B5044628229C492046A9F05CFC10BD10B5044635216143944A02EB0110FFF7ECFF35216143904A02EB0111887FFFF75AFE352161438C4A02EB74
:40A1C0000111088D0021FFF746FD35216143884A02EB0111C86AFFF7C0FD35216143844A02EB0111088EFFF7E7FD35206043804901EB0010B0F9320000EE900AF8EEE00A87
:40A20000B0EE600AFFF7FAFD35216143784A02EB011191F82000FFF741FE35216143744A02EB0111C87FFFF755FE55F0E8FA18B1022013F04DFC28E056F033F918B1012087
:40A2400013F046FC21E055F0DAFA18B96D480078012803D06B480078032809D135216143634A02EB011191F8350013F031FC0CE064480078022808D1352161435C4A02EB21
:40A28000011191F8340013F023FCFEF77FFE10BD01B500BF012269465848006800F5886005F0EDF820B99DF80010504880F8401800BF08BD31B584B000BF012204A95248BB
:40A2C00005F0DDF820B99DF81000484981F8010100BF464890F8010130B1012806D0022806D0032806D000BF48A405E049A403E04BA401E04CA400BF00BF2046A9F030FB8A
:40A30000401CC5B201202323002211468DE8310047488EF04DFB05B030BD0020334991F84414202900D101207047304890F8401490F85624082907D0092905D0712A03D08B
:40A340000A2901D00E2901D1012070470020FCE7264890F8401490F85624082905D0092903D0712A01D00E2901D1012070470020FCE71E4890F840140A2901D1012070472F
:40A380000020FCE7194890F84014082901D1012070470020FCE7154890F8401490F85624092901D0712A01D1012070470020FCE70E4890F840140E2901D1012070470020C6
:40A3C000FCE70020094991F85614432909D0074991F85614452904D0044991F85614472900D101207047000056010800602A0020C0E60C08C8020020DC0200202001001016
:40A40000782E0020300500100101006874726163746F7200696D706C656D656E7400000066656E64740000006D61737365790000BCDD00100020FE4991F85614422909D0F3
:40A44000FB4991F85614442904D0F94991F85614462900D1012070470020F54991F85614412900D10120704710B50024F04890F84C04032809D0EE4890F84C04042818D193
:40A48000EB4890F84D041B2813D1E94890F84404022809D0E64890F844040C2804D0E44890F844040A2804D1E24845F0BFFA00B10124204610BD70B504460025DE48007809
:40A4C00084421DD0032C02D1DB48047014E0012C01DD022510E02246D8A1DD488FF038FCD5480470DB48D0F898110220DFF868C300DF0020D94908704FF48570EEF745F805
:40A50000284670BDCC480078032813D1D448007808280DD2DFE800F004070C0C08090A0500BF0020704700BF00BF00BF0120F9E70020F7E7C0480078F4E770B50446002587
:40A54000C7480078844221D0BB480078032819D1082C01DD022510E02246B8A1BC488FF0F7FBBF480470BB48D0F898110220DFF8E8C200DF0020B94908704FF48570EEF786
:40A5800004F803E0FF20B64908700725284670BDB3480078704733B581B00D4600249DF80400012802DD012001900224A04890F8A8059DF8041088420FD000BF012201A931
:40A5C000A848006800F5D47004F059FF20B99DF80410974880F8A81500BFA020EDF7D5FF9C48D0F898110220DFF86CC200DF04F04EFB9848D0F870120120DFF85CC200DFFA
:40A600009DF086FD9348016E0220DFF84CC200DFFAF796FE94480068009094489DF8042003210368924842F01DFC3120EDF7ADFF20463EBD7E4890F85604352110FB01F0FC
:40A640008C4901EB0010408C7047794890F85604352110FB01F0874901EB0010808C704770B50124844885490978455C83480078A12822DA81480078A5281EDA35216943EC
:40A680007C4B03EB01123521694303EB0111888C1E2132F000FF044024B178480078401C7649087001207649087040F2C92073F0DAF8552073F0D7F807E001206F490870F1
:40A6C0007049087000206E490870204670BD70B501246D480078282832DA6B48007823282EDA6949097801EB0111684A02EB4101081DA9F035F985B26349097801EB011196
:40A70000624B03EB41010A1D5F49097801EB011103EB41014888294632F0BDFE044024B159480078401C5849087001205449087040F2C92073F097F8562073F094F807E06C
:40A740000120514908705249087000204C490870204670BD70B504460125354890F840040B2802D0FFF7E1FD08B101251CE055F086FE38B1022C05D00C2C03D00A2C01D07A
:40A78000002511E055F084FE18B1012C01D000250AE055F054FE18B1012C01D0002503E055F055FE00B10025284670BD70B5012674F093FD002871D03648007800286ED171
:40A7C00048F6426034490880012005E04FF6FF71314A22F81010401C2328F7DB0024E2E035206043234901EB001090F8F40203287DD03520604301EB001090F8F4020228B3
:40A8000075D03520604301EB001090F8FA0203286DD03520604301EB001090F8FA02022865D03520604301EB001090F8000337E0602A00201862022030010020537465655E
:40A8400072696E67206D6F646520256400000000BCDD0010F8FF0020099F0C08381600103101002020010010DC020020C802002058010800C0E60C08F4E00C08240100202D
:40A88000D1140010D3140010250100209AE10C08D214001036010020E0220020C2E08AE0032851D03520604301EB001090F80003022849D03520604301EB001090F80603C9
:40A8C000032841D03520604301EB001090F80603022839D03520604301EB001090F80C03032831D03520604301EB001000E02BE090F80C03022827D00EF0F1F9002851D0E5
:40A9000035206043F74901EB001090F8F402D8B93520604301EB001090F8FA02A0B93520604301EB001090F8000368B93520604301EB001090F8060330B93520604301EB11
:40A94000001090F80C0348B3E74890F8401435206043E44A02EB0010807F814222D101251EE035206043DF4901EB0010C07F05EB0511DE4A12F81110884210D105EB0511C9
:40A9800012F81100FFF7E6FE48B105EB0510D74901EB40004088D64921F8150002E06D1C232DDEDB641CB82CFFF61AAF0120D1490870D1490870CF48007828282CDCCC486D
:40A9C000CC49097830F811004FF6FF71884210D0C848007823280CDAC548C649097830F81120C448017842F21E7032F0C4FB064008E04FF6FF72BF48017842F21E7032F00A
:40AA0000BAFB064026B1BB480078401CB9490870542072F028FF05E00120B64908700020B549087001208CF0F6F940F25B2072F01AFF304670BD70B5B048B1490978445C54
:40AA40000125002142F21F7031F09FF8054000208CF0E1F974F041FC00287DD0A8480078A1287ADCA6480078A52878DA9E4890F84414352060439B4A02EB0010C07F814295
:40AA80006DD1994890F840143520604302EB0010807F814263D10EF022F938B335206043904901EB001090F8F402002874D13520604301EB001090F8FA0200286CD13520C2
:40AAC000604301EB001090F80003002864D13520604301EB001090F8060300285CD13520604301EB001090F80C03B8BB352060437C4901EB001090F8F40203284CD0352024
:40AB0000604301EB001090F8F402022844D03520604301EB001090F8FA0203283CD03520604301EB001090F8FA02022834D03520604301EB001090F8000303282CD035206A
:40AB4000604301EB001090F80003022824D03520604301EB001003E06CE045E01CE029E090F80603032817D03520604301EB001090F8060302280FD03520604301EB00101B
:40AB800090F80C03032807D03520604301EB001090F80C0302280DD135206043514901EB0010428C5648017842F21F7032F0E3FA054008E04FF6FF725148017842F21F707C
:40ABC00032F0D9FA054025B14D480078401C4C49087001204B49087040F2C92072F043FE532072F040FE25E001204549087000204449087040F2C92072F035FE3A4890F8C6
:40AC0000440420B1384890F84404172809D1002142F21F7030F0B9FF054000208CF0FBF808E0012142F21F7030F0AFFF054001208CF0F1F8284670BD014635204843294A67
:40AC400002EB001090F8FC00704701207047002070470020244991F84414102900D1012070470020204A92F856143C2907D0A02905D0AE2903D0942901D0AF2900D1012043
:40AC800070470020184991F844141F2900D1012070470020144991F85614822900D1012070470020104991F844141E2900D10120704700200C4991F85614142901D10121E3
:40ACC00000E00021084A92F85624152A01D1012200E000221143044A92F85624162A13D1012212E0C0E60C08602A00209AE10C08E02200202501002036010020F4E00C084E
:40AD000024010020D114001000221143FE4A92F85624172A01D1012200E000221143FA4A92F85624182A01D1012200E000221143F54A92F85624192A01D1012200E0002239
:40AD4000114301B1012070470020EF4991F84014042905D1EC4991F84414022900D1012070470020E84991F84014042905D1E64991F844140C2900D1012070470020E24969
:40AD800091F84414112900D1012070470020DE4991F85614652913D0DB4991F8561466290ED0D94991F85614672909D0D64991F85614682904D0D44991F85614692900D138
:40ADC000012070470020D04991F84414152900D1012070470020CC4991F844140F2900D1012070470020C84991F84414122900D1012070470020C44991F84414132900D172
:40AE0000012070470020C04991F84414162900D1012070470020BC4991F856146A2900D1012070470020B84991F856148F2900D1012070470020B44991F85614522909D01B
:40AE4000B14991F856141F2904D0AF4991F85614822900D101207047002070470020AA4991F85614952900D1012070470020A64991F84414222900D1012070470020A24957
:40AE800091F84014112900D101207047014601EB01109E4A12F8100070470246012109E001EB0110994B13F81000904201D1C8B27047491C2329F3DB0020F9E72DE9F041EB
:40AEC0000124914991F84404FFF7E7FF00EB00108E4901EB4000051D8B4991F84404FFF7DCFF00EB0010894901EB4000071D3846A8F036FD86B22A46314649F2FC1032F022
:40AF0000CAFA04462046BDE8F08170B57E4890F8564490F84C540A20DFF8F4C100DF352114FB01F17B4A02EB011101F2123101EBC5014878002198F06AFA0A20DFF8D0C15B
:40AF400000DF00209FED740A97F030FF0A20DFF8C0C100DF352114FB01F16E4A02EB01113C3101EB851108780021FEF7CDF80A20DFF89CC100DF352014FB00F0654901EB2E
:40AF800000103C3000EB8510B0F90E0000EE900AF8EEE00AB0EE600A002108469CF03EF90A20DFF86CC100DF352014FB00F0594901EB00103C3000EB8510B0F9160000EEB4
:40AFC000900AF8EEE00AB0EE600A002108469CF00EFA0A20DFF838C100DF352014FB00F04C4901EB00103C3000EB8510B0F9120000EE900AF8EEE00AB0EE600A00210846A8
:40B000009CF00FFB0A20DFF808C100DF352014FB00F0404901EB00103C3000EB8510B0F91A0000EE900AF8EEE00AB0EE600A002108469CF0DFFB0A20DFF8D4C000DF35214A
:40B0400014FB01F1334A02EB01113C3101EB8511087900231A4619469BF00EFE0A20DFF8B0C000DF352114FB01F12A4A02EB01113C3101EB8511887900231A4619469BF0F3
:40B080004AFF0A20DFF888C000DF352114FB01F1204A02EB01113C3101EB8511087A00231A4619469BF0F8FF0A20DFF864C000DF352114FB01F1174A02EB01113C3101EB76
:40B0C0008511C87800219BF084FE0A20DFF840C000DF9CF090FC0A20DFF834C000DF352114FB01F10B4A02EB01113C3101EB8511887A002211469CF08EFC0A20DFF810C084
:40B1000000DF35210AE00000602A00209AE10C08A99E0C08C0E60C080000000014FB01F1FE4A02EB01113C3101EB8511087B002211469CF016FD0A20DFF8E4C300DF3521F3
:40B1400014FB01F1F54A02EB01113C3101EB8511487800231A4619469BF0BDFC0A20DFF8C0C300DF352014FB00F0EC4901EB00103C3000EB8510D0ED080AB0EE600A0020F0
:40B180009CF0A3FE0A20DFF898C300DFFFF7BAF9064600219FEDE30A9EF017FC0A20DFF880C300DFFFF7AEF9064600219FEDDE0A9DF02AFF0A20DFF868C300DF352114FB30
:40B1C00001F1D64A02EB0111088D0021FEF743FD0A20DFF84CC300DF70BD10B50124D3480078152829DAD148007800EB4000D04901EB4000007970B1CC48007800EB400028
:40B2000001EB40004288C948017842F2217031F0B2FF044008E04FF6FF72C448017842F2217031F0A8FF0440C0480078401CBF4908704B2072F017FB02E00020BB49087006
:40B24000204610BD33B581B00D4600249DF80400012802DD012001900224B64890F8A9059DF8041088420FD000BF012201A9B248006800F2A91004F002F920B99DF8041002
:40B28000AC4880F8A91500BFCA20EDF77EF9AB48D0F898110220DFF8A8C200DF03F0F7FCA648D0F870120120DFF894C200DF9CF02FFFA248016E0220DFF884C200DFFAF74D
:40B2C0003FF8A048006800909F489DF80420032103689E4841F0C6FD20463EBD01B5954890F842069DF8001088420FD000BF012269469148006800F2422004F0C0F820B971
:40B300009DF800108B4880F8421600BF40F21510EDF73BF908BD01B500BF012269468648006800F2432004F0AAF820B99DF80010804880F8431600BF08BDF8B5FBF7C0FA76
:40B3400040B9FBF7A6FA28B9FBF7B3FA10B9FBF7A8FA58B17B48006800907B4803221146036840F2762041F07DFD88E0714890F8564490F84C5400267DE0352060436749EE
:40B3800001EB00103C3000EB85100E30694991F8A81530F9110000EE900AF8EEE00AB0EE600A304692F01DFB352060435B4901EB00103C3000EB851012305E4991F8A81512
:40B3C00030F9110000EE900AF8EEE00AB0EE600A304692F01EFB35206043504901EB00103C3000EB85101630524991F8A81530F9110000EE900AF8EEE00AB0EE600A3046F2
:40B4000093F037FB35206043444901EB00103C3000EB85101A30474991F8A81530F9110000EE900AF8EEE00AB0EE600A304693F007FB35216143394A02EB01113C3101EB60
:40B4400085110A313B4A92F8A825885C314693F0E4FA35216143314A02EB01113C3101EB85110C31334A92F8A825885C314693F0C2FA701CC6B2022EFFF67FAF00BFF8BD8A
:40B4800010B52DED020B002400BF042269462A48006800F24C4003F0F2FF20B99DED000A2B4880ED130A00BFCD20EDF76EF820461CBD10B50024FEF738FF08B101240AE030
:40B4C000FEF7CAFF08B1022405E0FFF7B3FC08B1032400E000242046FEF7DAFE10BD33B581B00C460025134890F84C04032809D0104890F84C04042838D10E4890F84D04E6
:40B500001B2833D100BF022201A90B48006800F24A4003F0B4FF08BB01981BE0C0E60C08A99E0C08B81E05BFB81E053F3701002040E60C08602A002020010010F8FF0020B6
:40B54000099F0C08DC020020C8020020EF0108006032002081B2FE48A0F84A1800BFE120EDF713F831203CF0FDF971E00CBBFBF7A7F940B9FBF78DF928B9FBF79AF910B99E
:40B58000FBF78FF9A8B10198322802DD3220019004E00198002801DA00200190ED4800680090ED4803680321EC48019A41F05AFC4EE04CB3E8480068C078A04224D0FBF7C6
:40B5C0007FF958B9FBF765F940B9FBF772F928B9FBF767F910B9FBF75CF9A8B10198322802DD3220019004E00198002801DA00200190D84800680090D74803680321D748B5
:40B60000019A41F02FFC23E0FBF75AF940B9FBF740F928B9FBF74DF910B9FBF742F9B8B1CD480068C078A04212D100BF022201A9CB48006800F24A4003F021FF20B90198AC
:40B6400081B2C348A0F84A1800BFE120ECF79DFF28463EBDBE4890F85604622827D0BC4890F85604632822D0B94890F8560490281DD0B74890F85604962818D0B44890F88B
:40B680005604972813D0B24890F8560498280ED0AF4890F856049A2809D0AD4890F856049B2804D0AA4890F856049C2801D1012070470020FCE7A64890F8860520B1A4482F
:40B6C00090F88605012801D1012070470020FCE79F4890F88605022804D09D4890F88605032801D1012070470020FCE7984890F88605042801D1012070470020FCE79448F1
:40B7000090F844041A280ED0914890F85604212809D08F4890F85604592806D18C4890F85308032801D1012070470020FCE72DE9F04104461B2709F062F9FA2803D009F087
:40B740005EF9FB2801D1012000E000206070804890F85654A570280AE070280C2071280E60717B4890F84004A071794890F84464E671300A2072FEF7CEF906466672300A61
:40B78000A072FEF7D8F900F5FA4086B2E672300A2073FEF717FADFED730A30EE200ABCEEC00A10EE100A86B26673300AA0736848B0F85C64E673300A20746B48A7F05CFFC0
:40B7C00005466574280AA074280CE074280E207507F0DBFC607507F0D5FF0546A575280AE075280C2076280E607607F0C7FFA0763846BDE8F08101B500BF0122694658480E
:40B80000006800F2124003F03AFE20B99DF800104F4880F8121800BF4FF48170ECF7B5FE08BD01B500BF012269464D48006800F5267003F024FE20B99DF80010444880F8C6
:40B84000981600BF08BD01B582B09DF80800002871D09DF8080001286DD09DF80800022829D10DF03CFA30B309F0C9F8FA2810D009F0C5F8FB280CD0354890F856043521A8
:40B8800010FB01F0394901EB001090F87C01FF2851D109F0B4F8FA2803D009F0B0F8FB2809D12B4890F85308022844D0284890F8530803283FD09DF8080003285CD109F079
:40B8C0009EF8FA282AD009F09AF8FB2826D0204890F85604352110FB01F0244901EB001090F87C01FF2819D0194890F85604352110FB01F01D4901EB001090F87E01FF28B3
:40B900000CD0134890F85604352110FB01F0174901EB001090F87D01FF280CD109F06FF8FA2803D009F06BF8FB2825D1084890F89806032820D100BF012202A90848006895
:40B9400000F2534003F09BFDA8B99DF808100FE0602A0020DC020020C802002062010800200100100000FA46786F0008C0E60C08354880F8531800BF344800680090324896
:40B9800090F85328324803210368324841F06AFA09F035F8FA2807D009F031F8FB2803D09DF80800FFF73DFFC220ECF7EEFD0EBD254890F85604622818D0234890F85604DD
:40B9C000902813D0204890F8560496280ED01E4890F85604982809D01B4890F856049A2804D0194890F856049C2801D1012070470020FCE7144890F85604632809D012485A
:40BA000090F85604972804D00F4890F856049B2801D1012070470020FCE710B500240A4890F84004022804D00C2803D00D2807D101E000BF00BFFCF77CFE00B1012400E04D
:40BA400000BF00BF204610BD602A0020DC020020C8020020AE04080000280BDB00F01F0201219140FE4A430942F82310BFF34F8FBFF36F8F70471FB50121084690F03DF8C6
:40BA80000121042090F039F80121082090F035F80121102090F031F8002000900190029003460122EF490390104654F03FF8002000900190029003460222EB490390104665
:40BAC00054F034F8002000900190029003460246E6490390052054F029F8002002220123CDE90120009303900346E149062054F01DF8002002220123CDE90120009303906A
:40BB00000346DC49072054F011F8002002220123CDE90120009303900346D749082054F005F8002000900190029001230222D3490390092053F0FAFF00200323CDE9003091
:40BB4000029003460222CE4903900A2053F0EEFF00200121CDE9000103460A46CDE90210C8490B2053F0E2FF002000900190029003460322C4490390112053F0D7FF0020BD
:40BB800000900190029003460322C0490390122053F0CCFF00200323CDE90030029003460222BB490390182053F0C0FF002000900190029003460122B6490390192053F03F
:40BBC000B5FF002000900190029003460122B24903901A2053F0AAFF00200222CDE9000202900346AD4903901B2053F09FFF00200222CDE9000202900346A94903901F2087
:40BC000053F094FF00200222CDE9000202900346A4490390202053F089FF002001210090CDE9010103460A469F490390212053F07DFF002001210090CDE9010103460A460B
:40BC40009A490390242053F071FF00200090019002900346024696490390252053F066FF00200090019002900346024691490390262053F05BFF002001210090CDE9010156
:40BC800003460A468C490390292053F04FFF002000900190029001230222884903902A2053F044FF00200121CDE9000103460A46CDE9021082492D2053F038FF00200090BE
:40BCC00001900290034602227E490390312053F02DFF0020009001900290034602227A490390322053F022FF00200121CDE9000103460A46CDE902107449332053F016FF8C
:40BD000000200121CDE9000103460A46CDE902106F49342053F00AFF00200121CDE9000103460A46CDE902106A49352053F0FEFE00200121CDE9000103460A46CDE9021056
:40BD40006549362053F0F2FE00200121CDE9000103460A46CDE902106049372053F0E6FE00200121CDE9000103460A46CDE902105B49382053F0DAFE002001210090CDE912
:40BD8000010103460A4657490390392053F0CEFE002001210090CDE9010103460A46524903903B2053F0C2FE002001210090CDE9010103460A464D4903903C2053F0B6FEFF
:40BDC00000200121CDE9000103460A46CDE9021047493D2053F0AAFE00200121CDE9000103460A46CDE9021042493E2053F09EFE002001210090CDE90101034602223E4971
:40BE00000390402053F092FE00200090019002900346022239490390412053F087FE00200090019002900346022235490390422053F07CFE002000900190029003460246EA
:40BE400030490390432053F071FE0020009001900290034601222C490390462056E0000080E100E04605001071050010470500105E0500105F05001060050010610500106E
:40BE800048050010790500104E0500108E05001049050010660500106705001068050010690500106A0500106C0500105A0500104A05001082050010720500106F050010D1
:40BEC00073050010640500106505001074050010750500107605001077050010530500105405001055050010560500105705001058050010590500108C0500107C0500107E
:40BF00007D0500108D0500108105001053F00EFE00200222CDE9000202900346FE490390472053F003FE002000900190029003460222FA490390482053F0F8FD0020009026
:40BF40000190029003460222F5490390492053F0EDFD002001210090CDE9010103460A46F04903904A2053F0E1FD00200222CDE9000202900346EC4903904D2053F0D6FD2E
:40BF800000200222CDE9000202900346E74903904E2053F0CBFD002000900190029003460322E3490390512053F0C0FD002000900190029003460322DE490390522053F04D
:40BFC000B5FD002000900190029003460322DA490390532053F0AAFD0021D848007853F02BFD0021D648007853F026FD0021D548007853F021FD0121D348007853F01CFDD2
:40C000000021D248007853F017FD0021D048007853F012FD0021CF48007853F00DFD0121CD48007853F008FD0121CC48007853F003FD0121CA48007853F0FEFC0021C948F3
:40C04000007853F0F9FC0021C748007853F0F4FC0021C648007853F0EFFC1FBD1FB5012108468FF04AFD012104208FF046FD012108208FF042FD012110208FF03EFD00203E
:40C0800000900190029003460122AC490390104653F04CFD002000900190029003460222B3490390104653F041FD002000900190029003460246AF490390052053F036FDC7
:40C0C000002002220123CDE90120009303900346A949062053F02AFD002002220123CDE90120009303900346A449072053F01EFD002002220123CDE9012000930390034642
:40C100009F49082053F012FD0020009001900290012302229B490390092053F007FD00200323CDE90030029003460222964903900A2053F0FBFC00200121CDE90001034658
:40C140000A46CDE902107E490B2053F0EFFC0020009001900290034603228C490390112053F0E4FC00200090019002900346032287490390122053F0D9FC00200323CDE9A0
:40C18000003002900346022282490390182053F0CDFC00200090019002900346012269490390192053F0C2FC002000900190029003460122644903901A2053F0B7FC002021
:40C1C0000222CDE9000202900346734903901B2053F0ACFC00200222CDE90002029003466E4903901F2053F0A1FC00200222CDE90002029003466A490390202053F096FCA1
:40C20000002001210090CDE9010103460A4645490390242053F08AFC002001210090CDE9010103460A464C490390292053F07EFC002000900190029001230222594903900C
:40C240002A2053F073FC00200121CDE9000103460A46CDE9021043492D2053F067FC0020009001900290034602224F490390312053F05CFC00200090019002900346022252
:40C280004A490390322053F051FC00200121CDE9000103460A46CDE902103049332053F045FC00200121CDE9000103460A46CDE902102D49342053F039FC00200121CDE938
:40C2C000000103460A46CDE902102549352053F02DFC00200121CDE9000103460A46CDE902102249362053F021FC00200121CDE9000103460A46CDE902102D49372053F0C8
:40C3000015FC00200121CDE9000103460A46CDE90210284938204FE05B0500104B0500104C0500105A0500105C0500105D050010890500108A0500108B05001046050010DF
:40C340007905001066050010670500108105001087050010880500107205001074050010760500107305001075050010770500107C050010470500105E0500105F0500105C
:40C380006005001061050010480500104E0500108E0500104905001068050010690500106A0500106F0500106405001065050010530500105405001053F0B8FB00200121D7
:40C3C0000090CDE9010103460A46FE490390392053F0ACFB002001210090CDE9010103460A46F94903903B2053F0A0FB002001210090CDE9010103460A46F44903903C20BF
:40C4000053F094FB00200121CDE9000103460A46CDE90210EE493D2053F088FB00200121CDE9000103460A46CDE90210E9493E2053F07CFB002001210090CDE901010346FF
:40C440000222E5490390402053F070FB002000900190029003460122E0490390462053F065FB00200222CDE9000202900346DC490390472053F05AFB002001210090CDE9AF
:40C48000010103460A46D74903904A2053F04EFB00200222CDE9000202900346D24903904D2053F043FB00200222CDE9000202900346CE4903904E2053F038FB00200090B0
:40C4C0000190029003460322C9490390512053F02DFB002000900190029003460322C5490390522053F022FB002000900190029003460322C0490390532053F017FB0021B0
:40C50000BE48007853F098FA0021BD48007853F093FA0021BB48007853F08EFA0121BA48007853F089FA0021AC48007853F084FA0021B648007853F07FFA0021B44800783B
:40C5400053F07AFA0121B348007853F075FA0121B148007853F070FA0121B048007853F06BFA0021AE48007853F066FA0021AD48007853F061FA0021AB48007853F05CFAC0
:40C580001FBD1FB5012108468FF0B7FA012104208FF0B3FA012108208FF0AFFA012110208FF0ABFA0020009001900290034603229E490390012053F0B9FA002000900190BE
:40C5C0000290034603229A490390022053F0AEFA00200090019002900346032295490390104653F0A3FA00200090019002900346032291490390042053F098FA00200222E5
:40C60000CDE900020290034603228C490390052053F08CFA002002220123CDE901200093039003468649062053F080FA002002220123CDE9012000930390034681490720ED
:40C6400053F074FA002002220123CDE901200093039003467C49082053F068FA00200090019002900123022278490390092053F05DFA002000900190029003460246744976
:40C6800003900A2053F052FA00200121CDE9000103460A46CDE9021061490B2053F046FA002001210090CDE9010103460A46594903900C2053F03AFA00200121CDE9000188
:40C6C00003460A46CDE9021052490C2053F02EFA0020009001900290034601224A490390192053F023FA002000900190029003460122444903901A2053F018FA0020022277
:40C700000092CDE901200346524903901B2053F00DFA0020009001900290034602464E4903901C2053F002FA002002220092CDE901200346494903901F2053F0F7F90020DE
:40C7400002220092CDE90120034645490390202053F0ECF900200090019002900346032240490390212053F0E1F90020009001900290034603223C490390242053F0D6F9F0
:40C78000002001210090CDE9010103460A4637490390252053F0CAF9002001210090CDE9010103460A4632490390262053F0BEF90020009001900290034601222D4903903F
:40C7C000272059E055050010560500105705001058050010590500108C050010810500105B0500105A0500105C0500105D050010890500108A0500108B050010460500106C
:40C8000079050010660500106705001087050010880500107205001074050010760500107305001075050010770500104D0500104E0500104F0500105005001084050010DA
:40C840005E0500105F05001060050010610500107B0500106805001086050010690500106A0500106B050010510500106C0500106D0500106E05001053F058F90020009091
:40C880000190029003460122FC490390292053F04DF9002000900190029001230222F84903902A2053F042F9002000900190029003460222F34903902B2053F037F900209B
:40C8C00000900190029003460222EF4903902C2053F02CF9002000900190029003460122EA490390312053F021F9002001210090CDE9010103460A46E5490390322053F06D
:40C9000015F900200121CDE9000103460A46CDE90210E049332053F009F900200121CDE9000103460A46CDE90210DB49342053F0FDF800200121CDE9000103460A46CDE97C
:40C940000210D649352053F0F1F800200121CDE9000103460A46CDE90210D149362053F0E5F800200121CDE9000103460A46CDE90210CC49372053F0D9F800200121CDE949
:40C98000000103460A46CDE90210C749382053F0CDF8002001210090CDE9010103460A46C2490390392053F0C1F8002000900190029003460122BE4903903A2053F0B6F86B
:40C9C000002001210090CDE9010103460A46B94903903B2053F0AAF8002001210090CDE9010103460A46B44903903C2053F09EF800200121CDE9000103460A46CDE90210FD
:40CA0000AE493D2053F092F800200121CDE9000103460A46CDE90210A9493E2053F086F8002000900190029003460122A54903903F2053F07BF801200021009101910B46DF
:40CA40000246CDE90210A049402053F06FF80020009001900290034602229C490390412053F064F800200090019002900346022297490390422053F059F800200090019011
:40CA800002900346012293490390432053F04EF80020009001900290034601228E490390442053F043F80020009001900290034601228A490390452053F038F80020009065
:40CAC000019002900346012285490390462053F02DF8002002220092CDE90120034681490390472053F022F8002001210090CDE9010103460A467C490390482053F016F82D
:40CB000000200222CDE90002029003460246774903904A2053F00AF800200222CDE90002029003460246724903904B2052F0FEFF0020009001900290034602466D49039010
:40CB40004C2052F0F3FF002002220092CDE901200346694903904D2052F0E8FF002002220092CDE901200346644903904E2052F0DDFF01200021009101910B460246CDE9CE
:40CB800002105F494F2052F0D1FF01200021009101910B460246CDE902105A49502052F0C5FF00200090019002900346032256490390512052F0BAFF0020009001900290A9
:40CBC0000346032251490390522052F0AFFF0020009001900290034603224D490390532052F0A4FF00213748007852F025FF00213548007852F020FF00214648007852F018
:40CC00001BFF01214448007852F016FF00213448007852F011FF00213948007852F00CFF00213848007852F007FF01213B48007852F002FF01213A48007852F0FDFE012153
:40CC40003848007852F0F8FE01211248007852F0F3FE01211148007852F0EEFE00213248007852F0E9FE00210B48007852F0E4FE00210B48007852F0DFFE1FBD52050010A2
:40CC80006F0500107D0500107C05001064050010650500107405001075050010760500107705001053050010540500105505001078050010560500105705001058050010A4
:40CCC000590500107A0500107905001071050010700500107E0500107F05001080050010810500105B0500105A0500108205001083050010850500105C0500105D050010C1
:40CD00008705001088050010890500108A0500108B05001066050010670500106D0500106E05001072050010730500101FB5002000900190029003460246FE49039001209F
:40CD400052F0F4FE002000900190029003460246F8490390022052F0E9FE002000900190029003460246F3490390032052F0DEFE002000900190029003460246ED4903905B
:40CD8000042052F0D3FE002000900190029003460246E8490390052052F0C8FE002000900190029003460246E2490390062052F0BDFE002000900190029003460246DD4918
:40CDC0000390072052F0B2FE002000900190029003460246D7490390082052F0A7FE002000900190029003460246D2490390092052F09CFE002000900190029003460246E6
:40CE0000CC4903900A2052F091FE002000900190029003460246C74903900B2052F086FE002000900190029003460246C14903900C2052F07BFE0020009001900290034653
:40CE40000246BC4903900D2052F070FE002000900190029003460246B6490390112052F065FE002000900190029003460246B1490390122052F05AFE002000900190029099
:40CE800003460246AB490390172052F04FFE002000900190029003460246A6490390182052F044FE002000900190029003460246A0490390192052F039FE0020009001901F
:40CEC0000290034602469B4903901B2052F02EFE002000900190029003460246954903901C2052F023FE002000900190029003460246904903901F2052F018FE0020009064
:40CF000001900290034602468A490390202052F00DFE00200090019002900346024685490390212052F002FE0020009001900290034602467F490390222052F0F7FD0020AB
:40CF4000009001900290034602467A490390232052F0ECFD00200090019002900346024674490390242052F0E1FD0020009001900290034602466F490390252052F0D6FD88
:40CF800000200090019002900346024669490390262052F0CBFD00200090019002900346024664490390272052F0C0FD0020009001900290034602465E490390282052F066
:40CFC000B5FD00200090019002900346024659490390292052F0AAFD002000900190029003460246534903902A2052F09FFD0020009001900290034602464E4903902B2020
:40D0000052F094FD002000900190029003460246484903902C2052F089FD002000900190029003460246434903902D2052F07EFD0020009001900290034602463D49039077
:40D040002E2052F073FD002000900190029003460246384903902F2052F068FD00200090019002900346024632490390302052F05DFD0020009001900290034602462D490A
:40D080000390312052F052FD00200090019002900346024627490390322052F047FD00200090019002900346024622490390332052F03CFD00200090019002900346024628
:40D0C0001C490390342052F031FD00200090019002900346024617490390352052F026FD00200090019002900346024611490390362052F01BFD0020009001900290034646
:40D1000002460C490390372052F010FD00200090019002900346024606490390382052F005FD0020009001900290034602460149039001E045050010392052F0F7FC00200D
:40D1400000900190029003460246FE4903903A2052F0ECFC002000900190029003460246F84903903B2052F0E1FC002000900190029003460246F34903903C2052F0D6FCB8
:40D18000002000900190029003460246ED4903903D2052F0CBFC002000900190029003460246E84903903E2052F0C0FC002000900190029003460246E24903903F2052F095
:40D1C000B5FC002000900190029003460246DD490390402052F0AAFC002000900190029003460246D7490390412052F09FFC002000900190029003460246D2490390422050
:40D2000052F094FC002000900190029003460246CC490390432052F089FC002000900190029003460246C7490390442052F07EFC002000900190029003460246C1490390BE
:40D24000452052F073FC002000900190029003460246BC490390462052F068FC002000900190029003460246B6490390472052F05DFC002000900190029003460246B1493A
:40D280000390482052F052FC002000900190029003460246AB490390492052F047FC002000900190029003460246A64903904A2052F03CFC002000900190029003460246DC
:40D2C000A04903904B2052F031FC0020009001900290034602469B4903904C2052F026FC002000900190029003460246954903904D2052F01BFC0020009001900290034676
:40D300000246904903904E2052F010FC0020009001900290034602468A4903904F2052F005FC00200090019002900346024685490390502052F0FAFB0020009001900290C2
:40D340000346032280490390512052F0EFFB0020009001900290034603227C490390522052F0E4FB00200090019002900346032277490390532052F0D9FB1FBD1FB5FFF757
:40D38000D5FC00200CE00021724A02EB001292681170704A02EB0012D2681170411CC8B25428F0DB52F034F952F032FA012102208EF0A3FB0020009001900290034601222B
:40D3C00065490390162052F0B1FB002001210090CDE9010103460A46604903901E2052F0A5FB002001210090CDE9010103460A465B4903901A2052F099FB52F0FDF9FF2880
:40D4000025D052F0D1FE0E281FD2DFE800F01E070D080E110F10121314150C0900BF00BFFFF7AFF812E000BF00BF00BF00BF00BF00BF00BF00BF00BF52F0E1F910B1FEF797
:40D440000DFE01E0FEF717FB00E000BF00BF1FBD10B500204349087055F0C2F8FA2055F031F9FFF78BFFEAF777FF002211463E48DFF8F8C000DF002010BD38B50446002581
:40D4800060680090009D206880F3088800BFA84738BD10B501203349087055F0E3F83149486001208EF0DAF91CE061208EF078F978B145F255502E4908600120486040F66C
:40D4C000B83088604CF6CC40086002202549087008E02449486855F003F9642802D90320204908701F4800780128DED010BD10B572B66FF00400FEF7AFFA6FF00100FEF727
:40D50000ABFA4FF0FF30FEF7A7FA0420FEF7A4FA0520FEF7A1FA0620FEF79EFA0720FEF79BFA0820FEF798FA0920FEF795FA0A20FEF792FA0B20FEF78FFA0C20FEF78CFA1B
:40D540000D2017E045050010890500108A0500108B0500104C7B0F086205001063050010660500103801002031A3020855A70C0800300040FEF770FA0E20FEF76DFA0F2039
:40D58000FEF76AFA1020FEF767FA1120FEF764FA1220FEF761FA1320FEF75EFA1420FEF75BFA1520FEF758FA1620FEF755FA1720FEF752FA1820FEF74FFA1920FEF74CFA30
:40D5C0001A20FEF749FA1B20FEF746FA1C20FEF743FA1D20FEF740FA1E20FEF73DFA1F20FEF73AFA2020FEF737FA2120FEF734FA2220FEF731FA2320FEF72EFA2420FEF7D8
:40D600002BFA2520FEF728FA2620FEF725FA2720FEF722FA2820FEF71FFA2920FEF71CFA2A20FEF719FA2B20FEF716FA2C20FEF713FA2D20FEF710FA2E20FEF70DFA2F2038
:40D64000FEF70AFA3020FEF707FA3120FEF704FA3220FEF701FA3320FEF7FEF93420FEF7FBF93520FEF7F8F93620FEF7F5F93720FEF7F2F93820FEF7EFF93920FEF7ECF956
:40D680003A20FEF7E9F93B20FEF7E6F93C20FEF7E3F93D20FEF7E0F93E20FEF7DDF93F20FEF7DAF94020FEF7D7F94120FEF7D4F94220FEF7D1F94320FEF7CEF94420FEF781
:40D6C000CBF94520FEF7C8F94620FEF7C5F94720FEF7C2F94820FEF7BFF94920FEF7BCF94A20FEF7B9F94B20FEF7B6F94C20FEF7B3F94D20FEF7B0F94E20FEF7ADF94F2043
:40D70000FEF7AAF95020FEF7A7F95120FEF7A4F96FF0040000F02AF96FF0010000F026F94FF0FF3000F022F9042000F01FF9052000F01CF9062000F019F9072000F016F947
:40D74000082000F013F9092000F010F90A2000F00DF90B2000F00AF90C2000F007F90D2000F004F90E2000F001F90F2000F0FEF8102000F0FBF8112000F0F8F8122000F07C
:40D78000F5F8132000F0F2F8142000F0EFF8152000F0ECF8162000F0E9F8172000F0E6F8182000F0E3F8192000F0E0F81A2000F0DDF81B2000F0DAF81C2000F0D7F81D2017
:40D7C00000F0D4F81E2000F0D1F81F2000F0CEF8202000F0CBF8212000F0C8F8222000F0C5F8232000F0C2F8242000F0BFF8252000F0BCF8262000F0B9F8272000F0B6F821
:40D80000282000F0B3F8292000F0B0F82A2000F0ADF82B2000F0AAF82C2000F0A7F82D2000F0A4F82E2000F0A1F82F2000F09EF8302000F09BF8312000F098F8322000F022
:40D8400095F8332000F092F8342000F08FF8352000F08CF8362000F089F8372000F086F8382000F083F8392000F080F83A2000F07DF83B2000F07AF83C2000F077F83D2016
:40D8800000F074F83E2000F071F83F2000F06EF8402000F06BF8412000F068F8422000F065F8432000F062F8442000F05FF8452000F05CF8462000F059F8472000F056F840
:40D8C000482000F053F8492000F050F84A2000F04DF84B2000F04AF84C2000F047F84D2000F044F84E2000F041F84F2000F03EF8502000F03BF8512000F038F862B610BD3F
:40D9000000BFBFF34F8F1F48006800F4E0601E490843001D1B490860BFF34F8F00BF00BF00BFFDE74AF6AA201849086070472DE9FC4106460C4617469846089D002000903E
:40D9400001902078B0280DD16078102802D0112805D103E0142006F0D2FA01E000E000BF00BF00E000BF00BFBDE8FC81002807DB00F01F0201219140054A430942F8231029
:40D98000704700000CED00E00000FA050030004080E200E0F94880ED000A704710B52DED028B0446B0EE408A0F2C43D2DFE804F0090B0C0D100E42080A0F1539301E27001D
:40D9C00000BF00BF00BF00BF00BF00BF00BF00BF0021EB4816F061F92CE00121E84816F05CF99FEDE80AFFF7D5FF23E09FEDE50AFFF7D0FF0421E24816F04FF91AE09FED14
:40DA0000E10AFFF7C7FF0321DD4816F046F911E0B0EE480AFFF7BEFF0121D94816F03DF908E0B0EE480AFFF7B5FF0221D44816F034F900BF00BFBDEC028B10BD70B50446BA
:40DA4000F5F7C0FA84ED010A9AF0FDFF84ED020ACD4848F059FD84ED030AF8F7F8F90546F7F7EFFA84ED040A04F1180029F071F970BD38B504466946C14816F0ADF818B1BF
:40DA80002146009816F017F838BDC04880ED000A704770B52DED028B0446F0EE408A0F2C3CD2DFE804F0090B0C0D1A0E3B080A19101B0F11330000BF00BF00BF00BF00BF71
:40DAC00000BF00BF00BF00BF9FEDAE0AFFF7DDFF0020FFF7CEFF21E000BF00BFB0EE680AFFF7D3FF9AF0AFFFB0EE408AB0EEC80ADFEDA70AB4EEE00AF1EE10FA01DD0120D9
:40DB000000E000200546FFF7B4FF07E09FED9D0AFFF7BBFF0120FFF7ACFF00BF00BFBDEC028B70BD70B52DED028B044600250120F8F73EF948B10120F7F783FAF0EE408AD5
:40DB40000120F7F76BFAB0EE408AEEF743FB48B9002084F878068F49087054F083FD8E49086032E0B0EEE80ADFED8C0AB4EEE00AF1EE10FA08D2B0EEC80ADFED890AB4EE74
:40DB8000E00AF1EE10FA05D3F8F7D9FA10B98148007878B1022084F878062F257E48006854F09EFD41F2883188420ED30120794908700AE0012084F878063025002075491E
:40DBC000087054F04FFD7449086094F8790694F8781688420BD094F8780684F879061A20EAF7D3FC1DB100212846F0F79FFDBDEC028B70BD70B50446F5F7E4F984ED040A45
:40DC0000F8F725F90546F8F7C3F884ED030AF8F71EF90546F7F702FA84ED010AF8F717F90546F7F70EFA84ED000A70BD70B504465C4890F84054102D7DD2DFE805F07CF8DA
:40DC400008437DF7F6F5F4F3F2F1090AF0EF00BF00BF9FED550A84ED060A9FED540A84ED070A9FED530A84ED080A9FED520A84ED090A9FED4A0A84ED0A0A9FED4F0A84ED55
:40DC80000B0A9FED4E0A84ED0C0A9FED4D0A84ED0D0A9FED4C0A84ED0E0A9FED4B0A84ED0F0A9FED4A0A84ED100A9FED490A84ED110A9FED480A84ED120AB5EE000A84ED44
:40DCC000130A91E19FED440A84ED060A9FED430A84ED070A9FED310A84ED080A9FED400A84ED090A9FED3F0A84ED0A0A9FED3E0A84ED0B0A9FED3D0A84ED0C0A9FED3C0A5B
:40DD000084ED0D0A9FED3B0A84ED0E0A9FED3A0A84ED0F0A9FED390A84ED100A9FED380A84ED110A9FED370A84ED120A9FED360A84ED130A58E11EE1F8F7C2FD40B9F8F771
:40DD4000A8FD28B9F8F7B5FD10B9F8F7AAFD20B19FED2E0A84ED060A03E09FED2D0A84ED060A9FED2A0A84ED070A9FED2A0A84ED080A9FED290A84ED090A59E004010010CA
:40DD8000604F001000000000986C0220FC0000108FC3643DF8000010100100109A99993E39FA0E3D602A0020EC51183F46B6F33E5C8FC23EC3F5A83E295C8F3E713D8A3E12
:40DDC00014AE873EDD24863EB81E853E9318843E6F12833E2506813E713D0A3F83C0CA3E5C8F823EEDD46C3E2366563E24ED463E74B73B3EC329333EA6422C3E0D6F263E68
:40DE000006A0213E707C1D3E9A99193E9A99193FCDCC4C3D8FC2F53E3D0AD73E32E0A5E031E0A5E0A3E0A0E066E0A2E0A2E028E09FEDFE0A84ED0A0A1FED220A84ED0B0A26
:40DE40001FED2A0A84ED0C0A1FED250A84ED0D0A1FED230A84ED0E0AB5EE000A84ED0F0A9FEDF30A84ED100A9FEDF20A84ED110A9FEDF10A84ED120A9FEDF00A84ED130ACF
:40DE8000B2E000BF00BF9FEDEE0A84ED060A9FEDE70A84ED070A9FEDEB0A84ED080A9FEDEA0A84ED090A9FEDE90A84ED0A0A9FEDE80A84ED0B0A9FEDE70A84ED0C0A9FEDAE
:40DEC000E60A84ED0D0A9FEDE50A84ED0E0A9FEDE40A84ED0F0A9FEDE30A84ED100A9FEDE20A84ED110A9FEDE10A84ED120A9FEDE00A84ED130A77E01FED3C0A84ED060A68
:40DF00001FED3E0A84ED070A1FED3E0A84ED080A1FED3F0A84ED090A9FEDC40A84ED0A0A1FED5C0A84ED0B0A1FED640A84ED0C0A1FED5F0A84ED0D0A1FED5D0A84ED0E0A8A
:40DF4000B5EE000A84ED0F0A9FEDB90A84ED100A9FEDB80A84ED110A9FEDB70A84ED120A9FEDB60A84ED130A3EE000BF00BF00BF00BF00BF00BFB7EE000A84ED060AB7EE95
:40DF8000000A84ED070AB7EE000A84ED080AB7EE000A84ED090AB7EE000A84ED0A0AB7EE000A84ED0B0AB7EE000A84ED0C0AB7EE000A84ED0D0AB7EE000A84ED0E0AB7EEBD
:40DFC000000A84ED0F0AB7EE000A84ED100AB7EE000A84ED110AB7EE000A84ED120AB7EE000A84ED130A00BF00BFB0EE000A84ED140AB7EE000A84ED150AB7EE000A84ED8B
:40E00000160AB7EE000A84ED170AB7EE000A84ED180AB7EE000A84ED190AB7EE000A84ED1A0AB7EE000A84ED1B0AB7EE000A84ED1C0AB7EE000A84ED1D0AB7EE000A84EDC4
:40E040001E0AB7EE000A84ED1F0AB7EE000A84ED200AB7EE000A84ED210A70BD2DE9F04104460D4617469846069E062D11D1012C0DD18049D1F89801042154F059FC7D48DC
:40E08000D0F898110420DFF8F0C100DF00BF00BF00BF00BFBDE8F0812DED048B4FF6FF760121744880F89C110020744981F878061FEDCC0A01F5806080EDA00ABFEE000A92
:40E0C0006F4880ED000A00206E49088090216E48A5F09FFD03F0F9FB6848FC306B490860001D6B490860001D6A490860001D6A490860001D6949086000F26C506849086075
:40E10000083068490860DFF8A0C100DF0746CD231122042154F092FBDFF88CC100DF0746042154F0C7FBDFF880C100DF074639460220DFF844C100DF04214E4880F89C1116
:40E1400000230622AFF2EB0158488FF0B4FA00BF002231464CF20700DFF854C100DF85B2012DF5D0DFF84CC100DF044604F4004028B14FF4167603213E4880F89C1104F4B4
:40E18000804028B14FF6FF7604213A4880F89C1104F00200002847D00121384880F81011FCF7B0F980464146434813F008F8434890F88675022F04D0032F08D0042F12D126
:40E1C0000BE03F483F4908603F48486015E03F483C4908603E4848600FE03E48394908603D48486009E03D49244847F0EDF93C48344908603B48486000BF00BF314801687F
:40E200001E4888471D48FFF711FD9FED370A9AF0BEFE364880ED000A35482A49C860354888600846816867E08BE00000A470BD3E8FC2753ED7A3703E1F856B3ED578693E56
:40E24000CDCCCC3E7B14AE3E52B89E3E745F8E3E28636C3E4E9D473E97FD2A3E520E163EF967063E07EAF43DC6BEE43D08ACDC3D3D0AD73DF8FF0020099F0C08B823002045
:40E28000EC0000100C01001028230020C4000010C8000010CC000010D0000010D4000010DC000010D800001031AB0C08986C0220699F0C08B19E0C0858490010602A0020CA
:40E2C000B55706084C2A0020BB580608A72B0608C32D0608B13A0608553D0608FC000010593106082F56060844D8F03BE00000105F4E0608A94C0608FE488847FE4890F8C7
:40E300005308022804D0FC4890F85308032801D1012000E000200146F84848F041FDF64890F85308032806D1F34890F81208012801D0012000E000200146F04848F0E1FE91
:40E3400000BF04F00100002870D0EA48FC30FFF751FCE848FFF7E6FBE948EA494268E5489047E948EDF7CBFF0746E648D0ED000AB0EE600A3846FFF78CFBFBF7FAFF28B3DD
:40E38000F7F7EEFE8046F4F71DFEF0EE408AEDF737FE074612F017F8B0EE408AD54890F8780608B1012000E000200346D14890ED431AD0ED400A90ED3F0A42463946D34808
:40E3C0000078F0EE481A04F081F92DE0F7F7C8FE8046F4F7F7FDB0EE409AEDF711FE074611F0F1FFB0EE408AF7F731FD8146F7F7CFFCF0EE408ABF4890F8780608B1012055
:40E4000000E000200346BB48D0ED431A90ED401AD0ED3F0A42463946BC480078B0EE482AB0EE680A03F05BFB99F0A4FE04F0040000283FF48DAEB648FFF700FBAE4890F887
